:020000040040BA
:10400000A05000201DD4400019D4400031F94000D8
:1040100019D4400019D4400019D440000000000019
:10402000000000000000000000000000C1D74000B8
:1040300019D440000000000021D8400085D840007D
:1040400019D4400019D4400019D4400019D44000BC
:1040500019D4400019D4400019D4400000000000D9
:1040600019D44000F1F8400000000000E5AF400026
:10407000F9AF400029CC400019D4400019D44000C9
:1040800019D4400019D4400039CC400019874000B1
:1040900005F9400019D4400019D44000214C4000DB
:1040A00019D4400019D4400019D4400019D440005C
:1040B00019D44000A94A400019D440000000000073
:1040C00000000000000000000000000000000000F0
:1040D00000000000000000000000000000000000E0
:1040E00000000000000000000000000000000000D0
:1040F00000000000000000000000000019D4400093
:10410000F9C0400019D44000000000000000000089
:10411000000000000000000000000000000000009F
:10412000000000000000000000000000000000008F
:10413000000000000000000000000000000000007F
:10414000000000000000000000000000000000006F
:104400003C10010010B5054C237833B9044B13B1AF
:104410000448AFF300800123237010BDA80C0020D6
:1044200000000000A44341000C4B43B10C480D496F
:1044300010B5AFF300800C48036823B910BD0A48DB
:10444000036833B97047094B002BF7D0BDE8104023
:104450001847064B002BF5D0184700BF000000009E
:10446000A4434100AC0C0020A44341000000000024
:104470000120704770470120704700207047704747
:1044800001207047014B1878704700BFCC0C00200A
:104490007047000058B908B5054B1B78012B00D0B8
:1044A00008BD044B1B68002BFAD09847F8E770470B
:1044B000D00C0020C40C002008B50C4B9847C378E2
:1044C0000B4A1370012B0CD101220A4B1A700022E7
:1044D000094B1A80094B9847094B1B681BB1984739
:1044E00001E0084B9847012008BD00BF2DAC4000FB
:1044F000CC0C0020D00C0020CE0C0020D5F84000C1
:10450000C40C0020E1F8400008B5054B1B78012BD6
:1045100000D008BD0022034B1A70034B9847F8E700
:10452000CC0C0020D00C0020E1F8400010B582B087
:10453000074B00930B46024600218420054CA04700
:1045400018B9054A13680133136002B010BD00BFEB
:104550009544400031C84000C80C0020014B186051
:10456000704700BFC40C00202DE9F0474FF400460F
:10457000BF4B5E600B20BF4CA0470C20A047BE4B3A
:104580004FF0400CC3F810C0C3F8A0C0C3F834C04B
:104590004FF0807EC3F810E0C3F8A0E0C3F834E029
:1045A000B64A01271761C2F8A0705763022414614C
:1045B000C2F8A04054631C61C3F8A0405C631F664E
:1045C000C3F890705F655F62C3F88070196F3943FC
:1045D0001967596F21F0010159675F604FF480310D
:1045E0001966C3F8901059655962C3F88010186FA6
:1045F00008431867586F20F48030586759601C6171
:10460000C3F8A0405C6304205861C3F8A00058665A
:10461000C3F8900058655862C3F88000196F21F004
:1046200004011967596F21F00401596718211966AF
:10463000C3F8901059655962C3F880101D6F25F0BA
:1046400018051D675D6F25F018055D675960082521
:104650001D66C3F890505D655D62C3F88050196FA8
:1046600021F008011967596F21F0080159675D6051
:1046700010211966C3F8901059655962C3F880106B
:10468000D3F8708028F01008C3F87080D3F87480D5
:1046900028F01008C3F8748059604FF48028C3F8DC
:1046A0001480C3F8A0804FF02009C3F81490C3F819
:1046B000A090C3F810C0C3F8A0C0C3F834C0C3F8BA
:1046C00010E0C3F8A0E0C3F834E01761C2F8A070AE
:1046D00057631461C2F8A04054634FF4007CC3F8E0
:1046E00060C0C3F890C0C3F854C0C3F824C0C3F876
:1046F00080C01C6F44EA0C041C675C6F24F40074D7
:104700005C67C3F804C04FF480641C66C3F8904033
:104710005C655C62C3F880401F6F27431F675F6F53
:1047200027F480675F675C604FF4006EC3F810E0A9
:10473000C3F8A0E0C3F834E04FF400275F61C3F88A
:10474000A0701F66C3F890705F655F62C3F88070E9
:104750001F6F27F400271F675F6F27F400275F672D
:104760004FF480175F61C3F8A0701F66C3F89070A4
:104770005F655F62C3F880701F6F27F480171F6743
:104780005F6F27F480175F674FF480575F61C3F84E
:10479000A0705F66C3F890705F655F62C3F8807059
:1047A0001F6F27F480571F675F6F27F480575F677D
:1047B0004FF400575F61C3F8A0704FF480775761E2
:1047C000C2F8A0704FF48048C3F86080C3F89080AE
:1047D000C3F85080C3F82480C3F88080D3F870A059
:1047E0002AF4804AC3F870A0D3F874A02AF4804A4F
:1047F000C3F874A0C3F81080C3F8A080C3F8308059
:104800005E61C3F8A0604FF400365E61C3F8A0603B
:104810001066C2F8900050655062C2F88000166FB2
:1048200026F004061667566F26F004065667506099
:104830001566C2F8905055655562C2F88050106FE9
:1048400020F008001067506F20F008005067556096
:104850000B4DD5F8140140F03000C5F8140151613A
:10486000C2F8A0105166C2F890105165516209E07B
:1048700050140E4061D14000000E0E4000100E405A
:1048800000020E40C2F88010116F21F01001116774
:10489000516F21F010015167C2F81090C2F8A0903A
:1048A000C2F83490C2F810C0C2F8A0C0C2F830C03C
:1048B0004FF400015961C3F8A0105966C3F8901075
:1048C00059655962C3F88010196F21F40001196706
:1048D000596F21F400015967C2F860E0C2F890E016
:1048E000C2F854E0C2F824E0C2F880E0116F21F46D
:1048F00000611167516F21F400615167C2F804E053
:104900001466C2F8904054655462C2F88040116F3A
:1049100021F480611167516F21F480615167546007
:104920001F66C3F890701F655F62C3F880701A6FCE
:1049300022F480721A675A6F22F480725A671F61DC
:10494000C3F8A0701F63BDE8F08700BF08B5034B34
:1049500053F8203003B1984708BD00BF281000204D
:1049600010B582B0036B0193002400E00134172CD2
:1049700009D8064B53F82420019B1A42F6D0204652
:10498000034B9847F2E702B010BD00BFAC364100C0
:104990004D49400000230360064A4260064A826097
:1049A0004FF48022C2600222027442748374C37482
:1049B000037570470000DC05808D5B00036C1943B4
:1049C0000164704710B58B7C23B34FF000434A68F5
:1049D0008C686400B2FBF4F2013A120292B2134303
:1049E0000A7C120602F0706213434A7C120702F03E
:1049F00040521343CA6813434360CB7C63B14FF00A
:104A000080730A7D52B90022134303640968054B81
:104A1000984710BD0023DAE70023F2E74FF4801235
:104A2000F2E700BFBD49400008B5036B13F0807F7B
:104A300001D0192008BD01230360064B98470023CD
:104A400004E00021044A42F823100133172BF8D95F
:104A5000002008BDC549400028100020B1F1FF3FEB
:104A600004D0044B53F82130436270474FF0FF33BA
:104A700043627047AC36410010B5084C44F8212021
:104A8000074A4FF00054C2F880411B01DBB282F8A4
:104A90001D331460034B984710BD00BF2810002041
:104AA00000E100E05D4A400008B50248024B98472B
:104AB00008BD00BF008003406149400010B51720C9
:104AC000234CA0471820A047224B4FF480321A668F
:104AD000C3F890205A655A62C3F88020196F1143B9
:104AE0001967596F21F4803159675A6001225A665B
:104AF000C3F890205A655A62C3F88020196F114399
:104B00001967596F21F0010159675A60A3F52063B5
:104B100040F21262DA644FF400621A600E4B0F4AE0
:104B20005A6041225A62052119600D4A5A644FF4B5
:104B3000F572DA6500229A6519640A4B1A700A4BFD
:104B40004FF400021A60702283F8172310BD00BFD3
:104B500061D14000000E0E40000001400406090033
:104B600001C4000A8C10002000E100E010B54FF4F1
:104B70000002124BC3F88020BFF34F8FBFF36F8F3B
:104B80000F4B4FF480321A66C3F890205A655A6270
:104B9000C3F88020196F21F480311967596F21F40F
:104BA000803159671A601A61C3F8A0205A63172030
:104BB000044CA0471820A04710BD00BF00E100E052
:104BC000000E0E40B5D14000642800D964200F4A81
:104BD000D36D03FB00F30E49A1FB03135B0993653F
:104BE00048B10A4B5A6C22F040625A645A6C42F047
:104BF00080625A6470471346526C22F040625A64D5
:104C00005A6C42F000625A64704700BF00000140D5
:104C10001F85EB51014B1888704700BF9010002092
:104C20000F4B1B6A13F0010F06D000220D490A70CA
:104C30000D490A600D490A6013F0400F0ED00122A1
:104C4000084B1A70064B9A69094BB3FBF2F3064AFC
:104C50001360C3EB03139A00044B1A60704700BF44
:104C6000000001408C1000208810002090100020CF
:104C70001F1A0500014B1870704700BFBC000020D0
:104C8000064B1B7823B94FF40062054B1A6370473B
:104C90004FF40062024B5A63704700BFBC00002013
:104CA000000E0E40064B1B7823B94FF40062054BF3
:104CB0005A6370474FF40062024B1A63704700BF9B
:104CC000BC000020000E0E402DE9F04186B00F46DA
:104CD00016469846B8B9344B9847044600250495C3
:104CE00098238DF8043001238DF805308DF8065097
:104CF00002238DF8083005AB03938DF8075020464A
:104D00002A4B98470EE02A4B98470446E6E7204690
:104D1000284B9847002044E09DF8153008F80530EE
:104D20000135EDB2B54238D28DF814708DF81550BA
:104D300000238DF80630322201A920461E4B9847E9
:104D4000A379DBB2022B0BD020461C4B98473222B2
:104D500001A92046184B9847A379DBB2022BD6D184
:104D600001238DF80630322201A92046124B9847C4
:104D7000A379DBB2022BCFD02046104B98473222CA
:104D800001A920460C4B9847A379DBB2022BC3D074
:104D90002046084B9847002003E02046054B9847E3
:104DA000012006B0BDE8F081C5F84000ED6A400082
:104DB000CDF84000016B4000196B4000C96C400009
:104DC0002DE9F04186B00C4617469846D8B9264BD7
:104DD000984705460026049698238DF80430012351
:104DE0008DF8053002238DF8063003238DF8083046
:104DF00005AB03938DF807408DF8156028461B4BD3
:104E00009847344605E01A4B98470546E2E70134D7
:104E1000E4B2BC4221D28DF8144018F804308DF869
:104E20001630322201A92846124B98470646AB7924
:104E3000DBB2022BEBD028460F4B9847322201A958
:104E400028460C4B98470646AB79DBB2022BDED0E6
:104E500028460A4B9847002602E02846074B984709
:104E6000304606B0BDE8F081C5F84000ED6A40006C
:104E7000CDF84000196B4000C96C4000016B400048
:104E8000F8B506460D461746344BAA221A70112271
:104E90005A700222F021324CA047012801D0002094
:104EA000F8BD2C0AEDB22D4B1C705D709C70DD704E
:104EB0001C715D7100229A719022DA7167B18222B1
:104EC0001A72264B0922C2213046254FB8470128C5
:104ED00006D001280BD0F8BD0222204B1A72F0E751
:104EE0001E4B0922C22130461E4EB047F1E71B4B34
:104EF0001B789C4201D00020F8BD184B9B789C4247
:104F000001D00020F8BD154B1B799C4201D0002038
:104F1000F8BD124B5B789D4201D00020F8BD0F4BCD
:104F2000DB789D4201D00020F8BD0C4B5B799D429F
:104F30000BD10A4B9B7953B9084BDB79902B08D1E5
:104F4000064B1B7A022B06D1F8BD0020F8BD0020CD
:104F5000F8BD0020F8BD0020BDE700BF9410002080
:104F6000C14D4000C94C400010B50022054B1A70DD
:104F700029B91121034B0122034CA04710BD102178
:104F8000F8E700BF94100020C14D400070B5044602
:104F90000022104B1A700D4639B129210D4B012208
:104FA00020460D4EB04715B970BD2821F6E7094DD2
:104FB000AA232B7011236B702B460222F02120466E
:104FC000B047FF232B702B460122C0212046B0475B
:104FD000EAE700BF94100020C14D400010B539B978
:104FE0000022044B1A7001223621034CA04710BD49
:104FF0000322F6E794100020C14D400038B5054665
:105000000C4BAA221A7012225A700222F0210A4C6A
:10501000A047012801D0002038BD064B0322BF2144
:105020002846064CA047012801D0002038BD014B7E
:10503000987838BD94100020C14D4000C94C400004
:1050400038B50D46094B0E228421094CA047012892
:1050500001D0002038BD054B186859689A6828604F
:105060006960AA609B89AB810E2038BD9410002036
:10507000C94C400010B50B462C227021014CA047B2
:1050800010BD00BFC14D40002DE9F04182B00023AA
:105090008DF80730013905292BD8DFE801F0070525
:1050A000030C0E10154D02E0154D00E0154D804625
:1050B000012000240FE0144DF9E7144DF7E7144DDB
:1050C000F5E70DF1070302464046124EB0473C4457
:1050D000E4B20134E4B201280CD123462F5D4FB174
:1050E000621CA95C012FECD902332B44781EC0B29C
:1050F000E9E7002002B0BDE8F08100BF8037410041
:1051000018394100B03941000C37410038384100AE
:10511000A8384100C14D400008B50621014B984711
:1051200008BD00BF8950400010B5274900238B728D
:10513000CB720B7340F2DC528A806422CA800B80EF
:1051400021F8083F0620214B98470B20204B984719
:1051500080B90C201E4B984788B900221A4B5A8000
:105160001C4B984701211C4B984701280CD0164B2B
:10517000987A10BD19490B20144B9847E9E7184954
:105180000C20124B9847E8E701220F4B9A72114B03
:1051900098470521134B9847034650B10A4AD372EA
:1051A000002BE4D00B4B98470F4B9847064B588089
:1051B000DDE7084CA0470021074B9847A047032193
:1051C000084B98470346E9E7F4100020617440005B
:1051D00095744000CDF84000D1524000F8100020F6
:1051E000FA1000200155400091544000014B987A7C
:1051F000704700BFF410002008B5224B9B7A8BB992
:10520000214A13781F490888204921F813000133E7
:10521000DBB213700F2B02D900221B4B1A70002334
:105220001A4615E01A4B98471A4B9847154B1B899D
:10523000984203D80022134B1A80E1E7C01A114BA1
:105240001880DDE7114931F813100A440133DBB24D
:105250000F2BF7D912090B4B1B7B4BB109498B88DC
:10526000C9885B1A9A420CD80022064B1A7308BDF3
:1052700004498B88C9880B449A4202D30122014B0E
:105280001A7308BDF4100020D10C0020D4100020A7
:10529000CDF8400021544000014B187B704700BFFF
:1052A000F4100020014B1888704700BFF410002054
:1052B00008B5014B984708BDD155400008B5024BD1
:1052C0009847024B984708BDCDF84000D95540009B
:1052D00030B587B005460C4600238DF807307222A2
:1052E0008DF808208DF80B3001228DF809208DF8FB
:1052F0000C200DF10702049202228DF80A2005937A
:10530000434B9847322202A92846424B9847002C2B
:1053100043D1012402238DF80A3080238DF80B300D
:1053200001238DF807309C4244D08F238DF80B3039
:1053300003238DF80A30012C43D09DF8073003F089
:10534000F00343F005038DF8073002238DF80A308F
:10535000012C3DD0AA238DF80B3001238DF80730A6
:105360009C423CD007238DF80730F9238DF80B3091
:10537000012C3BD005238DF8073080238DF80B30AE
:10538000012C3AD02846244B9847012C3CD00022CF
:10539000224B1A70204607B030BDA8238DF80B3081
:1053A00001238DF80730322202A92846194B98476D
:1053B0000446AFE7322202A92846164B9847044616
:1053C000B3E7322202A92846124B98470446B4E7B5
:1053D000322202A928460F4B98470446BAE73222E8
:1053E00002A928460B4B98470446BBE7322202A984
:1053F0002846084B98470446BCE7322202A92846B3
:10540000044B98470446BDE70122044B1A70C1E7DC
:10541000ED6A4000196B4000016B4000D20C002087
:1054200030B587B004460023059301AB0493722383
:105430008DF8083001238DF809309C238DF80B304E
:1054400002238DF80C3003238DF80A300C4B98475B
:10545000322202A920460B4B9847054620460A4BAC
:105460009847012D04D00020084B187007B030BDBC
:105470009DF804009DF8053000EB032080B2F5E7AD
:10548000ED6A4000196B4000016B4000D20C002017
:1054900030B587B004460023059301AB0493722313
:1054A0008DF8083001238DF80930C0238DF80B30BA
:1054B00002238DF80C3003238DF80A300C4B9847EB
:1054C000322202A920460B4B9847054620460A4B3C
:1054D0009847012D04D00020084B187007B030BD4C
:1054E0009DF804009DF8053000EB032080B2F5E73D
:1054F000ED6A4000196B4000016B4000D20C0020A7
:10550000F0B587B00646002305930DF10703049319
:1055100072238DF8083001238DF80930D9228DF8D7
:105520000B208DF80C3002238DF80A304901C9B2E6
:1055300041F010018DF80710214B9847322202A943
:105540003046204B98470546D7238DF80B30212352
:105550008DF8073001280BD030461B4B9847DC23D1
:105560008DF80B3003238DF80A300024274608E01D
:10557000322202A93046134B98470546ECE7013426
:10558000A4B2012D18D1BFB9092C15D819200F4B81
:10559000984730460A4B9847322202A93046094BB9
:1055A000984705463046084B98479DF8073013F05A
:1055B000010FE4D00127E2E7384607B0F0BD00BF95
:1055C000ED6A4000196B4000016B400081E640002D
:1055D0000048704704110020A84BDB78032B00F231
:1055E0004081A64B1B793F2B00F23D81A34B5B7999
:1055F000072B00F23A81A14B9B79082B00F23781EF
:105600009E4B1B7A013BDBB2022B00F232819B4B9B
:105610005B7A032B00F22F81984B9B7A072B01D9E1
:105620000020704710B586B004460023059372230E
:105630008DF8083001238DF809300DF1070204922E
:105640008DF80C308E4B984780238DF80B30032358
:105650008DF80A30322202A920468A4B9847012849
:1056600017D1864B1B78D3B19DF8073043F0100358
:105670008DF8073002238DF80A30322202A9204625
:10568000804B9847012811D020467F4B9847002037
:1056900003E020467C4B9847002006B010BD9DF8E3
:1056A000073023F010038DF80730E3E782238DF8ED
:1056B0000B30724B5B788DF80730322202A92046FE
:1056C000704B9847012817D18D238DF80B3040235C
:1056D0008DF80730694B9B7813B148238DF807305C
:1056E000322202A92046674B9847012809D020465C
:1056F000654B98470020D0E72046634B9847002031
:10570000CBE78E238DF80B305C4AD3789B01DBB25C
:10571000127902F03F0213438DF80730322202A9BA
:105720002046584B9847012804D02046564B9847AE
:105730000020B2E78F238DF80B30504A53795B017C
:10574000DBB2927902F00F0213438DF80730322258
:1057500002A920464B4B9847012804D020464A4BCB
:105760009847002099E7A9238DF80B30434BDB794C
:105770008DF80730322202A92046424B9847012873
:105780000CD1AA238DF80B303C4B1B7A022B18D07E
:10579000032B1AD0012B06D000207EE720463A4B7F
:1057A0009847002079E78DF80730322202A9204679
:1057B000344B984701280CD02046334B98470020A3
:1057C0006BE702238DF80730EFE703238DF80730EE
:1057D000EBE7B3238DF80B30284B5B7A03F0030320
:1057E0008DF80730322202A92046264B984701281F
:1057F00004D02046244B984700204EE7D9238DF84B
:105800000B3003238DF80A30322202A920461D4BAB
:105810009847012804D020461B4B984700203CE7BE
:105820009DF8073003F0F80343F01003134A927A0F
:1058300002F0070213438DF8073002238DF80A3077
:10584000322202A920460F4B9847012804D0204657
:105850000D4B9847002020E720460B4B984701202E
:105860001BE7002070470020704700207047002091
:105870007047002070470020704700BF04110020CF
:10588000ED6A4000196B4000016B400000FB01F025
:10589000C0F3C71070470000F0B587B004460E464D
:1058A000234B9847002304938A238DF80430012367
:1058B0008DF805308DF808300DF117030393342768
:1058C0008DF8077002238DF8063033788DF8173085
:1058D000322201A92046174DA8478DF8077033786A
:1058E0008DF81730322201A92046A8478DF807709D
:1058F00033788DF81730322201A92046A847352386
:105900008DF8073073788DF81730322201A92046C0
:10591000A84736238DF80730B3788DF81730322238
:1059200001A92046A8472046034B984707B0F0BD81
:10593000ED6A4000196B4000016B4000F0B587B084
:105940000446002505958A238DF8083001268DF838
:1059500009608DF80C600DF107030493254B9847FF
:1059600055238DF807308DF80B5002238DF80A303F
:10597000322202A92046204DA84703238DF8073084
:105980008DF80B60322202A92046A8478DF80760E7
:1059900004238DF80B30322202A92046A8470723A2
:1059A0008DF8073030238DF80B30322202A92046C3
:1059B000A8470F278DF8077031238DF80B3032225E
:1059C00002A92046A8478DF8077032268DF80B6093
:1059D000324602A92046A8478DF8077033238DF878
:1059E0000B30324602A92046A8472046034B984771
:1059F00007B0F0BDED6A4000196B4000016B40003C
:105A0000F0B583B007460C46802900D980240C4BA2
:105A10001C700C4E214630780B4DA8478DF80400C1
:105A200021467078A8478DF805002146B078A84730
:105A30008DF8060001A93846044B984703B0F0BD25
:105A4000BD000020D40C00208D5840009958400023
:105A500010B5054B0C888A781C809A70034B197816
:105A6000034B984710BD00BFD40C0020BD000020A0
:105A7000015A400010B586B004468DF80810002386
:105A80000593E7238DF80B300DF1070304930123F1
:105A90008DF80C308DF8093003238DF80A3032224E
:105AA00002A90A4B9847012801D006B010BD9DF805
:105AB000073043F001038DF8073002238DF80A30D8
:105AC000322202A92046014B9847EEE7196B4000AD
:105AD00010B586B004468DF80810002305930DF12B
:105AE0000703049301238DF80C308DF80930062349
:105AF0008DF80B3003238DF80A30322202A9224B95
:105B000098479DF8073063F07F038DF80730022334
:105B10008DF80A30012818D000238DF807300C23A7
:105B20008DF80B30012816D00D238DF80B3001288D
:105B300017D00E238DF80B30012818D00F238DF8C5
:105B40000B30012819D006B010BD322202A9204620
:105B50000D4B9847E0E7322202A920460A4B9847AE
:105B6000E2E7322202A92046074B9847E1E73222BA
:105B700002A92046044B9847E0E7322202A92046BA
:105B8000014B9847DFE700BF196B400010B586B0A6
:105B900004468DF8081000230593E7238DF80B3099
:105BA0000DF10703049301238DF80C308DF80930B3
:105BB00003238DF80A30322202A90A4B98470128A4
:105BC00001D006B010BD9DF8073023F001038DF819
:105BD000073002238DF80A30322202A92046014BF9
:105BE0009847EEE7196B400070B504462022214B20
:105BF0001A630A20204B98472046204B98471021D3
:105C000020461F4EB047054612212046B0470646A3
:105C1000012D0ED0012E12D0012D16D0012E1AD03A
:105C20002046184B9847012D1BD0012E1DD0284629
:105C300070BD10212046144B98470546EAE7122113
:105C40002046114B98470646E6E7102120460F4BA9
:105C500098470546E2E7122120460C4B9847064636
:105C6000DEE701220A4B1A70DFE70122094B1A70A6
:105C7000DDE700BF00100E4081E64000ED6A400005
:105C8000755A4000016B4000D15A40008D5B4000C6
:105C9000D70C0020D80C002010B1034B18787047A7
:105CA000024B1878704700BFD80C0020D70C00209A
:105CB00030B587B004460D4600220592A8238DF822
:105CC000083001238DF809308DF80B200DF1070203
:105CD00004928DF80C3002238DF80A30124B98474D
:105CE000012D0ED0022D15D000238DF80730322261
:105CF00002A920460D4B984720460D4B984707B008
:105D000030BD03238DF80730322202A92046074B0D
:105D10009847F1E702238DF80730322202A9204686
:105D2000024B9847E8E700BFED6A4000196B40005E
:105D3000016B400030B587B072238DF8003001232D
:105D40008DF8013000238DF802308DF803300822E1
:105D50008DF8042004AA029203938DF81000C0F37A
:105D600007238DF81130C0F307438DF81230000E71
:105D70008DF813008DF81410C1F307238DF815303A
:105D8000C1F307438DF81630090E8DF81710084C33
:105D9000A047084B9847A04732226946064B9847D0
:105DA0000546A047054B9847284607B030BD00BFC1
:105DB000C5F84000ED6A4000196B4000016B4000DF
:105DC00030B587B00D4672238DF8043001238DF86D
:105DD000053000238DF806308DF8073004228DF849
:105DE000082005AA039204938DF81400C0F307233A
:105DF0008DF81530C0F307438DF81630000E8DF87E
:105E00001700184CA047184B9847A047322201A909
:105E1000164B98470446012808D0124B9847144B5C
:105E20009847012C0DD0204607B030BD01238DF8D6
:105E300006300C4B9847322201A90C4B9847044678
:105E4000EBE79DF814309DF8152003EB02239DF835
:105E5000162003EB02439DF8172003EB02632B602F
:105E6000E1E700BFC5F84000ED6A4000196B400053
:105E7000016B40002DE9F04E82B082468946934680
:105E80001BB11E46002501272FE00127012F40D01E
:105E9000012F49D0012F4DD0012F51D04FF40003D5
:105EA00001932F4B98470446012F4FD1019B13F4C8
:105EB000000F4BD00A9920462A4B984700284DD115
:105EC00001A92948294B98470746EDE7EA18B25C33
:105ED0004FEAC30E02FA0EF211440133DBB2A342C1
:105EE000F4D3012F0DD02544EDB228464D45CDD237
:105EF000A9EB0504042C28BF0424E4B200231946AE
:105F0000EDE700F1201000F58070194B9847074627
:105F1000E9E74FEA0A4101F4FE0101F500011248E8
:105F2000134B98470746B3E749461248104B98472A
:105F30000746AFE7594610480D4B98470746ABE771
:105F4000F2210E480A4B98470746A7E71FB90520DC
:105F500002B0BDE8F08E9DF80700F9E70620F7E7EC
:105F6000517140006971400010012000C15D400086
:105F7000355D40001801200014012000FC002000C5
:105F800010B584B00A4B93E8030002908DF80C1012
:105F90003223009302AB002205210120054CA047CB
:105FA000034610B90121044A1170184604B010BD0F
:105FB000483A4100755E4000D90C002070B5074D8D
:105FC0004FF480466E630A20054CA0472E6340F2D2
:105FD0001310A047034B984770BD00BF000E0E4042
:105FE00081E64000815F400030B583B00D4632232A
:105FF00000930023024604213120074CA0470446A9
:1060000010B1204603B030BD29460448044B9847E0
:106010000128F6D00524F4E7755E40002001200039
:10602000C15D400010B584B08DF80C100B0A8DF8DE
:106030000D300B0C8DF80E30090E8DF80F10322339
:10604000009303AB024604212120024CA04704B078
:1060500010BD00BF755E400008B5044B1B780BB146
:10606000002008BD024B984708BD00BFD90C002096
:10607000815F40002DE9F04383B059B1012904D07C
:106080000124204603B0BDE8F08340F65D0740F6EA
:10609000050503E040F2DD7740F2857580464FF05C
:1060A00000094C4601E0002CEBD1BD42E9D225F0BD
:1060B0000306002CF7D101A93046164B9847044639
:1060C0000028F0D1019B8DF80030C3F307228DF832
:1060D0000120C3F307428DF802201B0E8DF8033018
:1060E000E9B2F3B2C91AC9B2C1F10403BE1B9E42A0
:1060F00028BF1E46042E28BF0426F6B23246694445
:1061000008EB0900044B984735444E445FFA86F982
:10611000C9E700BFE95F4000C10D410028B1012877
:1061200001D000207047094800E0094800B583B05D
:1061300001A9084B984728B9019B13F4006F02D0BE
:10614000012000E0002003B05DF804FB40003500B2
:1061500040003100E95F400010B52DED028B82B0A8
:10616000044601A93548364B98470346F8B14BB36E
:10617000002B32D0002B3BD0DFED328A002B49D0F0
:106180009FED308A73B9DDED017AB8EE677AC8EE1B
:10619000077A9FED2D7A67EE877AFCEEE77A17EEA5
:1061A000902A6281184602B0BDEC028B10BD02A994
:1061B00051F8043D23801B0C63802448204B9847F2
:1061C0000346D4E702A951F8043DA3801B0CE380E9
:1061D0001F481B4B98470346CAE702A951F8043DE4
:1061E00003F01F0323721B48154B98470346C1E772
:1061F00002A951F8043DC3F3094308EE903AF8EEC2
:10620000688A9FED158A68EE888A14480C4B984777
:106210000346B3E702A951F8043DDBB208EE103A99
:10622000B8EE488A28EE888ADFED077A28EE278ABA
:106230000B48034B98470346A4E700BF30082200F1
:10624000E95F4000000000000000C842380822005A
:10625000540822000800200000401C4604082200C8
:106260001408220000B583B001A941F23070094B37
:106270009847034618B1184603B05DF804FB01992E
:1062800021F00601019141F23070034B984703461B
:10629000F1E700BFE95F40002560400030B583B002
:1062A00015460C4AA2FB01231B090F330093002360
:1062B00002461120084CA047044610B1204603B006
:1062C00030BD29460548064B98470128F6D00524DD
:1062D000F4E700BF1F85EB51755E400020012000F0
:1062E000C15D400010B582B096230093134602466C
:1062F0002020024CA04702B010BD00BF755E4000D8
:10630000072801D90120704710B584B08DF80C0022
:1063100030238DF80D3041F28833009303AB002217
:1063200002211420014CA04704B010BD755E40004E
:1063300010F0800F11D110B584B08DF80C0010232F
:106340008DF80D3041F28833009303AB0022022117
:106350001420034CA04704B010BD0120704700BFBB
:10636000755E4000F0B583B0032832D8DFE800F056
:106370000209050747F6F07604E0184E02E0184ED1
:1063800000E0184E002401273D4604E09CB10F2C8C
:1063900011D00134E4B20F2C13D801AA0121A019A5
:1063A000114B9847B8B9002DF0D09DF80430FF2B61
:1063B000ECD00025EAE79DF80430002BE9D1002756
:1063C000E7E717B11DB1002006E0002004E001203E
:1063D00002E0002000E0002003B0F0BDF0FF01006B
:1063E000F0FF0300F07F02009D62400070B582B0B4
:1063F00006460020114B984720B14FF4BE6500249B
:1064000023460BE001200D4B984718B9032318468B
:1064100002B070BD0A4DF2E70134E4B20E2CF6D89A
:10642000002BF9D101AA01212819064B98470346F0
:106430000028F1D19DF804203255EDE76563400056
:10644000F00502009D62400030B587B01D201C4B56
:1064500098471C4C236C23F40013236468461A4BA2
:10646000984769462046194B9847636823F47F4351
:106470006360636843F47F436360042323610823FC
:10648000236101232361626822F08F026260104A57
:10649000032120460F4DA847002120460E4B984768
:1064A000636813F0800F01D1082222600B4B4FF07C
:1064B00000521A60702283F81D2307B030BD00BF60
:1064C00061D140000080034095494000294A4000C6
:1064D00001654000794A4000BD49400000E100E00C
:1064E0000222014B1A60704700800340024B188063
:1064F000024B1980704700BFBE000020C000002082
:1065000010B5064C206D80B2054B9847A06DE16D2B
:1065100089B280B2034B984710BD00BF0080034092
:10652000F5754000ED644000014B1888704700BFCE
:10653000BE000020014B1888704700BFC00000203B
:106540000D4B1B8840F68962934205D90B4A12888D
:106550003E2A01D803207047084A128840F6896114
:106560008A4203D93E2B01D804207047934201D8B8
:106570000220704701207047BE000020C0000020AC
:1065800008B50120034B9847034B186000B1012068
:1065900008BD00BF0DDD40001011002008B54FF010
:1065A000FF31024B1868024B984708BD10110020BC
:1065B000C9DE400010B500231A461946024800689B
:1065C000024CA04710BD00BF10110020D5DB4000D9
:1065D000154B98421BD003F5A033984219D003F510
:1065E0008043984217D0A3F54043984215D003F555
:1065F0008043984213D0A3F5A033984211D003F5FD
:106600006033984201D0322070471620704708202E
:106610007047092070470E207047132070471420E0
:1066200070471520704700BF00C000404900B0FB14
:10663000F1F00338002302E040080133DBB2FF2809
:10664000FAD8020202F47F4252FA80F01B0403F4EB
:10665000E0231844704700002DE9F843D0F800907B
:10666000037ADBB2012B00F0E68009F5C0650B79F7
:1066700013B91846BDE8F88317460E4604460123B1
:1066800003720023C371E1606E4B98478046B37874
:10669000022B08D07378012B18D033781B0403F435
:1066A000FE036B6050E07378012B09D033781B0434
:1066B00003F4FE0303F580736B60F378EB6043E053
:1066C00033785B081B0403F58073F5E733785B08C8
:1066D0001B04E6E70323A37100232372237A002B14
:1066E00000F0AB802B6A13F4807F53D113F4007F4A
:1066F00078D113F0400F7AD113F0800F7CD113F0D2
:10670000040F4BD1394640464F4B98470028E9D0FB
:106710000723A371002323724C4BC9F800363DE0D8
:106720000423A37100232372D8E70523A371002358
:106730002372D3E70623A37100232372CEE73946E1
:106740004046414B9847E8B93379E2799B1A002BD0
:10675000C4DD2B6A13F4807FBCD113F4007FDFD13A
:1067600013F0400FE1D113F0800FE3D113F0040FC9
:10677000E5D0B168E379DBB25A1CD2B2E271CB5CEE
:106780006B63DCE70723A371002323722F4BC9F847
:106790000036A3E70323A37100232372237A002B7F
:1067A0004DD00223C9F800362B6A13F0010F28D10F
:1067B00013F4807F2BD113F4007F2DD113F0400F01
:1067C0002FD113F0800F31D1394640461E4B9847E8
:1067D0000028E9D00723A371002323721B4AC9F8BC
:1067E000002646E70423A37100232372D6E705237E
:1067F000A37100232372D1E70623A3710023237220
:10680000CCE7002323720223A371012331E7032382
:10681000A371002323722CE70423A37100232372A6
:1068200027E70523A3710023237222E70623A37120
:10683000002323721DE700231BE7002319E7002331
:1068400017E700BF517140006971400002800005E8
:106850002DE9F84FD0F800B0037ADBB2012B00F03D
:10686000CE800BF5C0670B7913B91846BDE8F88FD9
:1068700090460E460546012303720023C371E9606A
:10688000614B98478146B378032B14D07378012B62
:1068900024D033781B0403F4FE0303F580537B609C
:1068A00096F804A0BAF1010F1ED00123CBF80036F0
:1068B0004FF0000A64E07378012B09D033781B0491
:1068C00003F4FE0303F588537B60F378FB60E7E78E
:1068D00033785B081B0403F58853F5E733785B08CE
:1068E0001B0403F58053DAE70323CBF8003647E0B7
:1068F0000323AB7100232B722B7A002B00F08180D5
:106900003B6A13F0010F60D113F4807F63D113F45D
:10691000007F65D113F0400F67D113F0800F69D16C
:1069200041464846394B98470028E9D00723AB71C8
:1069300000232B72364ACBF8002696E70423AB716E
:1069400000232B72D8E70523AB7100232B72D3E70A
:106950000623AB7100232B72CEE70723AB71002314
:106960002B722B4BCBF80036C6E714F0020F07D082
:10697000B168EB79DBB25A1CD2B2EA713A6BCA54F5
:10698000EB79DBB232799342B6D23C6A14F4807F61
:10699000AED114F4007FD1D114F0400FD3D114F054
:1069A000800FD5D141464846184B98470028D4D18E
:1069B000BAF1000FD9D13379EA799B1A012BD4D1DE
:1069C00002233B604FF0010ACFE700232B72022322
:1069D000AB71012349E70323AB7100232B7244E71A
:1069E0000423AB7100232B723FE70523AB71002317
:1069F0002B723AE70623AB7100232B7235E7002395
:106A000033E7002331E700BF517140006971400056
:106A1000028000052DE9F0410646884604682046BC
:106A20001B4B9847312801D9BDE8F0810546194B29
:106A30009847032323602423C4F8003641461648B0
:106A4000164B9847C4F81006002333720123B37124
:106A50006BB2002B07DB5A0905F01F0001218140B2
:106A60000F4840F82210002B0BDB03F1604303F5C5
:106A70006143202283F8002301200A4B98473061AC
:106A8000D2E705F00F05084B20225A55F4E700BF66
:106A9000D165400061D140000000DC052D6640005A
:106AA00000E100E00DDD400014ED00E008B50068F5
:106AB0000B4B9847312811D843B2002B0CDB5B09F4
:106AC00000F01F0101228A402033064941F82320AB
:106AD000BFF34F8FBFF36F8F034B984708BD00BFC5
:106AE000D165400000E100E0B5D1400008B54FF0AD
:106AF000FF310069014B9847C0B208BDC9DE4000B4
:106B000010B500231A4619460069024CA047C0B2CE
:106B100010BD00BFD5DB400008B5837963B18B7829
:106B2000032B0BD8DFE803F002050205044B98475E
:106B300008BD044B984708BD002008BD002008BDD3
:106B4000596640005168400080797047F8B50646A4
:106B5000036803F5C064256AC76815F0040F0BD0FD
:106B6000E26A12F0040F07D0BA78002A4DD0022A48
:106B70004BD0BA78032A5ED015F0020F08D0E26A33
:106B800012F0020F04D0BA78012A73D0032A71D010
:106B900015F4807F0DD0E36A13F4807F09D040F2B2
:106BA0000733A362002333720323B371FB6803B17D
:106BB000984715F4007F0DD0E36A13F4007F09D0E5
:106BC00040F20733A362002333720423B371FB68DE
:106BD00003B1984715F0010F16D0E36A13F0010FC7
:106BE00012D0BB780BB1022B09D140F20533A3625E
:106BF000002333720223B371FB6803B19847BB785B
:106C0000012B54D0032B52D0F8BDF279D2B239798E
:106C10008A4208D2B868F279D2B2511CC9B2F17175
:106C2000825C6263A5E70222C3F800260122626249
:106C30000422A2629DE77A78012A11D03A781204E0
:106C400002F4FE0202F5805262603A79012A0DD008
:106C50000122C3F800260422A262022262628BE7AC
:106C60003A785208120402F58052EDE70322C3F885
:106C70000026F0E7B868F279D2B2511CC9B2F171BE
:106C8000216B8154F179C9B23A79013A91420AD023
:106C9000F379DBB23A7993427FF47AAF01236362EE
:106CA0000223A36274E70222C3F80026F0E740F251
:106CB0000333A362002333720223B371FB68002BFA
:106CC000A2D09847A0E7000070B4056805F5C0663B
:106CD0000379202B0BD9A3F12001CBB21A4C01214F
:106CE00099402160216521612163002211E0174C48
:106CF000F5E701339BB2B3F52F7FFAD3616300232D
:106D000001E001339BB2B3F52F7FFAD32163013247
:106D1000D2B2092A01D80023EDE7616161603269CE
:106D20008023C5F80036002301E001339BB2B3F5A0
:106D30002F7FFAD332612423C5F800360023037273
:106D40000123837170BC704700100E40000E0E408E
:106D500030B591B000238DF835308DF836308DF890
:106D600037308DF839308DF83A30ADF83E300F239A
:106D70008DF834300223ADF83C3001248DF83840D2
:106D80000DAA0B4907A80B4DA8470DAA0A4901A84F
:106D9000A8471023079A1360019A1360074B1C70D1
:106DA000074B1C7045F6FF72064B1A8011B030BDC0
:106DB00000C0024049CC400000000340DC0C002031
:106DC000F4120020BE13002042B110B420B119B15A
:106DD000034B586099605A805DF8044B704700BFC0
:106DE000DC0C0020154B1B783BB3144B5B8823B3A2
:106DF000124A52680AB311498968F1B1F0B583B0FB
:106E0000009201930E4D6A46694628460D4FB847D9
:106E10004FF480362E62094B9B6800930A4C6A46F9
:106E200069462046B847266201212846074DA847F3
:106E300001212046A84703B0F0BD7047DC0C0020BC
:106E400000C1024085CB4000000103409DCB4000C3
:106E50000223034A136202F580421362704700BFA7
:106E600000C1024010B58CB00A4B9847069A1368CF
:106E700023F010031360009A136823F010031360CB
:106E80000D20054CA0471220A0470022034B1A708A
:106E90000CB010BD516E4000B5D14000DC0C00209C
:106EA000064B1B783BB1054B5888054BD3F8043192
:106EB000C01A80B270470020704700BFDC0C002071
:106EC00000C00240094AD36D23F4FF4323F07F033F
:106ED000C0F30E000343D36502F58042D36D23F463
:106EE000FF4323F07F031843D065704700C0024082
:106EF000014B1880704700BFBE130020014B187073
:106F0000704700BFF412002000487047C0130020F3
:106F10000048704714110020704770472DE9F8436E
:106F20004F4B984705464F4B984704467FE0A0EBF0
:106F3000070E1FFA8EFE0EF1F00E1FFA8EFE85E090
:106F40003121002308E02F21FBE747480078C0B239
:106F5000012831D001339BB2994259D9DA1992B242
:106F6000EF2A01D9F03A92B23F4800780028ECD1DC
:106F70003E48B0F9000035F9126006FB00F6F61342
:106F80004FEA8308DFF8ECC00CF8236008F1010930
:106F9000C6F307260CF8096034F9122000FB02F250
:106FA000D21308F102000CF8002008F10308C2F324
:106FB00007220CF80820CDE735F9120034F9122029
:106FC000024402EBD272521012F5004F05DBB2F50B
:106FD000004F03DB47F6FF7200E0254A2348B0F973
:106FE000000012B202FB00F2D21398005FFA82FC9A
:106FF000204E06F823C000F10108C2F3072206F86C
:10700000082000F1020806F808C003303254A1E756
:10701000194BA3F800E07744BFB2184B1F80EF2F45
:1070200001D9F03F1F8089001248154B98474FF057
:10703000FF310120134B9847134B98470F4B1F8884
:10704000B842FFF474AFC01B1FFA80FEBEF1300FD0
:107050003FF676AFBEF12F0F7FF675AF302170E7A8
:10706000096F4000116F4000F4120020BE13002091
:107070000080FFFFF8120020BC130020E80C002065
:107080002D45400071EB4000A16E4000F8B5084C62
:107090004FF4804666630A20064DA8474027676381
:1070A0000A20A84727630A20A8472663F8BD00BF27
:1070B000000E0E4081E64000F8B578B9114D4FF44E
:1070C00080736B630220104CA0474FF080736B639A
:1070D0000420A04701220D4B5A63F8BD094E4FF41E
:1070E00080737363094F02253D632846064CA04711
:1070F00001233B630420A0474FF08073336328468D
:10710000A047F8BD000E0E4081E6400000100E4082
:1071100010B5084C4FF4804363630020064B98473A
:107120000220064B98470222054B5A6340236363B3
:1071300010BD00BF000E0E40B970400081E6400057
:1071400000100E400322014B1A60704730140E40AD
:10715000044B986801E0034B9868024B9B68984287
:10716000F9D1704730140E4010B584B001900C4630
:10717000064B98470390039B019A9B1AA34202D2A5
:10718000002004B010BD0120FBE700BF517140009A
:1071900030B585B01E4B1B68002B31D01D4B984776
:1071A0004FF0FF311A4B18681B4B9847EFF31083D1
:1071B000B3FA83F35B09039372B6BFF35F8F0022C8
:1071C000164B1A70039D80230093154B1522142132
:1071D0001448154CA04704462DB101220F4B1A70DC
:1071E000BFF35F8F62B600231A461946084800684D
:1071F0000E4DA8470E4B984744B1002005B030BD56
:1072000001200C4B9847024B1860C7E70120F5E7B7
:10721000EC0C00209D654000C9DE4000EB02002020
:10722000A0150020000A0E4011000020D5DB400010
:10723000B56540000DDD400010B5074B98470022B2
:1072400013210648064B98470446064B9847B4FA64
:1072500084F0400910BD00BF9D654000000A0E404B
:10726000C1CE4000B565400038B5114B9847EFF3EB
:10727000108404B972B6002308E09A0002F5800277
:107280000C4951F82310116001339BB27F2BF4D9C4
:10729000002212210848094B9847C5B204B962B6CA
:1072A000074B98470DB1002038BD012038BD00BF05
:1072B0009D654000A0150020000A0E40C1CE400090
:1072C000B565400010B400240EE0400080F00700D7
:1072D000C0B20133DBB2072B05D810F0800FF4D118
:1072E0004000C0B2F5E70134944204D211F8013BEA
:1072F00058400023EFE75DF8044B704770B5064631
:10730000002501E02C44A5B2B5F5007F15D20E4B47
:10731000E918EA5CFF2A14D06B1C0B481B5C033392
:10732000DCB2B242EED1621EFF20084B98472B1907
:10733000074A9B5C9842E5D101E04FF6FF7528466D
:1073400070BD4FF6FF75FAE7A0150020C57240002A
:107350009F15002008B5094B1B781BB1022B01D0EB
:10736000074808BD074B9847012804D10122034B69
:107370001A70034808BD002008BD00BFF00C0020B3
:10738000A01500209171400008B5094B1B781BB176
:10739000022B01D0074808BD074B9847012804D1AC
:1073A0000122034B1A70034808BD002008BD00BF2E
:1073B000F00C0020A015002091714000A8B108B584
:1073C0000346B1F5007F12D28818B0F5007F01D9CD
:1073D000002008BD08461946064B1844064B98473E
:1073E0000222064B1A70012008BD002070470020C1
:1073F00008BD00BFA0150020C10D4100F00C002009
:1074000008B5064B1B78022B01D0002008BD044BA9
:1074100098470128FAD1034B984708BDF00C00208B
:10742000397240006972400090B110B5044602689C
:10743000094B9A4201D0002010BD9A220146FF203C
:10744000064B984794F89A30984203D0002010BD1C
:1074500000207047012010BD5FE1AD5AC5724000A9
:1074600010B50C46084B9847B0F5007F01D30020BB
:1074700010BD811C054B5A1C125C19442046044B5C
:107480009847012010BD00BFFD724000A0150020EC
:10749000C10D410008B5044B9847B0F5007F01D2FB
:1074A000012008BD002008BDFD72400008B5054B55
:1074B0009847B0F5007F02D2034BC05C08BD0020A6
:1074C00008BD00BFFD724000A1150020FF292FD08C
:1074D0002DE9F843D61CF6B28419B4F5007F03D920
:1074E0004FF6FF70BDE8F88317460C4605460221AB
:1074F000114A1170DFF84C8000EB080900F80840D1
:10750000421C02F8087008443A46194640440B4BA6
:1075100098477C190234721E4946FF20084B984751
:1075200008F80400E81980B2033080B2BDE8F8839F
:107530004FF6FF70704700BFF00C0020C10D4100F6
:10754000C5724000A015002010B5A8B0224B984786
:107550000446224B984708B928B010BD9B2221460B
:1075600001A81F4B98474FF40072FF211D481E4B86
:10757000984702AB1022012100201C4CA0474FF677
:10758000FF73984203D026AB03220221A0474FF697
:10759000FF73984205D00DF19B0301220321134C88
:1075A000A0474FF6FF73984204D027AB0122042175
:1075B0000E4CA0474FF6FF73984205D00DF19D0386
:1075C00001220521094CA0474FF6FF739842C3D012
:1075D000074B9847C0E700BF55734000297440002F
:1075E000C10D4100A0150020BD0F4100CD74400029
:1075F00001744000044B1880044A1378591C117020
:10760000034A22F813007047A4190020F10C00204F
:10761000A417002008B5194B1B8807EE903AF8EE26
:10762000677A9FED177A67EE877A164BC3ED007A7B
:10763000F7EE006A76EEE76A87EEA67ADFED126A69
:1076400067EE267A114BC3ED007A86EEA77A17EE25
:10765000100A0F4B9847DFED0F7A07EE100A27EE5E
:10766000277ADFED0D7A77EEC77ADFED0C6A86EECA
:10767000A77A0B4B83ED007A08BD00BFA419002048
:1076800001088039A017002000401C46AC190020DA
:1076900055F940003313954300F05745C47D7B49AD
:1076A000A8190020BFF35F8F024B1868BFF35F8FEC
:1076B000704700BFA819002068B90F4A1368B3F1DA
:1076C000FF3F0AD00320B3F1333F0ED013B9536804
:1076D00003B902207047094AF0E75168B1F1FF3F52
:1076E00001D00320EFE70020EDE75168B1F1333F0F
:1076F000ECD10120EAE700BF00C0470000E04700EE
:1077000018B101280FD0022070470B4841F6F873DA
:1077100083B130B4C518C4588C4206D0083B002B46
:10772000F8D1012004E00548F0E76B681360002001
:1077300030BC70470120704700C0470000E04700A0
:1077400070B505460020124CA04706460120A04710
:107750001DB1012D12D0022070BD022803D0022ECF
:1077600007D0022070BD012E01D0012070BD002085
:1077700070BD012801D0002070BD70BD022E05D063
:10778000022801D0022070BD012070BD002070BD14
:10779000B9764000F8B504460F461646450A094B2F
:1077A000984704F4FE7000F580031F605E602A466F
:1077B00001210548054B98470446054B984720464C
:1077C000F8BD00BF9D654000000A0E40C1CE4000DC
:1077D000B5654000012909D002290CD1002108B566
:1077E00038B906480A46064B984708BD4FF0333172
:1077F000F5E70448F6E70120704700BF00C04700E6
:107800009577400000E0470038B518B101280DD049
:10781000022038BD0A4C0823B3F5005F0ED2E018F1
:10782000E558B5F1FF3F03D00833F5E7054CF2E723
:10783000054B984708B1022038BD38BD012038BD3E
:1078400000C0470000E047009577400010B568B1E0
:1078500040F2F234074B9847224607210648074B6F
:1078600098470446064B9847204610BD40F2E23444
:10787000F0E700BF9D654000000A0E40C1CE400009
:10788000B565400070B505460E460B4C4FF0FF3114
:1078900020680A4B98470120094B984732462946F1
:1078A000084B9847054600231A4619462068064C9F
:1078B000A047284670BD00BFB0190020C9DE4000B7
:1078C0004177400001774000D5DB4000F8B5054620
:1078D0000E464FF0FF31144B1868144B98470020A8
:1078E000134B9847074632462946124B98470446A1
:1078F000012808D000231A4619460B4800680E4D8F
:10790000A8472046F8BDB7FA87F4640921463846EF
:107910000A4B984708B10224ECE732462946204634
:10792000044B98470446E5E7B0190020C9DE400043
:107930004177400009784000D5DB4000C579400020
:1079400030B583B000230193044660B9164D174942
:107950000023B3F5006F24D251F82320B2F1FF3F8A
:1079600004D10133F5E7124D1249F1E72046124BDD
:107970009847044610B1204603B030BD01A92846FF
:107980000E4B984740B90199013128460C4B984756
:107990000028F0D00124EEE701212846084B984743
:1079A000F6E70024E7E700BF0120FFFF00C0470023
:1079B0000220FFFF00E047004D784000857840003E
:1079C000CD78400070B582B005460E460846284B7B
:1079D0009847012806D001213046264B9847044697
:1079E000002841D1002400E00134234B1B689C4255
:1079F00015D201AA214B53F824102846204B984752
:107A0000022830D00028EFD1019A1C4B53F82410E3
:107A100030461C4B98470028E6D0012424E0284635
:107A2000194B98470446F8B902213046114B984744
:107A30000446C8B985B9154D02A9002341F8083D8F
:107A40002846134B984748B9009901312846114BF5
:107A5000984748B1012407E00F4DEDE70121284682
:107A60000C4B9847F5E70124204602B070BD00BFDB
:107A7000B9764000D5774000DC000020C40000202B
:107A800001774000097840004D7840000120FFFF59
:107A900085784000CD7840000220FFFF10B500201F
:107AA0000E4B9847044608B1204610BD01200B4BF1
:107AB000984704460028F7D10221094B984704460D
:107AC0000028F1D101210748074B984708B101244C
:107AD000EAE701210548044B9847E5E74D78400067
:107AE000D57740000120FFFFCD7840000220FFFF46
:107AF00038B501202D4B98472D4B1860002852D0E7
:107B000000202C4DA84704460120A847012C20D076
:107B100034B1022C35D0284B98470346184638BD5F
:107B2000012806D0022810D10020244B9847034694
:107B3000F4E70020214B984703460028EED10221AC
:107B400001201F4B98470346E8E71B4B9847034625
:107B5000E4E738B1022810D100210120194B9847E1
:107B60000346DBE70120154B984703460028D5D193
:107B70000221134B98470346D0E70F4B9847034623
:107B8000CCE728B1022808D10B4B98470346C5E73C
:107B900001200A4B98470346C0E701210020094B0A
:107BA00098470346BAE70123B8E700BF0DDD400060
:107BB000B0190020B97640009D7A4000417940001C
:107BC000D5774000C579400008B50020094B98479B
:107BD00008B1012008BD2022074B5A630A20074B39
:107BE0009847074B9847074B9847012801D000203A
:107BF00008BD08BD995C400000100E4081E64000C1
:107C0000CDF84000E95B400030B587B0174B98478E
:107C100004468A238DF808300025059501238DF848
:107C200009308DF80C300DF107030493104B984781
:107C30008DF80B5003238DF80A30322202A920461A
:107C40000C4B984720460C4B9847022806D000253D
:107C500020460A4B9847284607B030BD9DF80730AC
:107C6000092B01D00025F3E70125F1E7CDF840000D
:107C7000ED6A4000196B4000496B4000016B400009
:107C800030B587B01A4B9847044600220592A823C6
:107C90008DF8083001238DF809308DF80B2001AAEA
:107CA000049202228DF80C208DF80A30114B98476F
:107CB000322202A92046104B984720460F4B984786
:107CC000022806D0002520460D4B9847284607B0CD
:107CD00030BD9DF8043033B99DF8053013F0F80F2E
:107CE00003D00025EFE70025EDE70125EBE700BF16
:107CF000C5F84000ED6A4000196B4000496B400038
:107D0000016B400008B5034B984708B1002008BD3F
:107D1000012008BD5960400030B587B0184B984726
:107D200004460023059372238DF8083001238DF853
:107D3000093092228DF80B200DF1070204928DF884
:107D40000C3003238DF80A300E4B9847322202A9DB
:107D500020460D4B984720460C4B9847022806D0EA
:107D6000002520460A4B9847284607B030BD9DF8AD
:107D70000730442B01D00025F3E70125F1E700BFD0
:107D8000CDF84000ED6A4000196B4000496B40009F
:107D9000016B400070B586B0002832D11C4B98476B
:107DA00004460025059598238DF8083001268DF8A6
:107DB00009608DF80A5002238DF80C3001AB049352
:107DC0008DF80B502046134B984736238DF804301E
:107DD0008DF80550322202A920460F4DA8478DF894
:107DE0000A60322202A92046A84720460B4B98473A
:107DF00002280AD000252046094B9847284606B09D
:107E000070BD084B98470446CBE73546F3E700BF03
:107E1000C5F84000ED6A4000196B4000496B400016
:107E2000016B4000CDF8400038B50020064CA0475B
:107E300005460120A047012D01D0002038BD0128B2
:107E4000FCD0002038BD00BF957D40002DE9F047F3
:107E50003D4BD3F8588019203C4B98474FF496700F
:107E60003B4B9847002409E03A4B98473A4B23F89C
:107E700014000320364B98470134E4B21F2CF3D989
:107E8000364B9847824600263746354634463FE013
:107E9000314931F813100A440133DBB21F2BF7D9F3
:107EA0004FEA5219B9F10A0F17D92A4B9847631CA8
:107EB000DBB2294A22F814001F2B1DD81C46A9F159
:107EC000FA0398421AD309F1FA02904225D80135F3
:107ED000EDB2202D13D9012611E0B8F1000F05D025
:107EE000194BC3F858800020BDE8F0870020174BDD
:107EF00098470020BDE8F0870024E0E70025032034
:107F0000134B98474FF47A615046154B98470746F4
:107F10002FB926B900231A46C0E70025EFE7B8F1CC
:107F2000000F07D0084BC3F8588057B936B101206D
:107F3000BDE8F0870020054B9847F6E70020BDE834
:107F4000F0870020BDE8F08700000140C94B4000E9
:107F500081E64000154C4000B419002051714000EA
:107F60006971400000487047503A4100072070474F
:107F70002DE9F84305460E4617460A469C211E4B3E
:107F800098470446451B40B1731B052B05D9437820
:107F9000552B07D010237B7001E000237B70204617
:107FA000BDE8F88390F80280C37888EA0303FF2BCA
:107FB00002D011237B70F2E790F80490437909EB2B
:107FC00003291FFA89F9B9F13A0F06D84D4406354D
:107FD000AE4205D200237B70E1E712237B70DEE71F
:107FE0004A46811D381D054B9847A7F8029087F82F
:107FF000008001237B70D2E7C10C4100C10D41001C
:1080000010B553889C1D8C4219D83A2B01D90020F9
:1080100010BD11469C230370552343701378837061
:108020001378DB43C3709378037153881B0A437141
:10803000528804310630034B9847012010BD0020C0
:1080400010BD00BFC10D410070B582B00446037879
:10805000253B332B00F21982DFE813F045001702AD
:10806000170217021702340017021702170217022D
:108070001702170217021702170217021702170238
:108080001702170217021702170217021702170228
:10809000170217023E0117021702FA001702170211
:1080A000170217021702BA0113015C001702170228
:1080B0001702170217021702170265017900CB0099
:1080C000A600E3009C4C2A2323709C4DA8476080A7
:1080D0009B4B98470646A84702463146201D994BC0
:1080E000984702B070BD0120974B984780B2924BE1
:1080F000588010B945221A70F3E794490120944B37
:10810000984718B125228C4B1A70EAE745228A4B12
:108110001A70E6E74388032B05D0874B00225A806C
:1081200045221A70DDE703798DF8043043798DF824
:10813000053083798DF80630864B984701A9864B28
:1081400098477D4B00225A8024221A70C9E7438841
:10815000012B05D0784B00225A8045221A70C0E7C7
:1081600003790F2B05D9744B00225A8045221A70CF
:10817000B7E77A4B9847704A5523137020235380F2
:10818000237900EB4310066845688468C16856602F
:108190009560D4601161066945698469C169566159
:1081A0009561D46111629CE74388212B05D0624B15
:1081B00000225A8045221A7093E701790F2905D9C8
:1081C0005D4B00225A8045221A708AE7202249011D
:1081D0000530634B9847012805D0574B00225A8041
:1081E00045221A707DE7544B00225A8024221A70CF
:1081F00077E743882BB1504B00225A8045221A70F2
:108200006FE7584B9847012805D04B4B00225A8006
:1082100045221A7065E7484B00225A8024221A70C2
:108220005FE743882BB1444B00225A8045221A70E5
:1082300057E74D4B984728B93F4B00225A802422DC
:108240001A704EE73C4B00225A8045221A7048E7CC
:108250004388012B05D0384B00225A8045221A70E2
:108260003FE70079414B984728B9334B00225A80A9
:1082700024221A7035E7304B00225A8045221A70AA
:108280002FE74388082B05D02B4B00225A8045222C
:108290001A7026E70379427903EB0223827903EB14
:1082A0000243C079217A627A01EB0221A27A01EBC2
:1082B0000241E47A01AA01EB046103EB00602C4B5C
:1082C000984700287FF40DAF1B4B019A5A604B2250
:1082D0001A7004225A8004E74388063B9BB21F2B86
:1082E00005D9154B00225A8045221A70F9E64379C8
:1082F000807903EB0023E07903EB0043207A04F15B
:108300000902217903EB00601A4B984728B90A4B00
:1083100000225A8024221A70E3E6074B00225A807A
:1083200045221A70DDE6438833B3034B00225A809E
:1083300045221A70D5E600BFF41900206D7F400079
:10834000657F4000C10D4100AD744000F819002068
:1083500061744000CDF84000515A400089734000DC
:10836000BD7340000174400059604000016340004B
:108370009D624000E56240000020474B1871474B6A
:10838000984720B1444A137943F001031371012047
:10839000424B984720B1404A137943F002031371CE
:1083A00002203E4B984720B13B4A137943F0040327
:1083B00013710320394B984720B1374A137943F0A2
:1083C00008031371344B01225A8054221A7088E634
:1083D0004388012B05D0304B00225A8045221A7069
:1083E0007FE60379463B102B49D8DFE803F03F488E
:1083F00009484848124848362D48481B4848240038
:10840000274B9847244B18714A221A7001225A8030
:1084100067E6244B9847204B18714A221A700122B4
:108420005A805EE6204B98471B4B18714A221A70FF
:1084300001225A8055E61D4B9847174B18714A2266
:108440001A7001225A804CE6194B9847124B18714A
:108450004A221A7001225A8043E6164B98470E4B67
:1084600018714A221A7001225A803AE6124B984734
:10847000094B18714A221A7001225A8031E6064BC4
:1084800045221A7000225A802BE6034B00225A80A4
:1084900045221A7025E600BFF419002065634000EC
:1084A000C97B4000097C4000817C4000057D400084
:1084B000197D4000297E40004D7E400000487047F5
:1084C000F4190020F0B583B0EFF31083B3FA83F30F
:1084D0005B09019372B6BFF35F8F0022364B1A70AF
:1084E000019E364B1B68364A15682B447F2B2AD8D1
:1084F000324B1C682246334933482844334B984753
:108500002C442F4B1C6000222C4B1A602EB10122F0
:10851000294B1A70BFF35F8F62B62D4A284B19683A
:1085200029482C4B98470146D0B1274BC31A2848FD
:1085300042881A44951D4478012C15D044BB802BE9
:108540001CD900242AE01D4A136814682C441B1B04
:1085500003F18004204A137843F001031370C9E744
:108560000024174B1C6019E01748154F3E68761B16
:1085700032464119194B98473E600FE0104D2C6868
:10858000E41A22461048154B98472C60002405E059
:108590000133802B05D90024094B1C60204603B011
:1085A000F0BD0948064D2C68E41A2246C1180B4B51
:1085B00098472C600024F1E7EB0200203C1D0020CE
:1085C0004C1D0020941D00203C1C0020C10D4100CA
:1085D000501D0020717F4000481D0020F50E410015
:1085E00010B50DE0144B195D1448154B9847013434
:1085F000E4B2144B1B689C42F4D30022114B1A6066
:108600000120114B9847114B98470128F8D1104889
:10861000104B9847104B98470246802106480F4B55
:1086200098470128ECD10C4B984743880633054AFC
:1086300013600024DDE700BFBC1C00200082014065
:108640004BD34000441D002081E64000C58440001B
:10865000501D002049804000BD8440000180400042
:1086600030B583B08024224600211C481C4DA84709
:10867000224600211B48A84700231B4A13601B4ABF
:1086800013601B4A13701B4A10215166C2F89010E8
:1086900051655162C2F88010116F21F0100111670D
:1086A000516F21F010015167134A4FF400211160FE
:1086B000202182F813130121104A9160104A01927F
:1086C000009322460F491048104CA047012802D0C1
:1086D0000F48104B984703B030BD00BF941D0020D9
:1086E000BD0F4100BC1C00203C1D0020441D00208B
:1086F000481D0020000E0E4000E100E00082014015
:10870000401D0020583A4100E1854000ADE34000A3
:10871000603A410015074100104B1B6913F0010F2F
:1087200012D00E4B5B6913F0010F0DD00C4B1B6880
:108730007F2B0AD90B4A137843F001031370074BC0
:108740009A69094B83F87F207047054A1368591CC2
:108750001160024A9169044AD15470470082014075
:108760003C1D0020481D0020941D0020064A9368EF
:1087700023F07F4323F4706343F0254343F4E06325
:108780009360024B1360704700140E40080000A570
:1087900070B506460D46094B98470446002040B97F
:1087A00029462046064B984728B93046054B98473E
:1087B000F5E7012070BD002070BD00BF5171400081
:1087C0006971400055A5400010B54FF47A722B4BEB
:1087D0001A8004E04022002129482A4B9847274B61
:1087E000188880B2284B9847254C232323701423E4
:1087F0006370264B9847C0F30F23A370E070244B9F
:108800009847C0F30F2323716071224B9847C0F340
:108810000F23A371E071204B9847C0F30F232372FD
:1088200060721E4B9847C4F80A001D4B1B7807EE78
:10883000103AB8EE477A9FED1B6A27EE067ADFED15
:108840001A6A37EE667A17EE103AC4F80E30174BF4
:108850001B7807EE903AF8EE677A67EE867A77EE45
:10886000E67A17EE903AC4F81230114B9847002878
:10887000B0D0322120460F4B9847ABE7881E00202E
:10888000381E0020BD0F410081E64000154C40001D
:10889000A55240002965400035654000A57640009E
:1088A000B4010020B4C8363F6FDB4A42B501002056
:1088B000EDF8400091874000F0B583B040220021E0
:1088C0009A489B4B9847FCE19A4B98479A4B98479C
:1088D00002E2984B9847994BBB221A601A225A60C1
:1088E000954B9847FBE191490B462A2203F8012B4F
:1088F000934A1068C1F801009188927910469980D6
:108900009A71EFE101208F4B984728B9874B452298
:108910001A7002225A70E8E18449252301F8013BCC
:108920000120894B9847E0E10820864B984728B9F9
:108930007E4B45221A7002225A70D9E17B492623C8
:1089400001F8013B0820804B9847D1E109207D4B7D
:10895000984728B9754B45221A7002225A70CAE10D
:1089600072497E2301F8013B0920774B9847C2E109
:10897000C4F30723032B09D8DFE803F0020B040636
:10898000724807E0724805E0724803E04FF0FF309C
:1089900000E07148B0F1FF3F10D001A96F4B98473C
:1089A00030B9624B5A221A70019AC3F80120A6E12D
:1089B0005E4B45221A7002225A70A0E15B4B4522A1
:1089C0001A7001225A709AE1C4F30723032B09D8C5
:1089D000DFE803F0020B04065C4807E05C4805E0B2
:1089E0005C4803E04FF0FF3000E05B48B0F1FF3F30
:1089F0000ED05B4B19685B4B984718B924224B4B40
:108A00001A707FE1494B45221A7003225A7079E1AE
:108A1000464B45221A7001225A7073E12422434BBF
:108A20001A7072E1414B45221A704F4A12785A70FF
:108A30006EE14E4B1B780F2B05D93C4B45221A702B
:108A400001225A7067E14A4B9847384A5523137000
:108A500020235370454B1B7800EB4310D0F800E007
:108A600047688668C168C2F802E0C2F80670C2F8BA
:108A70000A60C2F80E10D0F810E047698669C16933
:108A8000C2F812E0C2F81670C2F81A60C2F81E10DE
:108A900041E1264B4B221A7004225A706A44354B2E
:108AA0001968354B1868354B984720B91F4B019A08
:108AB000C3F8022032E10022314B1A602EE11B4B39
:108AC00054221A70002058702E4B984720B1174A34
:108AD000537843F00103537001202A4B984720B18B
:108AE000124A537843F0020353700220254B9847F3
:108AF00020B10E4A537843F0040353700320214BF6
:108B00009847002800F00D81084A537843F0080385
:108B1000537006E11C4B1878072837D9802841D0BC
:108B2000024B45221A7001225A70FDE0901E00206F
:108B3000BD0F410049F840006D87400090140E4081
:108B4000F83A4100AD744000617440000110FFFF2D
:108B50000310FFFF0410FFFF0210FFFF85784000A5
:108B6000841E0020CD7840008A1E0020801E002038
:108B7000897340008C1E00207C1E00209D624000F6
:108B8000921E002065634000141E0020724B98471F
:108B900018B92422714B1A70C6E0704A4521117031
:108BA0005070C1E06E4B187810F0800FB8D16D4B4B
:108BB000984718B92422694B1A70B5E0674B4521D4
:108BC00019705870B0E0684A684B1968684B1868AB
:108BD000684B984718B92422604B1A70A7E05F4B86
:108BE000452119705870A2E05C484E2300F8013B03
:108BF000614B9847002800F09D80604B4FF0203279
:108C00001A605A609A60C3F80B2093E014F47F4F07
:108C1000524E31464FF05E0301F8023B14BF012073
:108C20000020574B98477070002840F086804522FE
:108C3000327082E04A22494B1A70C4F30723463B44
:108C4000102B2DD8DFE803F0272C092C2C2C0E2C10
:108C50002C221D2C2C132C2C18004A4B98473F4BD0
:108C600058706DE0484B98473C4B587068E0474B54
:108C700098473A4B587063E0454B9847374B5870CC
:108C80005EE0444B9847354B587059E0424B98474B
:108C9000324B587054E0414B9847304B58704FE07E
:108CA0002E4B45221A7001225A7049E03C4B9847DE
:108CB00024222A4B1A7045E0402200212748394BD4
:108CC00098474FF0FF310120374B98470446002862
:108CD000F7D043283FF4F8AD422C3FF4FAAD2A2CEC
:108CE0003FF401AE252C3FF40DAE262C3FF41CAE14
:108CF0007E2C3FF42BAEE5B25A2D3FF439AE7A2DDF
:108D00003FF462AE242C3FF489AE452C3FF48AAE8A
:108D1000552C3FF48EAE4B2C3FF4BBAE542C3FF49D
:108D2000CEAE442C3FF4F6AE412C3FF44CAF4E2C6B
:108D30003FF45AAF5E2D3FF469AF4A2D3FF47AAF4E
:108D40003D2CB3D0194B98470028B5D032210348A9
:108D5000174B9847B0E700BF01634000901E00200A
:108D6000781E002031634000181E00208C1E002059
:108D70007C1E0020E5624000ED634000911E002053
:108D800041504000C97B4000097C4000817C40008C
:108D9000057D4000197D4000297E40004D7E400049
:108DA000499D4000BD0F410071EB4000EDF84000CF
:108DB0009187400010B50023032201460248006855
:108DC000024CA04710BD00BFF40C002099EC4000FD
:108DD00010B584B0002304AA42F8043D09490C6888
:108DE0000092032201462046074CA047039B3BB15B
:108DF0004FF08052054B1A60BFF34F8FBFF36F8F58
:108E000004B010BDF40C002045ED400004ED00E07E
:108E100010B582B00F4B01930123009300238022F1
:108E20000D490E480E4CA047012802D00D480E4BAC
:108E30009847002301930122009280220B490C489D
:108E4000074CA047012802D00A48074B984702B0B8
:108E500010BD00BFF40C0020803A4100B9884000EA
:108E6000ADE34000903A410015074100C03A41008F
:108E7000C9874000CC3A410070B584B004460378FD
:108E80002A2B00F086802378252B00F0868023781B
:108E9000262B00F0868023787E2B00F086802378B6
:108EA0005A2B00F0868023787A2B00F08980237873
:108EB000532B00F098802378472B00F0A180237873
:108EC000672B00F0AE802378462B00F0B580237826
:108ED000522B00F0B8802378502B00F0C880237804
:108EE0005E2B00F0EC802378492B00F0F98023788A
:108EF000432B00F008812378422B00F0088123786F
:108F0000552B00F008812378572B00F00B81237834
:108F1000562B00F01A8123784C2B00F02381237804
:108F20004D2B00F0338123784B2B00F0798123788F
:108F3000542B00F091812378442B00F09181237809
:108F4000412B00F0A4812378592B00F0C2812378B3
:108F50004E2B00F0D78123784A2B00F0D78123785D
:108F6000402B00F0D98123786F2B00F0EE8123781D
:108F7000642B00F0FC812378702B00F01A82237898
:108F80005B2B00F02F8223783D2B00F0318204B060
:108F900070BD2A20934B984775E72520914B984741
:108FA00075E726208F4B984775E77E208D4B9847B5
:108FB00075E76078000240F05A008A4B984772E7E4
:108FC000A378E27803EB0223227903EB0243627970
:108FD00003EB0263844A13606078000240F07A0079
:108FE000804B984763E7637833B901207F4B9847FC
:108FF00024207C4B98475EE700207C4B9847F7E79E
:109000006378A07800EB032080B210F4004F05D104
:10901000774B98472420734B984750E747F6FF70EB
:10902000F6E76378A07800EB032000B2714B984715
:1090300024206C4B984746E760786F4B9847242074
:10904000684B984743E76278A37803EB02239BB20F
:10905000092B05D9694A13802420624B98473AE7C7
:109060000122674B1A7045205E4B984733E76378BF
:109070005BB1012B16D00022624B1A700122604BAB
:109080001A704520574B984729E702205E4B9847B6
:1090900030B904225A4B1A704520524B98471EE7AC
:1090A0002420FAE70120584B984720B90422544B5A
:1090B0001A70452000E024204A4B98470FE7637858
:1090C0002BB1012B07D04520464B98470BE75E207C
:1090D000444B984707E74FF4AF70424B984702E77D
:1090E0006278A37803EB0223484A13800520464B9D
:1090F000984720B90422424B1A70452000E02420F2
:10910000384B9847F3E64320364B9847F3E6422026
:10911000344B9847F3E662783D4B1A705520314B3B
:109120009847F0E661780F2908D820224901A01C51
:10913000384B984724202B4B9847E8E60122304BC8
:109140001A704520274B9847E1E608202E4B984798
:1091500020B904222A4B1A70452000E02420214B1C
:109160009847D8E62C4B62781A70A2785A70E27849
:109170009A700720244B984720B90422204B1A707C
:10918000452000E02420174B9847C8E6234B98471A
:109190006378003318BF01230370A3784370E3782A
:1091A000003318BF012383702379C370637903717F
:1091B000A3794371E3798371237AC371637A03726C
:1091C000A37A4372E37A837209200F4B984720B940
:1091D00004220B4B1A70452000E02420014B9847D5
:1091E000A1E600BFD18D4000841E0020FD6E40002E
:1091F000C56E4000F16E4000C94B4000881E002043
:109200008A1E00203B1F002029A44000561F00207A
:10921000801E0020BD734000381F0020B152400066
:109220006378A27803EB0223E27803EB024322790E
:1092300003EB0263704A13606379A27903EB0223A4
:10924000E27903EB0243227A03EB02636B4A136079
:109250004B206B4B98476AE65420694B98476AE667
:1092600009226849E01C684B984748B96278674B07
:109270001A70A278664B1A704420614B98475EE6DC
:109280000122644B1A7045205D4B984757E662787F
:10929000531EDBB21F2B06D901225E4B1A704520EC
:1092A000574B98474FE6554B1A60A378E17803EB8C
:1092B0000123217903EB0143617903EB01634E49FB
:1092C0000B60A11D5448554B984741204C4B984783
:1092D00039E6002604AD45F8046D514B98470095DA
:1092E0003346012204214F4DA847039B002B3FF436
:1092F0002EAE4FF080524C4B1A60BFF34F8FBFF32E
:109300006F8F24E64E203E4B984724E6607800029B
:109310004A303B4B984722E60120444B9847404B4C
:10932000984703AB00930023012204213D4DA84739
:10933000039B002B3FF417AE4FF080523A4B1A605C
:10934000BFF34F8FBFF36F8F0DE6E21C6178A078FB
:10935000374B98470620374B984720B904222D4BAE
:109360001A70452000E02420254B9847FFE56078DF
:10937000314B9847012803D04520214B9847FAE507
:1093800024201F4B9847264B984703AB009300239C
:1093900001220421234DA847039B002B3FF4EBAD92
:1093A0004FF08052204B1A60BFF34F8FBFF36F8F87
:1093B000E1E5224B98471A4B984703AB00930023F3
:1093C00001220821174DA847039B3BB14FF0805263
:1093D000154B1A60BFF34F8FBFF36F8F2420084BDC
:1093E0009847CCE5164B98472420054B9847CAE58B
:1093F0003D20034B9847CAE57C1E00208C1E0020B0
:10940000D18D4000003B4100610D4100141E002041
:10941000781E00208A1E0020181E0020C10D410069
:109420001996400045ED400004ED00E079964000BB
:1094300021A3400029A4400099964000659D40006A
:10944000719D40008388B3F59F5F0DD0B3F5706FB9
:109450001DD0B3F5206F27D0B3F5A05F30D0B3F5A2
:10946000706F39D000207047C288B2F51F6FEDD100
:109470004289A2F5E751093989B2C6293DD9A2F539
:10948000DD521D3A92B2C62AE0D802207047C28847
:10949000B2F5F06FDDD14289A2F50B52053A92B2D6
:1094A000C62AD6D803207047C288B2F5206FD3D120
:1094B0004289A2F6553292B2C62ACDD8052070470D
:1094C000C288B2F5206FCAD14289A2F6553292B253
:1094D000C62AC4D805207047C388B3F5F06F01D001
:1094E000002070474389A3F5B8530D3B9BB2C62BB0
:1094F00001D8042070470020704701207047000009
:1095000038B50125044B1D7000210846034CA047C7
:1095100000212846A04738BDF90C00208D4F40009F
:1095200010B50024022C09D80B4B1A7800210846EC
:109530000A4B9847012801D00134F3E70024022C9C
:1095400009D8054B1A7800210120044B98470128BF
:1095500001D00134F3E710BDFA0C0020814E400029
:1095600010B5154B1B786BB90024022C15D8134B82
:109570001A78134B19880020124B984701280CD0F9
:109580000134F2E7012100200F4CA04701210846D9
:10959000A04701200D4B9847E6E70024022C0AD88B
:1095A000064B1A78064B19880120064B984701286C
:1095B00001D00134F2E710BDF90C0020FA0C0020B4
:1095C000E8000020814E40008D4F400081E64000C1
:1095D000F8B505460E460024204601E00134A4B249
:1095E0002746B4EB960F14D215F8241005EB84032C
:1095F0005A7801EB02219A7801EB0241DB7801EB0A
:1096000003610028EAD107F540608000014B9847CC
:10961000E4E7F8BD25604000014B1868704700BFC3
:10962000000D0020014B1878704700BFFD0C002092
:1096300010B582B0074B01930023009380220649A6
:109640000648074CA047012802D00648064B984719
:1096500002B010BD000D00200C404100E596400016
:10966000ADE340001840410015074100014B187858
:10967000704700BFF80C002018B9044A044B1A6068
:109680007047044A024B1A60704700BF0C3F41000C
:10969000E40000200C3B4100032817D8DFE800F06D
:1096A00002070C110A4A0B4B1A60012070470A4A44
:1096B000084B1A6001207047084A064B1A600120C7
:1096C0007047074A034B1A6001207047002070471B
:1096D0000C3F4100E40000200C3E41000C3D4100E5
:1096E0000C3C4100F0B585B001238DF80B309B4B4D
:1096F000009300231A469A499A489B4CA0479B4BDB
:10970000186004A9502301F8063D0320984CA04797
:1097100004A9002301F8073D0D20A04710B900233C
:1097200003930BE09DF80900924B9847F7E74FF041
:10973000FF3303AA002108468F4CA047039B13F078
:10974000010FF4D040F213108C4B98478C4B984784
:109750004FF480718B4B18688B4B984706E04FF0A5
:10976000FF3303AA00210846834CA047039B13F054
:10977000020FF4D01920814B9847844B4FF480722C
:109780001A63DB6B13F4004F19D0814B98470F20FD
:10979000804B984701467D487F4B984700227F4B7E
:1097A0001A700DF10B010420714B984728B19DF8F8
:1097B0000B3083F001038DF80B30002403E0784B6D
:1097C0009847E4E7002414206C4B9847002303AA31
:1097D0001C211846684DA847039B13F0080F00D0C2
:1097E000012413F0100F6FD1039B13F0040F2ED040
:1097F0006A4B1B78002B40F0FF800F20654B984789
:1098000001466248674B9847654B9847664B9847B7
:109810005B4B98475B4D4FF4807128685A4B9847D3
:109820002A68624B9A4200F0F380584BDB6B13F4CA
:10983000004F00F0F080564B98470F20554B98474B
:1098400001465248544B98472420594B9847534B54
:109850001B78002B40F0E280564B9847002840F0E0
:10986000FF8000224D4B1A709DF80B3093B1524B84
:109870001B787BB1514B1B78002B00F0D181504BF2
:10988000984738B900224D4B1A704E4B9847002824
:1098900040F0B481002C96D0484B1D78002D91D11A
:1098A0003E4B1C78002C8ED00122474B1A70474B40
:1098B00098472E4B18680A23009300231A46032169
:1098C000434CA0472C467EE70F20324B98472F4E43
:1098D00001463046334B9847314B98474FF4804709
:1098E00077630A20254DA8473A4B98474FF4FA7002
:1098F000A847394B984777630120384B9847192080
:10990000A8474FF4807333630020354EB0470120E1
:10991000B04700210846334EB04700210120B04730
:1099200001210020304EB04701210846B0470127F1
:109930001A4B1F702D4B98479DF80A1000230322E5
:1099400041F480712A4EB0472A4B984700233A468B
:109950000221B0474FF0FF30A84745E7019540008E
:10996000E0930400404041002DF04000D01E002054
:109970006174400099964000F5EB400081E640009C
:10998000815F4000E4000020D1954000000E0E40B1
:10999000A54C40003FCD40001BCD4000FD0C0020F9
:1099A000814C40001FCD4000BD5F40000C3B41009A
:1099B000B58D400019F94000E0000020EA000020C9
:1099C0009952400025964000F80C00206195400017
:1099D00069F04000117140008D704000B970400086
:1099E00019514000694F40008D4F400081A4400054
:1099F00099EC40008DA440000022974B1A70974DBF
:109A00004FF480766E631920954B98472E63F4E6E9
:109A1000944B984709E7944B98470EE7934B984728
:109A200020B1934B984700287FF416AF00258A4B4E
:109A30001D70904B98472B4603224FF480718E4E39
:109A4000B0478E4B98472B4601220421B047834DE7
:109A50004FF480766E631920814B98472E63FBE6A6
:109A6000834B984700283FF4FCAE7B4B1B78002BC0
:109A70007FF4FAAE0020824EB047824D287001205C
:109A8000B047814B18702B78002B3FF4EDAE0028C7
:109A90003FF4EAAE0122704B1A707C4D28467C4B95
:109AA000984728467B4B98470746052816D0002242
:109AB000794B1A704FF4FA70694B98470020704E3A
:109AC000B047704D28700120B0476F4B18702B784D
:109AD00003B138B90022604B1A70C5E601226E4B03
:109AE0001A70E7E7634B98479DF80A10002303229A
:109AF00041F48071604DA847604B984700230122D4
:109B00000221A84739460020644DA8473946012064
:109B1000A8470A20624B9847D8B9624D00212846D1
:109B2000614B98472B78112B18D0002108465F4DC8
:109B3000A84700210120A8470025022D20D8564B18
:109B40001A78002108465A4B9847012818D0013549
:109B5000F3E758490A20584B9847DEE76B78002B0B
:109B6000E3D1AB78002BE0D1EB78892BDDD12E4609
:109B700029460020514DA84731460120A847D4E787
:109B80000025022D09D8444B1A7800210120484BAA
:109B90009847012801D00135F3E701210020484D05
:109BA000A84701210846A8479DF80B3003B3454B51
:109BB0009847E8B1444B1B78D3B1444B1B782BB189
:109BC0000122434B1A70434B98474DE60025404B0A
:109BD0001D70414B9847414B1E68414B98470A23E3
:109BE00000932B460246012130463E4DA8473BE6F6
:109BF0000122374B1A70374B984735E60025344B16
:109C00001D70354B9847354B1E68354B98470A23D6
:109C100000932B46024601213046324DA84739E6D3
:109C2000314B984700283FF435AE0122274B1A707C
:109C30002E4B984700283FF42DAE0122244B1A707A
:109C4000244B9847254B18680A23009300231A4693
:109C50000321244DA8471DE6FD0C0020000E0E40F8
:109C600081E6400065624000814C400019F94000E7
:109C700025F9400081A4400099EC40008DA44000EB
:109C80001D614000FB0C0020FC0C00202C1F00205C
:109C90005961400045944000FA0C00208950400072
:109CA000AD744000D41E002075604000694F400034
:109CB000814E4000E8000020617440007550400073
:109CC0008D4F4000ED514000E0000020EA000020F0
:109CD000F80C00206195400021954000D01E002026
:109CE000A9E4400069F040009952400025964000E8
:109CF00038B5114B1880114B1B786BB10446002509
:109D0000022D0AD80E4B1A78214600200D4B984799
:109D1000012802D00135F3E738BD0025022D09D80E
:109D2000074B1A7821460120064B9847012801D09D
:109D30000135F3E738BD00BFE8000020F80C002033
:109D4000FA0C0020814E400010B5044B98470023C8
:109D500003221021024CA047012010BD199640009B
:109D600099EC40000022014B1A707047E00000207F
:109D70000122014B1A707047E000002038B5002422
:109D8000204609E000F47F43B3F5007F0CD000F4D7
:109D90007F43B3F5807F0CD00028F3D14FF0FF3123
:109DA0000120134B9847EDE70020124B9847002005
:109DB000EDE7C5B2002008E00134A4B220460D4B07
:109DC00098470A2101200A4B984758B9AC42F3D36F
:109DD00008E0013CA4B22046064B98470A21012026
:109DE000034B98470028D7D1AC42F2D8D4E700BF44
:109DF00071EB4000C94B4000F0B583B00224002055
:109E000010F0010F0AD14FF0FF310120314B98477C
:109E100000F00E03042BF3D10424F1E72E4B1B6852
:109E2000ADF804301B0C8DF8063001A902202B4B35
:109E30009847042C07D02A4B984701A9294B9847EB
:109E400000252E4607E0264B98470021264B9847D1
:109E5000F1E72E460225322101201E4B984700F0E3
:109E60000E00042812D0022814D0042CF3D1C5B15E
:109E7000022D22D0032DEED10136F6B2182EEAD9EA
:109E800000252E46E7E703250026E4E700252E46B9
:109E90000424E8E7124B98478021134B984702248B
:109EA000E3E70F4B9847771CFFB2104B995D0E4BC1
:109EB0009847632FCDD83E46CDE7094B9847771C8E
:109EC000FFB20B4B995D084B9847632FDBD83E469A
:109ED000C1E700BF71EB4000544041006174400095
:109EE000CDF84000515A4000015A40005001002076
:109EF000EC00002008B5044B98476420034B9847BA
:109F0000034B9847F7E700BFE164400081E640005B
:109F10001576400070B582B0944B9847944B9847A3
:109F20000120944B984702A9002301F8013D052028
:109F3000914B984728B19DF8073013B100208D4B05
:109F400098478E4B98478E4B98478E4A8E4B1A6097
:109F500001208E4B9847044690B98A4D8C4C0FCC0B
:109F600028606960AA60EB608A4B98478A4B9847E3
:109F700002228A4B1A638A4B98470546002416E052
:109F8000814B196801207C4B984705E07E4B1B688C
:109F900000221A550134E4B20F2CF7D9E4E705206A
:109FA000804B98477E4B984705460134E4B20DB983
:109FB000132CF4D97C4B984729467C4B98477C4B13
:109FC00098477C4DA8470023012211467A4CA047B0
:109FD00001207A4B9847A847002301220221A0477D
:109FE000774B98476B4B9847764B98470023012255
:109FF000052175480068A04700252C4680E01146E1
:10A00000002341F8043B7148714B984738B9714BB4
:10A010005968013159606D486F4B98477BE00121C9
:10A020006A486D4B984776E01146002341F8043B9F
:10A030006A48674B984798B9694B5968013159602C
:10A040006648654B984767496748614B984760B9D0
:10A05000634B59680131596063485F4B984768E02A
:10A0600001215E485C4B9847EDE701215E485A4B61
:10A0700098475EE0134600221A605A6801325A601F
:10A0800069465A48524B984750B9594B5968009BFA
:10A09000994201D8002514E054484F4B9847F9E7FE
:10A0A000534B596851484C4B9847F3E7514A136852
:10A0B00001331360052B44D94D4B00251D605D60B5
:10A0C00015604D4BA3FB0423DB0803EB83035A000D
:10A0D000944238D0494B9847002840F09D80484B27
:10A0E000A3FB04235B09642202FB1343002B00F053
:10A0F00096800A202B4B98470134632C00D900240A
:10A100000135B5F57A7FDCD3324A13680133136029
:10A110003B2B3FF674AF3B4B98470028C6D000223C
:10A12000344B1A602E4A1368013313603B2B3FF601
:10A130007BAF2F4A1368013313603B2B9AD800255D
:10A14000BFE70025BDE7304B984728B947232F4A82
:10A1500013702F4A1370BDE700202E4EB0472B4BD3
:10A1600018700120B0472A4B1870B3E7F17A40000D
:10A1700049754000754C400061744000814C4000BE
:10A18000BD4A40005C1F00203C1F0020AD74400011
:10A190000C414100CDF84000E95B4000000E0E404C
:10A1A0004165400081E64000C5F84000B15C4000D8
:10A1B0008D7040001996400099EC4000B970400045
:10A1C000295140003D594000280D00200110FFFF9B
:10A1D00085784000180D0020CD7840000210FFFF68
:10A1E000080D00200C0D00200410FFFF0310FFFFDE
:10A1F000100D0020040D0020CDCCCCCCED51400042
:10A200001F85EB516D96400025964000B40100205B
:10A21000B5010020FD4F4000024B984769E7024B13
:10A22000984766E7F95140002951400008B509E018
:10A23000002108462D4CA04700210120A047002204
:10A240002B4B1A704FF0FF3101202A4B9847284BB7
:10A250001B78013B082BF2D801A252F823F000BF73
:10A2600085A2400031A240009FA24000AFA2400062
:10A2700095A24000D7A24000BFA24000CBA2400060
:10A28000D1A2400001210020184CA047012108461E
:10A29000A047D4E7184B1888184B9847CFE7002100
:10A2A0000846174CA04700210120A047C7E701211D
:10A2B0000020134CA04701210846A047BFE7114BDF
:10A2C00098471149114B9847B9E7114B9847B6E7A2
:10A2D000104B9847B3E7104AD01E134612F8032CD0
:10A2E000817840780D4CA047A9E700BFDD4F4000C2
:10A2F0003B1F002071EB4000561F0020F19C4000E6
:10A300008D4F4000CDF84000381F0020515A4000CA
:10A3100001744000BD5240006F1F0020C14D40003D
:10A3200010B51446044B1870597002462146981C0B
:10A33000024B984710BD00BF6C1F0020C10D4100AB
:10A3400010B582B0234B0193032300930023802296
:10A3500021492248224CA047012802D02148224B03
:10A360009847224B019300230093802220492148E3
:10A370001B4CA047012802D01F481B4B98470023C5
:10A380000193009380221D491D48154CA0470128C8
:10A3900002D01C48144B98471B4B01930023009399
:10A3A00080221A491A480E4CA047012802D01948A9
:10A3B0000D4B9847184B01930023009380221749B7
:10A3C0001748074CA047012802D01648064B98476B
:10A3D00002B010BD240D0020584041002DA24000C5
:10A3E000ADE340005C404100150741002C0D00200A
:10A3F00078404100159F400084404100AC4041003E
:10A40000F59E4000B0404100280D0020CC404100A6
:10A41000F99D4000D0404100200D0020EC4041005B
:10A420007D9D4000F040410010B584B0104B187085
:10A430000022039204AB43F8082D0E4A106803AAC9
:10A440000092042201210C4CA047029B5BB9039BA4
:10A4500063B14FF08052094B1A60BFF34F8FBFF3C7
:10A460006F8F012000E0002004B010BD0120FBE749
:10A470003B1F0020240D002045ED400004ED00E0CE
:10A48000014B1868704700BF200D0020014B186871
:10A49000704700BF280D00200023044A1370044AAF
:10A4A00013700120034B1870704700BF380D002057
:10A4B000340D0020300D0020704700207047000050
:10A4C0000D4B5B881A0A032A01D00020704713F055
:10A4D000FF0F0ED1084BDB88402B01D000207047C6
:10A4E000054B064A9A60064A1A6140229A81012069
:10A4F00070470020704700BFD01F00203C0D002097
:10A5000035A540000122014B1A707047300D002024
:10A5100010B5034B034A04490448054CA04710BD3D
:10A52000C1A4400088020020340D0020380D002016
:10A5300055A6400008B5044B9B89402B00D008BDB0
:10A540000248034B9847FAE7D01F00203C0D00203B
:10A55000798E4000224B1B780BB9184670472DE9C5
:10A56000F04184B00746EFF31083B3FA83F35B093D
:10A57000039372B6BFF35F8F00211A4B1970DDF899
:10A580000C80194D40222846184B98473C464037CE
:10A590002E4620686168A268E3680FC6103435460D
:10A5A000BC42F5D1124B009340230F4A0021812079
:10A5B000104CA04780F00100094B1870B8F1000F53
:10A5C00005D00122074B1A70BFF35F8F62B6044BB0
:10A5D0001B7883F00103184604B0BDE8F08100BF8A
:10A5E000300D0020EB0200207C0D0020BD0F41004B
:10A5F00005A5400031C8400010B50446134B9847EC
:10A60000837A212B01D0002010BD00F10902104BEC
:10A610005B881B0A212B04D0C27B93420BD0002005
:10A6200010BD0B4B9A60427AD9888A4228BF0A46ED
:10A630009A81012010BD064B9C60028AD9888A420B
:10A6400028BF0A469A81012010BD00BF2DAC4000F2
:10A65000D01F0020F8B5264C247865B2002D07DB0A
:10A66000002D40DB04F06004202C22D00020F8BD37
:10A6700014F0600603D11E4F7F78062F0BD0202EDA
:10A68000EED11B4A5278022A09D0032A0CD0012AA3
:10A69000E6D19847F8BD1046164B9847F8BD144BC5
:10A6A000986001209881F8BD114B99600120988134
:10A6B000F8BD0F4A52780A2A07D00B2A0BD0092A74
:10A6C00001D00020F8BD9847F8BD094B5B881B0AF4
:10A6D00003700120F8BD064BDB8833B9044B5B885F
:10A6E0000B700120F8BD0020F8BD0020F8BD00BFB0
:10A6F000D01F0020F9A54000014B1868704700BF2B
:10A700003C1F0020024B1B681B6858881844704788
:10A71000C80D002038B504460D46094B984702463F
:10A7200020782044904207D24378042B06D0AB42D5
:10A7300005D003781844F5E7002038BD002038BD67
:10A7400005A7400038B5144B1B780BB3134B1B689F
:10A750001B681A7982421DD90D460446104A1360BF
:10A76000104B984703E01A7813440D4A13600C4BC2
:10A770001B6898420AD95A78042AF4D19A789442EC
:10A78000F1D1DA78AA42EED1012038BD002038BDDF
:10A79000002038BD002038BDC40D0020C80D0020A9
:10A7A000CC0D002005A74000084BDB8863B9074BA0
:10A7B0005B88012B01D000207047054A138823F0E5
:10A7C000020313800120704700207047D01F002033
:10A7D000BC0D002000207047044BDB8823B9044ADD
:10A7E000024B1A610120704700207047D01F0020E3
:10A7F0001DAB400038B5134B1B7803B3124B1C79CB
:10A80000124B1B681B681B799C4201D3002317E085
:10A81000002120460E4B9847034688B10B4B1B681E
:10A820005B6853F82450EB68984701462046084B74
:10A830009847034620B1AB689847034600E00023E1
:10A84000184638BDC40D0020D01F0020C80D0020C0
:10A8500045A7400038B5104B1B78D3B100240F4BEF
:10A860001B681A681279944211D25B6853F824501D
:10A87000EB68984701462046094B9847034648B184
:10A88000AB689847034628B90134E4B2E7E70023F0
:10A8900000E00023184638BDC40D0020C80D00207C
:10A8A00045A7400070B504460021114B9847054666
:10A8B00008B9284670BD0F4B1B685B6853F82460CD
:10A8C000F368984701462046094B984705460028FB
:10A8D000EFD0094B1C6805212046084B98470446D9
:10A8E00018B18078064B9847F5E773689847E0E71A
:10A8F00045A74000C80D0020CC0D002015A7400042
:10A90000B1C5400008B5064BDB88022B01D0002002
:10A9100008BD02210348044B9847012008BD00BF31
:10A92000D01F0020BC0D002095C4400010B5184B6E
:10A930009B78032B2AD8DFE803F00502100B0920CF
:10A94000144C0CE004211448144B9847002006E0F6
:10A95000134B98470446102001E00620114C08B123
:10A96000002308E0012010BDE15C0F4A02EB430226
:10A9700051800133DBB28342F6D3411C4900C9B296
:10A9800009480170054B9847012010BD002010BDFB
:10A99000D01F0020D8020020D402002095C440001F
:10A9A000F9A64000E4020020B002002008B5234BC5
:10A9B0005B88DAB21B0A013B0E2B38D8DFE803F0C4
:10A9C00008173137373737373737373737372A00B0
:10A9D0001B4B186801781B4B9847184BDA889B89EA
:10A9E0009A4228D2154B9A810123184608BD144B70
:10A9F0001B685B7C9A4201D30023F6E7104B5B682F
:10AA000053F8320041880F4B98470C4B9B68022249
:10AA10005A70E2E70A4B986858B14188094B984749
:10AA2000DBE7094B984703460028D6D1DDE7002332
:10AA3000DBE70023D9E70123D7E700BFD01F0020C1
:10AA4000B801002095C440002DA9400008B5064B70
:10AA5000DB88012B01D0002008BD01210348044BF5
:10AA60009847012008BD00BFD01F0020C40D002062
:10AA700095C4400038B5154BDB88012B02D000246B
:10AA8000204638BD124B1B78F3B1104B1D79114B8A
:10AA90001B681B681B799D4201D30024F0E700214D
:10AAA00028460D4B984704460028E9D0094B1B68FF
:10AAB0005B6853F82530DB689847084B1870012114
:10AAC0001846074B9847DBE70024D9E7D01F002042
:10AAD000C40D0020C80D002045A74000C00D002077
:10AAE00095C4400008B5094BDB88022B01D000203B
:10AAF00008BD064B1879064B9847064B1880022173
:10AB00001846054B9847012008BD00BFD01F002004
:10AB100001C64000BE0D002095C4400008B5034B9F
:10AB2000588800F07F00024B984708BDD01F0020D6
:10AB30003DC4400038B505460F4B98470346C0B1A9
:10AB40000E4B1C68052120460D4B9847044640B12A
:10AB50008288C17880780B4B984703460028F1D152
:10AB600007E0094B1B685B6853F825301B68984762
:10AB70000346184638BD00BF45A74000CC0D002055
:10AB800015A74000A1C44000C80D002038B50C4BEB
:10AB9000DB8893B90B4B1B780BB900230EE0084BF5
:10ABA0001C799D782046084B9847034630B12946CA
:10ABB0002046064B9847034600E00023184638BD60
:10ABC000D01F0020C40D0020A5A8400035AB4000D8
:10ABD00008B5074BDB884BB9054B5B880BB10020F0
:10ABE00008BD034B1879034B984708BD002008BDEA
:10ABF000D01F00203DC74000094BDB886BB9084BD4
:10AC00005B880BB10020704710B5054C2079054BCF
:10AC100098472079044B984710BD0020704700BF2B
:10AC2000D01F0020ADC9400045C64000014B186848
:10AC3000704700BFCC0D002008B5014B984708BDF8
:10AC4000DDC2400010B50B4B1B7863B1002404E05B
:10AC50002046094B98470134E4B2084B1B681B6837
:10AC60001B799C42F4D30022024B1A700122044B40
:10AC70001A8010BDC40D0020A5A84000C80D0020FA
:10AC8000BC0D002008B5024B9847024B984708BD01
:10AC9000C5C3400045AC40001C4BDB8813B100230A
:10ACA0001846704710B51A4B984750B3174B9A780F
:10ACB000184B1B685B7C9A4201DD002322E0164B97
:10ACC0009847124B9B78154A1370EBB1114A5268A2
:10ACD00003F10053013B02EBC303114A136000244C
:10ACE0000F4B1B681B681B799C4208D20021204631
:10ACF0000C4B9847034628B10134E4B2F0E7012336
:10AD000000E00023184610BD0123FBE7D01F002000
:10AD100079C44000B801002045AC4000C40D0020BB
:10AD2000C80D002035AB400008B5344B1B7813F03C
:10AD3000800F0ED113F01F0343D1304A5278013AED
:10AD4000082A3ED8DFE802F0343D373D313D3D3D35
:10AD50003A002A4AD288002A4ED013F01F0306D1A7
:10AD6000264A5278062A0BD0082A0CD02AB1012B89
:10AD70000CD0022B11D0002008BD214B984708BDF4
:10AD8000204B984708BD204B984708BD1B4A527876
:10AD90000A2AEED11D4B984708BD184B5B780BB1C2
:10ADA000002008BD1A4B984708BD1A4B984708BDAC
:10ADB000194B984708BD194B984708BD184B984741
:10ADC00008BD012B03D0022B08D0002008BD0B4A80
:10ADD00052780B2AF7D1134B984708BD074B5B7885
:10ADE000012B03D0032B04D0002008BD0E4B984745
:10ADF00008BD0E4B984708BD002008BDD01F00209D
:10AE000005A94000ADA940004DAA400075AA400028
:10AE1000E5AA4000D9A74000A9A74000D5A7400057
:10AE200099AC40008DAB4000D1AB4000F9AB400085
:10AE30000B4B1B7813B110B5002402E070470134AE
:10AE4000E4B2084B1B681A681279944207D25B6817
:10AE500053F824301B69002BF1D09847EFE710BD61
:10AE6000C40D0020C80D002008B5184B00229A819F
:10AE70001A615A611B7813F0800F11D113F0600F23
:10AE800014D0124B1B7803F01F03012B14D00F4B6F
:10AE90001B7803F01F03022B14D00023184608BDB3
:10AEA0000A4AD288002AE9D10023F7E7084B9847DD
:10AEB00003460028E5D0F1E7064B984703460028F3
:10AEC000E5D0EBE7044B98470346E7E7D01F0020A7
:10AED00029AD4000F5A7400055A84000F8B504464C
:10AEE0000E46114B984705462046104B98470540A3
:10AEF00001D0002403E0F8BD0134062C11D88DB137
:10AF000023010B4AD058B042F6D102EB0413596822
:10AF10000D42F1D01F46DB6898477B6825EA0305A0
:10AF2000EAE7F8BDF8BD00BF23CD400027CD4000C3
:10AF3000D00D0020F8B5164C2768062F26D800241F
:10AF400001E00134E4B2A446A7420AD3114E250120
:10AF500006EB050E75598D42F3D1DEF8045095428B
:10AF6000EFD1CEF80010CEF80420CEF808300699C4
:10AF7000CEF80C100137BC4505D011461A46064BD9
:10AF800098470020F8BD02490F60F6E70120F8BDA0
:10AF9000400E0020D00D0020E9CC40002DE9F0410A
:10AFA00082B004460F4690460A4B98470546204615
:10AFB000094B984706462046084B9847CDF8008035
:10AFC0003B46024631462846054CA04702B0BDE844
:10AFD000F08100BF2BCD400039CD40003FCD400077
:10AFE00035AF400008B50B210148024B984708BD1A
:10AFF000000E0E40DDAE400008B50C210148024BAA
:10B00000984708BD00100E40DDAE4000F8B506467A
:10B010000C461546224B984707464FF0FF31304605
:10B02000204B98473046204B9847002C0CDB630997
:10B0300004F01F0101228A4020331C4941F82320DB
:10B04000BFF34F8FBFF36F8F002C08DB630904F051
:10B050001F0101228A406033144941F82320002C4B
:10B0600017DB2D01EDB204F1604303F5614383F872
:10B070000053002C08DB620904F01F04012303FACB
:10B0800004F40A4B43F8224039463046084B9847AF
:10B09000F8BD04F00F022D01EDB2064B9D54E8E718
:10B0A00027CD40001FCD400023CD400000E100E04F
:10B0B0001BCD400014ED00E082B0024610B9244BD5
:10B0C0001B783BB912B1224B1B780BB3204B1A7083
:10B0D00002B070471F4B1B7803B9FEE7EFF31083F4
:10B0E000B3FA83F35B09009372B6BFF35F8F00215D
:10B0F000194B1970009817490B78013B0B70002809
:10B10000E0D00121144B1970BFF35F8F62B6D9E70D
:10B11000104B1B78FF2B19D0EFF31083B3FA83F396
:10B120005B09019372B6BFF35F8F00210A4B197060
:10B13000019808490B7801330B700028C6D0012113
:10B14000054B1970BFF35F8F62B6BFE7FEE700BF24
:10B15000450E0020E81F0020EB02002084B02A4B9F
:10B160009A6842F480729A609A6822F07F029A602C
:10B170001A6B0192019A42F04F020192019A22F455
:10B18000074222F080020192019A42F400420192A9
:10B19000019A1A631C4B1B6B13F4004FFAD01A4A26
:10B1A000136B0293029B43F04F030293029B43F401
:10B1B00000430293029B136300238DF8033006E0E3
:10B1C00000BF9DF803300133DBB28DF803309DF8EA
:10B1D0000330DBB2132BF3D9EFF31083B3FA83F30D
:10B1E0005B09039372B6BFF35F8F0022074B1A709F
:10B1F000039B0121044A116123B1044B1970BFF371
:10B200005F8F62B604B0704700400440EB0200203C
:10B21000034A0023136153619381024A13707047FC
:10B22000D01F00204A0E002082B00522104B1A7059
:10B23000104A136B0193019B43F04F030193019B51
:10B2400043F020030193019B136300238DF8033027
:10B2500006E000BF9DF803300133DBB28DF8033008
:10B260009DF80330DBB2132BF3D902B0704700BF57
:10B270004A0E00200040044082B00322104B1A7096
:10B28000104A136B0193019B43F04F030193019B01
:10B2900043F010030193019B136300238DF80330E7
:10B2A00006E000BF9DF803300133DBB28DF80330B8
:10B2B0009DF80330DBB2132BF3D902B0704700BF07
:10B2C0004A0E0020004004400422014B1A707047CF
:10B2D0004A0E002008B5024B1B6903B1984708BD10
:10B2E000D01F002030B589B06A4B1B78032B29D0C2
:10B2F000694B9C89694B1B88E41AA4B2002C43D18A
:10B30000674A11880B449BB21380634AD2889342E8
:10B3100003D0644B1B78002B2CD0634B9847634AB7
:10B32000136B0393039B43F04F030393039B23F09F
:10B3300001030393039B13635C4B1B6B13F0010F1F
:10B34000FAD115E0594A136B0293029B43F04F0365
:10B350000293029B23F001030293029B1363534B5E
:10B360001B6B13F0010FFAD1514B9847514B984783
:10B3700009B030BD484B5B6933B1984720B100221A
:10B38000464B1A80444B9C893F2C37D90022454BB1
:10B390001A704024404B9A68404B1B881A44EFF3C4
:10B3A0001083B3FA83F35B09079372B6BFF35F8F21
:10B3B0000021414B197007983C4B1B6B13F0020F97
:10B3C0003ED028B101223C4B1A70BFF35F8F62B6AA
:10B3D0000422304B1A70354A136B0493049B43F0DC
:10B3E0004F030493049B23F001030493049B136312
:10B3F0002E4B1B6B13F0010FFAD1B9E70122294B39
:10B400001A70C7E7157829490D650133DBB201329F
:10B4100099B28C42F6D8214B1A8814441C80234AD6
:10B42000136B0593059B43F04F030593059B43F076
:10B4300010030593059B136300238DF8073008E084
:10B440000023E5E700BF9DF807300133DBB28DF83C
:10B4500007309DF80730DBB2132BF3D9134A136B77
:10B460000693069B43F04F030693069B23F00103CC
:10B470000693069B13630D4B1B6B13F0010FFAD160
:10B4800000283FF475AF01220B4B1A70BFF35F8F9A
:10B4900062B66DE74A0E0020D01F0020460E002045
:10B4A000480E0020440E0020C9B240000040044075
:10B4B000D5B2400011B24000EB02002010B586B0BA
:10B4C000654B1B78012B1ED0022B04D0042B02D01D
:10B4D000624B984701E0624B9847624A136B0093B6
:10B4E000009B43F04F030093009B23F00203009363
:10B4F000009B13635B4B1B6B13F0020FFAD15A4B8B
:10B50000984706B010BD574B186BC0F30A40574B15
:10B510009B89574A14882218934201DA181B80B27B
:10B52000524B9A682244002305E04E49096D117080
:10B530000133DBB2013299B28842F6D80444A4B296
:10B540004B4B1C8040281BD0484B9C815B6913B13E
:10B550009847002832D0434A136B0293029B43F072
:10B560004F030293029B23F002030293029B136397
:10B570003C4B1B6B13F0020FFAD13E4B9847C0E7D0
:10B580003A4BDA883C4B1B8823449A42DCDD374B2C
:10B590009B899C4227D0334A136B0593059B43F04C
:10B5A0004F030593059B23F002030593059B13634B
:10B5B0002C4B1B6B13F0020FFAD1A2E7274B9847D5
:10B5C000284A136B0193019B43F04F030193019BA6
:10B5D00023F002030193019B1363224B1B6B13F0B7
:10B5E000020FFAD18DE7214B5B6953B19847E8B15F
:10B5F00021491F4A0B88108803440B8000231380C5
:10B60000C9E7164B9847174A136B0393039B43F004
:10B610004F030393039B23F002030393039B1363E2
:10B62000104B1B6B13F0020FFAD16AE70B4B9847D4
:10B630000C4A136B0493049B43F04F030493049B45
:10B6400023F002030493049B1363064B1B6B13F05C
:10B65000020FFAD155E700BF4A0E002029B2400080
:10B66000D5B240000040044011B24000D01F00207D
:10B67000460E002079B24000480E00200023042B23
:10B6800014D810B40A499A00D418A00004460844FB
:10B69000407C214400F083026FF3C7124A740133E7
:10B6A000DBB2042BEED95DF8044B7047704700BF46
:10B6B0004C0E002038B5437C13F0100F16D00D4609
:10B6C000437C6FF30413437404687CB102F10C03F0
:10B6D000074951F8233013F4806F01D042F0800203
:10B6E0008168012D14BF00200120A04738BD00BF94
:10B6F0000040044010B500240BE023460134E4B2BE
:10B7000003EB8303980022460121034B1844034BAB
:10B710009847042CF1D910BD4C0E0020B5B640005E
:10B7200010B500F00F02531E03EB83039C000121B0
:10B7300002482044024B984710BD00BF4C0E002029
:10B74000B5B6400030B482B00246441E3B4900F119
:10B750000C0551F8253051F8251013F0020302D0E2
:10B7600001F0400151B9002B39D004EB840399005A
:10B77000334B0B44597C6FF38301597404EB8403FE
:10B7800099002F4B0B445B7C13F00C0F32D12B49EB
:10B7900000F10C0551F825300093009B43F04F0356
:10B7A0000093009B23F002030093009B41F8253097
:10B7B00002F10C03214951F8233013F0020FF7D1A5
:10B7C000002838D0032836D004EB8404A2001C4B98
:10B7D00013445A7C012161F383025A742BE004EB79
:10B7E00084039900164B0B44597C012565F38301B2
:10B7F0005974C3E711490C3051F820300193019B73
:10B8000043F04F030193019B23F040030193019BFD
:10B8100041F8203002F10C03084951F8233013F0AD
:10B82000400FF7D104EB8404A200054B13445A7C6B
:10B830006FF383025A7402B030BC7047004004407A
:10B840004C0E0020F0B4461EB300334499002A4A3F
:10B850000A445368D1680B449468641A128AC2F38C
:10B860000902944209D31446002706EB860295008C
:10B87000214A2A442144D1601EE00127F5E71D78C2
:10B880001E4A00F1140142F821505D7842F821501F
:10B890009D7842F82150DD7842F821501D7942F818
:10B8A00021505D7942F821509D7942F82150DD798F
:10B8B00042F82150083C0833072CE0D807E01D78F7
:10B8C00000F114020D4941F82250013C0133002CD3
:10B8D000F5D1094BB1008819820010461A44527CF8
:10B8E000C2F3810203440132597C62F3830159742B
:10B8F0003846F0BC704700BF4C0E002000400440AA
:10B9000070B582B0441E04EB84039A00364B134496
:10B910005B7CC3F3810328B1032801D0022202E03B
:10B92000012200E001229A4254DDA2002244950047
:10B930002D4B2B44DA689B689A4205D32A4B2B4443
:10B940005B7C13F0400F48D00E460546274B9847C6
:10B95000FEB1274A0C3552F825300193019B43F084
:10B960004F030193019B43F010030193019B42F8A5
:10B97000253000238DF8033006E000BF9DF803302A
:10B980000133DBB28DF803309DF80330DBB2132BAB
:10B99000F3D940B104EB84039A00134B13445A7C4F
:10B9A0006FF386125A74A200224491000E4B0B448E
:10B9B000DA689B689A4212D30B4B0B445B7C13F002
:10B9C000400F0ED1084B0B445A7C42F080025A744F
:10B9D000002000E0012002B070BD0020FBE7012044
:10B9E000F9E70120F7E700BF4C0E002045B8400002
:10B9F000004004402DE9F84305468446471EBB003D
:10BA00003B449A002A4C1444A268E368A2EB030E5C
:10BA1000B4F81080C8F3090862681A440C3025494C
:10BA200051F82060C6F30A4666B3B6450BD9B64650
:10BA30004FF0000907EB870188001D49014473445A
:10BA4000CB6000210AE04FF00109F3E70CF1140389
:10BA5000184850F823301370013101328E45F5D863
:10BA60002846154B9847B9F1000F01D1B04507D9C9
:10BA700005F10C030F4A52F8233013F0200F04D0C5
:10BA8000BDE8F8834FF00009EAE70123AB405361BA
:10BA9000074ABB00D819810008461144C96802440E
:10BAA00091602A4600212046044B9847E8E700BFF2
:10BAB0004C0E00200040044045B74000B5B64000A1
:10BAC0002DE9F0418CB00124ADE12046B34B9847FD
:10BAD0000120FAE1BB003B449900B14A0A44537C7F
:10BAE000C3F38101033161F383035374537C13F077
:10BAF000200F00F0848013F00C0F3BD0A94A04F112
:10BB00000C0152F821300193019B43F04F03019344
:10BB1000019B43F010030193019B42F82130002365
:10BB20008DF8013006E000BF9DF801300133DBB233
:10BB30008DF801309DF80130DBB2132BF3D9994A0F
:10BB400006F10C0152F821300293029B43F04F039F
:10BB50000293029B23F001030293029B42F82130DF
:10BB600006F10C038F4A52F8233013F0010FF7D17E
:10BB70000120AAE18B4A04F10C0152F82130039311
:10BB8000039B43F04F030393039B23F001030393B1
:10BB9000039B42F8213006F10C03824A52F823300D
:10BBA00013F0010FF7D1114606F10C0352F82320D0
:10BBB0000492049A42F04F020492049A42F0200246
:10BBC0000492049A41F8232000238DF8023006E005
:10BBD00000BF9DF802300133DBB28DF802309DF8D2
:10BBE0000230DBB2132BF3D907EB8707BA006C4B9B
:10BBF00013445A7C6FF345125A74012065E113F027
:10BC0000800F42D1BB003B449A00654B1344DA6875
:10BC10009B689A424CD307EB87039A00604B13440E
:10BC20005B7C13F04C0F43D1EFF31083B3FA83F333
:10BC30005B090B9372B6BFF35F8F00225A4B1A70E9
:10BC40000B9B584A55612BB10122574B1A70BFF319
:10BC50005F8F62B6534A06F10C0152F8213005930A
:10BC6000059B43F04F030593059B23F001030593C8
:10BC7000059B42F8213006F10C034A4A52F8233062
:10BC800013F0010FF7D101201FE1BB003B449A00E4
:10BC9000434B1344597C6FF3C7115974DA689A60A7
:10BCA000404B5D61224600214046404B9847A9E742
:10BCB000002C4AD0032C48D007EB87039A00384B5E
:10BCC00013445B7C13F00C0F3FD0364A06F10C0195
:10BCD00052F821300693069B43F04F030693069BD0
:10BCE00043F010030693069B42F8213000238DF8A1
:10BCF000033006E000BF9DF803300133DBB28DF85E
:10BD000003309DF80330DBB2132BF3D9254A06F13B
:10BD10000C0152F821300793079B43F04F03079320
:10BD2000079B23F001030793079B42F8213006F19C
:10BD30000C031C4A52F8233013F0010FF7D10021F5
:10BD400020461B4B98470120BFE0002C4AD0032C13
:10BD500048D001212046164B984758B3114A06F1A6
:10BD60000C0152F821300893089B43F04F030893CD
:10BD7000089B23F001030893089B42F8213006F149
:10BD80000C03084A52F8233013F0010FF7D10021B9
:10BD90002046074B9847012097E000BFF5B94000C7
:10BDA0004C0E002000400440EB020020B5B64000DD
:10BDB00001B940004749BB00D81982000A4492F8F3
:10BDC00011E06FF3C71E82F811E0D2681F44BB0078
:10BDD00019448A60404B5D612246002140463F4B3A
:10BDE0009847BBE7012120463D4B98473A4A06F168
:10BDF0000C0152F821300993099B43F04F0309933A
:10BE0000099B23F001030993099B42F8213006F1B5
:10BE10000C03314A52F8233013F0010FF7D10120FF
:10BE200053E00134E4B2052C4ED82B4B9B692646D7
:10BE30000125A5402B42F4D0671E07EB8702930033
:10BE4000244A02EB030804F10C03234A52F823307E
:10BE500013F0420F7FF439AE04F10C031E4A52F87E
:10BE6000233013F0010F7FF435AE04F10C031A4AAE
:10BE700052F8233013F0080FD3D004F10C0152F81C
:10BE800021300A930A9B43F04F030A930A9B23F045
:10BE900008030A930A9B42F8213006F10C030E4A6C
:10BEA00052F8233013F0080FF7D106F10C0352F8C3
:10BEB000233003F4E063B3F5807F09D006F10C036F
:10BEC00052F82330012000E000200CB0BDE8F081E2
:10BED0000120FAE74C0E002000400440B5B64000B7
:10BEE00001B9400000B587B0534B1B78E3B9534B01
:10BEF0001B6BC3F30A43082B3BD0504A136B0193CF
:10BF0000019B43F04F030193019B23F00403019332
:10BF1000019B1363494B1B6B13F0040FFAD1484B81
:10BF2000984707B05DF804FB464B9847464B984747
:10BF3000DDE7424A116D454A99540133DBB2072BC4
:10BF4000F7D9434B9847B0B93C4A136B0293029B15
:10BF500043F04F030293029B23F004030293029BDE
:10BF60001363364B1B6B13F0040FFAD1344B984715
:10BF7000D7E70023E3E7354B93F90030002B1EDBB6
:10BF80002E4A136B0593059B43F04F030593059BC6
:10BF900023F004030593059B1363284B1B6B13F0DD
:10BFA000040FFAD1294BDB88002B42D00023294A09
:10BFB0001380294A138001221F4B1A70B1E71F4AD0
:10BFC000136B0393039B43F04F030393039B43F0D3
:10BFD00080030393039B136300238DF8033006E073
:10BFE00000BF9DF803300133DBB28DF803309DF8BC
:10BFF0000330DBB2132BF3D9104A136B0493049B69
:10C0000043F04F030493049B23F004030493049B25
:10C0100013630A4B1B6B13F0040FFAD100230D4A74
:10C0200013800D4A13800222034B1A700B4B984762
:10C0300077E70B4B984774E74A0E00200040044016
:10C0400029B24000D5B2400011B24000D01F0020FC
:10C0500069AE4000480E0020460E0020E5B24000C8
:10C0600079B24000204BDB6913F0010F37D000B5E7
:10C0700083B01D4B1B6B13F0040F24D11A4B1B6BA9
:10C0800013F0010F23D1184B1B6B13F0020F22D1B9
:10C09000154B1B6B13F0080F23D0134A136B01933E
:10C0A000019B43F04F030193019B23F0080301938D
:10C0B000019B13630C4B1B6B13F0080FFAD101208B
:10C0C00003B05DF804FB094B98470120F8E7084BE3
:10C0D00098470120F4E7074B98470120F0E700203C
:10C0E00070470020ECE700BF00400440E5BE400080
:10C0F000E5B24000BDB4400010B54C4B984720B9A4
:10C100004B4BDB6913F4807F10D03020494B9847AC
:10C11000474B9B6913F4006F04D0454BDB6913F464
:10C12000006F0AD1444B984770B110BD72B6BFF38F
:10C130005F8F0022414B1A7010BD4FF400623C4BE0
:10C140001A623F4B984710BD3E4B98470028ECD1F0
:10C15000374B9B6913F4005F04D0354BDB6913F454
:10C16000005F3DD1324B9B6913F4007F04D0304B0C
:10C17000DB6913F4007F33D12D4B9B6913F4806F7F
:10C1800004D02B4BDB6913F4806F29D1284B9B69BA
:10C1900013F4807F04D0264BDB6913F4807F2FD10A
:10C1A000234BDB6913F4805FBFD0214C4FF48053E5
:10C1B0002362254B9847254B9847636823F001037A
:10C1C0006360636823F002036360214B9847214B4F
:10C1D00098474FF4807323614FF400632361A4E711
:10C1E000134C4FF418532362636101201A4B984794
:10C1F0004FF48073236223614FF40063236110BD09
:10C200000B4B4FF480721A625A614FF400521A615C
:10C210004FF400721A614FF480621A6130200F4BA4
:10C22000984700200C4B984710BD00BF99D24000A2
:10C230000040044061D1400065C04000EB02002096
:10C2400031AE4000C1BA4000F5B6400045AC4000F8
:10C250005DB1400011B24000B9B04000B5D140001E
:10C2600010B582B0EFF31083B3FA83F35B09019347
:10C2700072B6BFF35F8F0022144B1A70019C01202D
:10C28000134B98473020134B9847134B5A6F22F4A7
:10C2900080725A675A6F42F400725A674FF4807284
:10C2A0001A614FF400521A614FF400721A614FF490
:10C2B00080621A614FF400621A612CB10122034BB3
:10C2C0001A70BFF35F8F62B602B010BDEB020020A0
:10C2D000B9B0400061D140000040044030B583B0A7
:10C2E000EFF31083B3FA83F35B09009372B6BFF3E5
:10C2F0005F8F0024204B1C70009D204B98473020FE
:10C300001F4B98471F4B98471F4B502283F83023F1
:10C310004FF480325A601D4B98474FF480201C4BDD
:10C3200098471C4B1C701C4B1B78FF2B22D0EFF343
:10C330001083B3FA83F35B09019372B6BFF35F8F87
:10C3400000220D4B1A700199134A137801331370B0
:10C3500029B10122084B1A70BFF35F8F62B60F4BF1
:10C3600098472DB10122044B1A70BFF35F8F62B65C
:10C3700003B030BDFEE700BFEB02002065CB4000FC
:10C3800061D140004DCD400000E100E07DB64000AD
:10C3900085D24000450E0020E81F002061C2400009
:10C3A00008B5064B5A6F42F480725A675A6F22F4EE
:10C3B00000725A670020024B984708BD00400440B5
:10C3C000B9B0400010B582B0EFF31083B3FA83F335
:10C3D0005B09009372B6BFF35F8F0022144B1A7093
:10C3E000009C144B9847144B1B7803B9FEE7EFF3FE
:10C3F0001083B3FA83F35B09019372B6BFF35F8FC7
:10C4000000220B4B1A7001990B4A1378013B1370F1
:10C4100029B10122064B1A70BFF35F8F62B62CB1AF
:10C420000122034B1A70BFF35F8F62B602B010BDDA
:10C43000EB020020A1C34000E81F00200D4B5A680A
:10C4400022F001025A609A6822F480729A600246D1
:10C4500070B1986820F07F0002F07F02104398606E
:10C460009A6842F480729A605A6842F001025A60F7
:10C47000704700BF00400440054B5B6813F0010F9C
:10C4800004D0034B986800F07F007047002070478D
:10C4900000400440014B986099817047D01F0020F4
:10C4A000F0B583B045B200F00F00052873D801F055
:10C4B0000306044600F10C033B4F57F8233013F4F6
:10C4C000004F6BD1012E53D0031FDBB2012B54D987
:10C4D0004023934266DB461E06EB8607334B03EB95
:10C4E000870303F11007B3F810E062F3090EA3F815
:10C4F00010E05B7C03F07F036FF345137B70002D2E
:10C500003EDB294EB36A012282401343B362264BBD
:10C510009B6A1A42FBD0244B9E6A26EA02029A6268
:10C5200000F10C0253F822300193019B43F04F03BA
:10C530000193019B23F4074323F080030193002D13
:10C5400023DB0A0202F4407242F40042019B1343CF
:10C55000019301990C30144B43F8201004F10C03A3
:10C56000114951F8233032EA0303F7D1012013E0D7
:10C57000B0B10328A8D100200EE04FF40073A8E763
:10C580007B786FF383037B70BBE70A0202F440728F
:10C5900042F40442DAE7002003B0F0BD0020FBE7DC
:10C5A0000020F9E70020F7E7004004404C0E00208F
:10C5B00000F00F03052B1ED810B582B019460E4CA3
:10C5C0000C3354F823200192019A42F04F02019259
:10C5D000019A22F400420192019A44F8232001F1C9
:10C5E0000C03054A52F8233013F4004FF7D1034BE4
:10C5F000984702B010BD70470040044021B740008A
:10C6000000F00F00431E052815D803EB83039A00A2
:10C610000A4B13445B7C13F0200F08D10C30084BFD
:10C6200053F8203013F0280F03D001207047012069
:10C630007047002070470020704700BF4C0E00205C
:10C640000040044010B485B044B200F00F0005284B
:10C6500065D8421EEFF31083B3FA83F35B090393AB
:10C6600072B6BFF35F8F0021314B19700399002C14
:10C6700014DB304A00F10C0452F824300293029B80
:10C6800043F04F030293029B43F020030293029B6B
:10C6900042F8243000238DF807302EE000F10C031F
:10C6A000244C54F8233013F0100F09D102EB82030D
:10C6B0009C00214B23445B7CC3F38103012BD8DD19
:10C6C00002EB820294001C4B23445A7C42F020026D
:10C6D0005A74012303FA00F0164B186121B30120AC
:10C6E000134B1870BFF35F8F62B619E000BF9DF85F
:10C6F00007300133DBB28DF807309DF80730DBB22D
:10C70000132BF3D9012303FA00F00A4B186169B126
:10C710000120074B1870BFF35F8F62B600E0002066
:10C7200005B05DF8044B70470120F9E70120F7E7F9
:10C73000EB020020004004404C0E002000F00F00EF
:10C7400005286CD830B583B00246441E04EB840340
:10C750009900354B0B44597C6FF34511597400F126
:10C760000C03324951F8233013F0200F59D000F157
:10C770000C0551F825300093009B43F04F030093C4
:10C78000009B23F020030093009B41F8253002F129
:10C790000C03264951F8233013F0200FF7D10D4632
:10C7A0008B6A012181400B43AB62204B9B6A19428B
:10C7B000FBD01E4B9D6A25EA010199620C3053F8AB
:10C7C00020100191019941F04F010191019921F04F
:10C7D00008010191019943F8201002F10C0313495B
:10C7E00051F8233013F0080FF7D104EB84039A00BB
:10C7F0000D4B13445B7C13F0100F01D1012011E0AD
:10C800000949A200101983000B44587C6FF30410EF
:10C8100058741444A300CB589847012002E000202C
:10C820007047012003B030BD4C0E00200040044092
:10C83000F0B583B000F00F04052C00F2A28047B2DF
:10C84000651E04F10C00554E56F8200010F4004F00
:10C8500000F09A8005EB8500514E06EB8000407C8D
:10C8600010F0200F40F0928004F10C004B4E56F86F
:10C87000200010F0200F40F08B80EFF31080B0FA12
:10C8800080F04009009072B6BFF35F8F00264548E4
:10C890000670DDF800E005EB8500414E06EB8000F8
:10C8A000407C10F0100F0AD0BEF1000F72D00122B0
:10C8B0003C4B1A70BFF35F8F62B6002062E005EB5D
:10C8C0008500374E06EB8000467C46F01006467425
:10C8D000BEF1000F05D0012632480670BFF35F8F0E
:10C8E00062B6DFF8BCE005EB850080000EEB0006C9
:10C8F0007260B3600022F260089A4EF8002011B90D
:10C900005BBB012000E00120254AA9004B1902EB86
:10C9100083035B7C60F386130D4402EB85026FF3A7
:10C92000C7135374EFF31083B3FA83F35B090193D6
:10C9300072B6BFF35F8F00221A4B1A70019D01235C
:10C94000A340164A1361002F09DB2DB30120154BBC
:10C950001870BFF35F8F62B614E00020D4E704F1D3
:10C960000C0352F8233013F0110FEED101212046B1
:10C970000D4B98470028E8D0002120460A4B9847E5
:10C98000E3E7002003B0F0BD0020FBE70020F9E75B
:10C990000020F7E70020F5E70120F3E7004004401E
:10C9A0004C0E0020EB02002001B9400070B586B0AB
:10C9B00000F00F04052C00F2C98042B2EFF310839F
:10C9C000B3FA83F35B09059372B6BFF35F8F00215F
:10C9D0005F4B1970059B26460125A5405D494D61B9
:10C9E0002BB101215A4B1970BFF35F8F62B6002A39
:10C9F00080F2948004F10C03564A52F8233013F06D
:10CA0000100F64D0002C49D0032C47D004F10C0146
:10CA100052F821300193019B43F04F030193019B96
:10CA200023F010030193019B42F8213006F10C031F
:10CA3000484A52F8233013F0100FF7D106F10C03D7
:10CA4000444A52F8233013F0100FF7D104F10C01CF
:10CA500052F821300293029B43F04F030293029B52
:10CA600043F010030293029B42F8213000238DF81B
:10CA7000033006E000BF9DF803300133DBB28DF8D0
:10CA800003309DF80330DBB2132BF3D906F10C030E
:10CA9000304A52F8233013F0100FF7D02D4A04F12A
:10CAA0000C0152F821300393039B43F04F0303938F
:10CAB000039B23F010030393039B42F8213006F1FC
:10CAC0000C03244A52F8233013F0100FF7D1214AF7
:10CAD00004F10C0152F821300493049B43F04F03FE
:10CAE0000493049B23F001030493049B42F8213038
:10CAF00006F10C03174A52F8233013F0010FF7D157
:10CB0000621E02EB82029100134B0B445A7C6FF3BE
:10CB100083025A740AE02046104B984706F10C0332
:10CB20000C4A52F8233013F0420FF4D1094A936AA9
:10CB30002B439362074B9B6A1D42FBD0054A936AC5
:10CB400023EA050595622046054B984706B070BD5F
:10CB5000EB020020004004404C0E002045B740008E
:10CB600021B74000064BD3F8142122F44062C3F8E9
:10CB70001421D3F8202142F00102C3F8202170478C
:10CB800000020E400B4619B1096801605B68436002
:10CB90001AB11368036153684361704721F0FE01C5
:10CBA000C905C90D0162704710B51E4B53F82040EE
:10CBB0002268536A13F0805F11D00223C2F820313B
:10CBC00023684FF0FF32DA6100232375236913F0E5
:10CBD000010F26D0636823B32046984710BD13F099
:10CBE000006F13D00223C2F8203123684FF0006297
:10CBF000DA61236913F0020F03D0A3680BB120465A
:10CC0000984723680122C3F8202110BD13F0007F4C
:10CC100007D0236913F0040F03D0E3680BB120465B
:10CC2000984710BDB00E002008B50020014B984772
:10CC300008BD00BFA9CB400008B50120014B9847B3
:10CC400008BD00BFA9CB400070B505460E4614468E
:10CC5000016001230B60214B99422BD00D20204B0A
:10CC60009847204B1D6023781B0203F4FE4373603A
:10CC700063782BBB0022A3780BB142F00402E37867
:10CC80000BB142F0080223790BB142F01002637934
:10CC90001B0203F47063A179090389B20B431343A8
:10CCA000B3652389C3F30E03628943EA0243F36544
:10CCB00000230CE012200A4B98470A4B5D60D2E734
:10CCC0000222D8E705EB8302002151600133022BD9
:10CCD000F8D900202861287570BD00BF000003400E
:10CCE00061D14000B00E002012F0100F12D0C0F839
:10CCF000B01012F0200F07D0C0F8D41012F0400F7F
:10CD000005D0C0F8C0107047C0F8D010F6E7C0F8E2
:10CD1000C4107047C0F8B410704701647047416494
:10CD20007047C06C7047806C7047400900F5001078
:10CD300000F207704002704740090B30704700F066
:10CD40001F00012303FA00F07047000008B500201F
:10CD50000A4B98470A4B98470028FBD0094B984745
:10CD6000094A0A4BDA620A4B98470028FBD0002098
:10CD7000084B9847084B984708BD00BFDDD04000DE
:10CD800001D1400045D14000013FB80500040E40EC
:10CD900051D1400065D2400079D2400010B5A2B018
:10CDA0001848194B98470020184B9847184B98473C
:10CDB0000028FBD0174B9847174A184B9A62184B1C
:10CDC00098470028FBD00020164B9847164B9847F1
:10CDD00016480D4B9847164B1A68164B1344164AC3
:10CDE000934201D922B010BD2023009302AB0F2241
:10CDF0000E211248124CA047BDF848101148124BA2
:10CE00009847EFE7000E2707D1D54000DDD040005E
:10CE100001D1400029D14000013FB70B00040E4072
:10CE200035D1400089D04000DDD440000000DC0551
:10CE3000EC020020C0D3BDF980C3C901000A0E4036
:10CE40001100002010140E40A9D2400070B50D460C
:10CE50001446064658B14FF0FF360AE0064B1868F4
:10CE6000064B1B682946984701350136013C002CCA
:10CE7000F4DC304670BD00BFF81F0020F01F00201A
:10CE800070B5013802280FD8144600258CB10A4B22
:10CE900018684E1C094B1B6809789847002806DB68
:10CEA0000135013C3146F1E74FF0FF3501E04FF02D
:10CEB000FF35284670BD00BFF81F0020F41F00207A
:10CEC000A1F10E03012B02D84FF0FF30704710B5CF
:10CED00082B0EFF31083B3FA83F35B09019372B668
:10CEE000BFF35F8F00240B4B1C70019C120222F0D9
:10CEF0007F4222F0FF02C9B2114341F0B441064B18
:10CF000098472CB10122034B1A70BFF35F8F62B6B2
:10CF100002B010BDEB020020790000204C4B1B78C2
:10CF2000FF2B31D000B583B0EFF31083B3FA83F356
:10CF30005B09019372B6BFF35F8F0022454B1A70F5
:10CF40000199434A13780133137029B10122414BEF
:10CF50001A70BFF35F8F62B63F4A904215D03F4AC6
:10CF6000904220D03E4A90422BD03E4A904236D04A
:10CF70003D4A904241D03D4A90424CD03C4A90427A
:10CF800057D003B05DF804FBFEE71620394B9847F5
:10CF90000720394B984700210720384B9847072036
:10CFA000374B9847EDE71520324B98470720324B17
:10CFB000984700210720314B98470720304B98476E
:10CFC000DFE714202B4B984707202B4B9847002175
:10CFD00007202A4B98470720294B9847D1E7132071
:10CFE000244B98470620244B984700210620234BCA
:10CFF00098470620224B9847C3E70E201D4B9847C1
:10D0000006201D4B9847002106201C4B9847062000
:10D010001B4B9847B5E70920164B98470620164B3F
:10D02000984700210620154B98470620144B984737
:10D03000A7E708200F4B984706200F4B9847002181
:10D0400006200E4B984706200D4B984799E700BFE6
:10D05000E81F0020EB020020000004400080004098
:10D0600000C001400080014000400240000002403A
:10D0700000C0004061D1400051D2400009D24000C0
:10D080003DD2400001607047134A136B23F07003D8
:10D09000184310634FF400630F4A926E12F0080FAA
:10D0A00002D1A3B1013BF7E70B4A136B23F0030353
:10D0B00043F0020313634FF40063074A926E12F0C9
:10D0C000080F02D12BB1013BF7E700207047012088
:10D0D00070470120704700BF00040E40012803D0B4
:10D0E000054A064B1A607047044A936843F025438B
:10D0F00043F480139360F3E7080000A510140E407A
:10D10000074B5B6913F0800F06D0064B9B6E13F044
:10D11000800F03D100207047002070470120704726
:10D1200010140E4000040E400022014B9A6270471A
:10D1300000040E40024B986E00F00200704700BFE2
:10D1400000040E400022014BDA62704700040E40DA
:10D15000024B986E00F00400704700BF00040E40C0
:10D1600032281ED81F280CD8114B9A6901238340FE
:10D17000934318D0012303FA00F00D4B18610020EF
:10D18000704720380A4BD3F808210123834093438A
:10D190000BD0012303FA00F0054BC3F80001002077
:10D1A000704701207047002070470020704700BF83
:10D1B00000040E40322822D81F280ED8114B9A693D
:10D1C00001238340934301D000207047012303FAD9
:10D1D00000F00C4B5861002070472038094BD3F801
:10D1E000082101238340934301D00020704701238D
:10D1F00003FA00F0034BC3F804010020704701203C
:10D20000704700BF00040E4041F0040100F110021D
:10D21000094B43F822104FF40062074B996E4FF40C
:10D2200080738340194202D11AB1013AF5E7002018
:10D2300070470120704700BF00040E404FF4807318
:10D2400003FA00F0014B1860704700BF00040E4065
:10D250004FF4807303FA00F0014B5860704700BF31
:10D2600000040E40000200F4706040F00100014B29
:10D270009863704700040E408022014B1A6070478B
:10D2800000040E40C0F31200024B1A6F10431867DF
:10D29000704700BF00040E40024B187880F0010078
:10D2A000704700BFB80E0020C36923F4F053490251
:10D2B00001F4F051194341F0B44141F48071C1616E
:10D2C000704730B4B2EB011F17D3102401FB04F1F7
:10D2D0004B0803EBC202B2FBF1F2D3085D1E4FF61E
:10D2E000FE718D4210D8082C09D0120402F4E022FD
:10D2F0001A430262002030BC70470824E6E7416808
:10D3000041F400214160F0E70120F4E7402303608D
:10D3100070478823036070471023036070472423FD
:10D32000036070474FF48073036070474FF400232D
:10D3300003607047436913F0020F04D0C1F3080182
:10D34000C1610020704701207047436913F0020F4C
:10D35000FBD0C1F30801C16100207047436913F09D
:10D36000010F05D08369C3F308030B6000207047E9
:10D3700001207047014BC0F8E4307047004153551D
:10D3800010B50446094B9847002363606362A362AB
:10D390002046074B98472046064B98472046064BA9
:10D3A00098472046054B984710BD00BF75D34000F5
:10D3B00013D340001FD3400025D340002DD340009D
:10D3C00070B505460C461646104B98470022104B88
:10D3D0001A60B4B13246216828460E4B984702467F
:10D3E00088B96368A1680B4321690B43E1680B436B
:10D3F0000749086803430B6069680B436B6010467C
:10D4000070BD0122FBE70122F9E700BF81D3400094
:10D41000BC0E0020C3D24000FEE7000000B583B080
:10D42000234B244A9A4209D0214B224A03E0116837
:10D4300019600433043220498B42F8D31F4B02E0B9
:10D4400000221A6004331E4A9342F9D31D4A22F087
:10D450007F011D4B9960EFF31083B3FA83F35B09EF
:10D46000019372B6BFF35F8F0021184B19700198BA
:10D4700017490B6843F470030B60BFF34F8FBFF382
:10D480006F8F28B10121114B1970BFF35F8F62B606
:10D4900002F16042B2F5203F04D20B4A936843F098
:10D4A000005393600B4B98470B4B9847FEE700BF28
:10D4B00010000020A4434100A80C0020A80C00206C
:10D4C0009C2000200040400000ED00E0EB02002026
:10D4D00088ED00E0C506410055F64000344B1B6B5B
:10D4E00003F00303012B20D083B1022B39D0304B42
:10D4F0001B6B03F07003702B51D02D4B1A6BC2F3D2
:10D5000002122C490B68D3400B6070472A4B5B69B1
:10D5100013F0800F04D04FF40042264B1A60E6E768
:10D520004FF4FA42234B1A60E1E7214B1B6A13F0D8
:10D53000807F03D0214A1F4B1A60D8E7204A1D4B39
:10D540001A601B4B1B6A03F07003102B05D0202BB5
:10D55000CDD11C4A174B1A60C9E71B4A154B1A60FC
:10D56000C5E7154B5B6913F0800F13D04FF40042F1
:10D57000104B1A600E4B1B6B03F00303022BB6D14A
:10D580000B4B9A6AC2F30C420A490B6802FB033345
:10D590000B60ACE74FF4FA42064B1A60EAE7054A23
:10D5A00013680A49A1FB03135B081360704700BFAF
:10D5B00000040E40EC02002010140E40001BB700C7
:10D5C00000127A0000366E010024F400ABAAAAAA69
:10D5D000144B98420FD9144B984211D9134B9842CF
:10D5E00012D9134B984213D9124B984214D9124AAC
:10D5F000124B1A6070474FF08062104B1A607047F0
:10D600000F4A0E4B1A6070470E4A0C4B1A60704757
:10D610000D4A0A4B1A6070474FF00422074B1A60FC
:10D62000704700BFFF2C3101FF596202FF86930350
:10D63000FFB3C404FFE0F50500050004000A0E4036
:10D640000001000400020004000300040A4B1B68F0
:10D6500053B1094B1B681A180849914208DB104660
:10D66000054A106018467047054A034B1A60F0E7F8
:10D670004FF0FF30704700BFC00E0020FC7F02203B
:10D68000A05000204FF0FF3070474FF400534B6024
:10D6900000207047012070470020704700F1080308
:10D6A00043604FF0FF328260C36003610023036078
:10D6B000704700230361704743684B609A688A6033
:10D6C0009A6851609960086103680133036070478C
:10D6D00030B40D68B5F1FF3F02D000F1080202E05E
:10D6E000026904E01A4653681C68A542FAD25368DE
:10D6F0004B6099608A605160086103680133036080
:10D7000030BC7047036942688168916082684168F3
:10D7100051605A68904206D0002202611A68013AAC
:10D720001A601868704782685A60F5E782B0002373
:10D7300001934FF0500383F31188BFF36F8FBFF352
:10D740004F8F019B002BFCD002B070470848006847
:10D75000006880F308884FF0000080F3148862B6F8
:10D7600061B6BFF34F8FBFF36F8F00DF00BF0000C4
:10D7700008ED00E0DFF80C00016841F47001016081
:10D780007047000088ED00E04FF0807340F8043CE3
:10D7900021F0010140F8081C054B40F80C3C40F812
:10D7A000202C6FF0020340F8243C4438704700BF3F
:10D7B0002DD7400000000000000000000000000025
:10D7C000074B19680868B0E8F04F80F30988BFF389
:10D7D0006F8F4FF0000080F311887047AFF3008027
:10D7E000C40E00204FF0500383F31188BFF36F8FF6
:10D7F000BFF34F8F024A136801331360704700BFB5
:10D80000F0020020034A1368013B13600BB983F355
:10D8100011887047F00200200000000000000000A6
:10D82000EFF30980BFF36F8F154B1A681EF0100FCE
:10D8300008BF20ED108A20E9F04F10602DE90900A3
:10D840004FF0500080F31188BFF34F8FBFF36F8FFD
:10D8500000F072FF4FF0000080F3118809BC1968D6
:10D860000868B0E8F04F1EF0100F08BFB0EC108A47
:10D8700080F30988BFF36F8F704700BFAFF300805C
:10D88000C40E002008B54FF0500383F31188BFF396
:10D890006F8FBFF34F8F054B984718B14FF08052F1
:10D8A000034B1A60002383F3118808BDB5E44000E0
:10D8B00004ED00E0054B00221A6005490A600549A5
:10D8C000054A116007221A60704700BF10E000E0AF
:10D8D00018E000E0FF7F010014E000E010B50E4BFF
:10D8E0001A6842F470021A601A6842F070421A60B4
:10D8F0000A4B984700240A4B1C600A4B98470A4A77
:10D90000136843F040431360084B9847084B98470F
:10D91000084B9847204610BD20ED00E0B5D84000E8
:10D92000F002002075D7400034EF00E04DD74000F2
:10D9300039E740002DD7400010B50446044B984706
:10D940002046044B98470446034B9847204610BD99
:10D9500099E440003D074100A9E5400048B110B5F9
:10D960000446044B98472046034B9847034B98477F
:10D9700010BD704799E440004D074100A9E5400003
:10D98000436A23B1036B1868C0F10500704700209B
:10D990007047000010B50446064B9847A26BE36B36
:10D9A0009A4204D00024044B9847204610BD01241D
:10D9B000F9E700BFE5D7400005D8400010B50446A0
:10D9C000054B9847A36B23B10024044B984720468E
:10D9D00010BD0124F9E700BFE5D7400005D840009D
:10D9E00070B504461646856B026C5AB903681BB1C4
:10D9F00000200135A56370BD4068174B9847002390
:10DA00006360F6E76EB98068144B9847226CA36890
:10DA10001344A3606268934219D32368A360002073
:10DA2000E7E7C0680D4B9847226C5242E368134405
:10DA3000E36021688B4202D263681A44E260022EDE
:10DA400001D00020D5E725B1013D0020D1E700201D
:10DA5000CFE70020CDE700BF2DEA4000C10D410017
:10DA6000026C72B110B5C3681344C3604468A3422A
:10DA700001D30368C3600C46C1682046014B984738
:10DA800010BD7047C10D410038B505461A4B984787
:10DA900095F8454064B201E0013C64B2002C0ADD17
:10DAA0006B6A43B105F12400144B98470028F3D06A
:10DAB000134B9847F0E7FF2385F84530114B984703
:10DAC0000D4B984795F8444064B201E0013C64B2C4
:10DAD000002C0ADD2B6943B105F11000074B984774
:10DAE0000028F3D0064B9847F0E7FF2385F8443031
:10DAF000044B984738BD00BFE5D740003DE84000E3
:10DB000039E9400005D8400038B504460D46144BAD
:10DB100098472168E26B236C03FB021060600020D1
:10DB2000A063A160013A02FB0313E360FF2384F8C2
:10DB3000443084F8453055B923691BB9094B9847DF
:10DB4000012038BD04F11000074B9847F6E704F1B7
:10DB50001000064DA84704F12400A847EEE700BFD7
:10DB6000E5D7400005D840003DE840009DD6400084
:10DB700038B51D46049C0B4649B12260E06323641E
:10DB800001212046034B984784F84C5038BD24604F
:10DB9000F4E700BF09DB4000F0B583B00546174647
:10DBA0000E4689B100FB01F05030084B98470446FF
:10DBB00038B100903B4600F1500231462846044DF2
:10DBC000A847204603B0F0BD0020EDE739D940005A
:10DBD00071DB4000F0B585B004460F4601921E4649
:10DBE000002526E0324639462046354B9847636A81
:10DBF00023B9344B9847012005B0F0BD04F124004F
:10DC0000314B9847F5E72F4B98470020F4E702A8DF
:10DC10002E4B9847012519E0002384F8443021E079
:10DC2000002384F8453023E02046294B9847294BB0
:10DC30009847294B9847A26BE36B9A42D2D3022EA6
:10DC4000D0D0019B002BDED0002DE0D01D4B98479B
:10DC5000224B9847204B984794F844305BB2B3F17D
:10DC6000FF3FD9D094F845305BB2B3F1FF3FD7D036
:10DC7000144B984701A902A8194B9847C8B92046E8
:10DC8000184B98470028CFD0019904F11000164B8B
:10DC9000984720460E4B98470E4B98470028C8D10E
:10DCA0004FF08052114B1A60BFF34F8FBFF36F8F4D
:10DCB000BFE72046064B9847064B984700209BE756
:10DCC000E1D9400005D840003DE84000BDE84000F3
:10DCD00089DA4000A9E54000E5D7400099E440001A
:10DCE000D5E8400095D94000EDE7400004ED00E0A4
:10DCF00048B110B5002141600160C1600B460A4681
:10DD0000014CA04710BD7047D5DB400010B502465E
:10DD100000210120034B98470446034B98472046B7
:10DD200010BD00BF99DB4000F1DC4000F8B5EFF317
:10DD300011864FF0500484F31188BFF36F8FBFF347
:10DD40004F8F856BC46BA54205D3022B03D00020F7
:10DD500086F31188F8BD1746054690F8454064B231
:10DD60001A460E4B9847B4F1FF3F05D0013464B218
:10DD700085F845400120EBE76B6A0BB90120E7E726
:10DD800005F12400064B984718B127B101203860EF
:10DD9000DEE70120DCE70120DAE700BFE1D940003F
:10DDA0003DE84000F0B585B004460F4601920026DC
:10DDB00032E039462046384B9847013DA563236938
:10DDC00023B9364B9847012005B0F0BD04F110008F
:10DDD000334B9847F5E7314B98470020F4E702A80A
:10DDE000304B9847012621E0002384F8443029E095
:10DDF000002384F845302BE020462B4B98472B4BD3
:10DE0000984709E02046284B9847284B98472046DA
:10DE1000274B984700283DD1264B9847A56B002DEE
:10DE2000C7D1019B002BD6D0002ED8D01B4B9847D2
:10DE3000214B98471F4B984794F844305BB2B3F19D
:10DE4000FF3FD1D094F845305BB2B3F1FF3FCFD064
:10DE5000124B984701A902A8184B98470028D1D126
:10DE60002046134B98470028C6D0019904F124009E
:10DE7000134B984720460C4B98470C4B984700286B
:10DE8000CAD14FF080520F4B1A60BFF34F8FBFF3D0
:10DE90006F8FC1E7002097E761DA400005D84000A6
:10DEA0003DE84000BDE8400089DA4000A9E54000B7
:10DEB000BDD94000E5D7400099E44000D5E84000D6
:10DEC000EDE7400004ED00E070B584B00446019138
:10DED000002635463EE0013BA36323683BB123693E
:10DEE0004BB9444B98470126304604B070BD424BB5
:10DEF00098476060F3E704F11000404B9847F0E763
:10DF00003C4B98470026EFE702A83D4B9847012578
:10DF10002AE0002384F8443032E0002384F84530BE
:10DF200034E0384B98476068374B98470646314B8A
:10DF300098473BE02046354B9847354B984709E0DA
:10DF40002046324B9847324B98472046314B9847F2
:10DF5000002840D12B4B9847A36B002BBBD1019BD2
:10DF6000002BCDD0002DCFD0224B98472A4B98477D
:10DF7000244B984794F844305BB2B3F1FF3FC8D0CC
:10DF800094F845305BB2B3F1FF3FC6D0194B9847C8
:10DF900001A902A8214B98470028D1D120461D4B4A
:10DFA00098470028C6D02368002BBAD0019904F105
:10DFB00024001B4B98472046144B9847144B984716
:10DFC0000028C7D14FF08052164B1A60BFF34F8F15
:10DFD000BFF36F8FBEE7002E86D00A4B98472046CE
:10DFE000114B984701466068104B9847014B984782
:10DFF000002679E705D8400055EB40003DE8400099
:10E00000BDE84000E5D7400065E9400089DA4000FE
:10E01000A9E54000BDD9400099E44000D5E84000A2
:10E02000EDE7400004ED00E081D94000B5EA400092
:10E030000023092B0CD8074A52F833200AB10133C8
:10E04000F7E7044A42F8331002EBC3035860704705
:10E05000704700BFFC1F002070B504460D461646F1
:10E06000124B984794F844305BB2B3F1FF3F0DD0A8
:10E0700094F845305BB2B3F1FF3F0BD00C4B98479F
:10E08000A36B5BB120460B4B984770BD002384F80F
:10E090004430EDE7002384F84530EFE73246294667
:10E0A00004F12400044B9847ECE700BFE5D740009B
:10E0B00005D8400089DA400011E84000F0B5036857
:10E0C0004BB343685B68436000F10807BB4204D070
:10E0D0004368D3F80CE0002609E05B684360F7E78B
:10E0E0005B68436008E02E46B6B9AE4514D043687D
:10E0F0005B6843609F42F3D04368DD6800230F2BC9
:10E10000F2D8EA1892F83420CC5CA242ECD1002A72
:10E11000E9D00133F3E700263046F0BD0A4B1B6817
:10E120001B684BB901234BB9074B1B68DB68DB68E5
:10E130005A68064B1A6070470023F4E74FF0FF322D
:10E14000024B1A60704700BFC80E0020740F0020F9
:10E150002DE9F84F81460D4617469A460A9EDDF88E
:10E160002C800C9C9200A521206B1D4B9847236BA3
:10E1700007F18042013A03EB820727F007070023EB
:10E180000F2B07D8E95CE21882F83410EA5C0AB178
:10E190000133F5E7002384F84330042E00D9042628
:10E1A000E662E66400252565201DDFF83CB0D8470F
:10E1B00004F11800D8472461C6F10506A66164621F
:10E1C000656584F85850524649463846054B98478D
:10E1D0002060B8F1000F01D0C8F80040BDE8F88F0A
:10E1E000BD0F410089D74000B3D6400070B5002470
:10E1F00007E004EB840293000B4818440B4B98474C
:10E200000134042CF5D90A4E3046084CA047094D7C
:10E210002846A0470848A0470848A047084B1E606A
:10E22000084B1D6070BD00BFD00E00209DD6400081
:10E23000480F00205C0F00207C0F0020940F00206E
:10E24000C80E0020CC0E002010B504461C4B984789
:10E250001C4A1368013313601B4B1B68002B26D02C
:10E260001A4B1B683BB9184B1B68DA6AE36A9A427F
:10E2700001D8154B1C60164A1368013313606364A0
:10E28000E36A01229A401349086802430A6003EBDB
:10E2900083039A00211D10481044104B9847104BDF
:10E2A00098470A4B1B680BB1074B1B6810BD064B08
:10E2B0001C601368012BDED10A4B9847DBE700BFD7
:10E2C000E5D74000340F0020C40E0020900F00203E
:10E2D000400F0020440F0020D00E0020B9D640008F
:10E2E00005D84000EDE1400070B504460E461D4BD8
:10E2F0001D681D4B186804301C4B984750B91A4BC9
:10E300001B68DA6A012303FA02F219490B6823EA4F
:10E3100002030B60B4F1FF3F13D02C44124B1B6877
:10E320005C60A54216D8134B18680F4B196804316E
:10E33000114B9847114B1B689C4201D20F4B1C603C
:10E3400070BD002EE9D0084B196804310C480D4B04
:10E35000984770BD0C4B1868034B19680431064B85
:10E36000984770BDA80F0020C40E002005D74000BC
:10E37000440F0020C80E0020D1D64000740F0020AA
:10E38000940F0020B9D64000CC0E002008B54FF005
:10E390008052044B1A60BFF34F8FBFF36F8F024B55
:10E3A0009847F4E704ED00E051F640002DE9F04312
:10E3B00085B006460F46154698469000144B984780
:10E3C00000B381465C20124B98470446B0B1C0F8B8
:10E3D0003090CCB10023039302940D9B01930C9BCE
:10E3E000009343462A46394630460A4DA847204600
:10E3F000094B9847012005B0BDE8F0834846074B1C
:10E400009847E6E70024E4E74FF0FF30F3E700BF6A
:10E4100039D9400051E1400049E240005DD9400057
:10E4200010B582B0134B019300230093462212498A
:10E430001248134CA047012803D0012804D002B091
:10E4400010BD104B9847F8E74FF0500383F3118845
:10E45000BFF36F8FBFF34F8F4FF0FF320A4B1A603D
:10E4600001220A4B1A600022094B1A60094B984797
:10E47000E5E700BF700F0020204141008DE3400020
:10E48000ADE34000E9EF4000740F0020900F002042
:10E49000A80F0020DDD84000024A13680133136042
:10E4A000704700BF3C0F0020014B1868704700BF49
:10E4B000A80F002070B52F4B1B68002B52D12E4B9C
:10E4C0001E6801361E604EB12C4B1B689E422FD237
:10E4D0002B4B1B68002B42D0002070BD294A1168CD
:10E4E000294B186810601960284A136801331360BB
:10E4F000274B9847E8E7012320E04FF0FF321F4BFE
:10E500001A60E5E71D4A1360E2E704F11800214BA9
:10E510009847E36A01229A401F49086802430A604B
:10E5200003EB83039A0029461C4810441C4B984770
:10E53000144B1B681B68002BDDD00023002BDCD1A3
:10E54000104B1B68DB68DC6863689E42DAD3251DCC
:10E550002846104B9847A36A002BD6D1D9E7114B18
:10E560009847B9E7064A1368013313600D4B984783
:10E57000B2E700BF3C0F0020A80F0020740F00205E
:10E58000380F0020C80E0020CC0E0020780F00208D
:10E590001DE1400005D74000440F0020D00E0020B0
:10E5A000B9D6400053F6400070B5274B9847274B2B
:10E5B0001A68013A1A601B68002B32D1244B1B6881
:10E5C000002B2ED00024234B1B6813B3214BDB6898
:10E5D000DC6804F11800204EB047251D2846B047DE
:10E5E000E36A01229A401D49086802430A6003EB6E
:10E5F00083039A0029461A4810441A4B9847E26A46
:10E60000194B1B68DB6A9A42DDD30122174B1A6053
:10E61000D9E70CB1164B9847164B1C683CB9134B05
:10E620001B68154B9847002070BD013C07D0134B69
:10E6300098470028F9D001220C4B1A60F5E7002218
:10E640000C4B1A60EBE700BFE5D740003C0F002001
:10E65000340F00207C0F002005D74000440F00201D
:10E66000D00E0020B9D64000C40E0020AC0F002010
:10E670001DE14000380F002005D84000B5E44000FF
:10E6800010B550B9002038B94FF08052084B1A60CD
:10E69000BFF34F8FBFF36F8F10BD0446054B9847F4
:10E6A00000212046044B9847044B9847EBE700BFF6
:10E6B00004ED00E099E44000E9E24000A9E54000F3
:10E6C00070B50646154B98470524013C04EB8402BF
:10E6D0009300314612481844124B9847054608B932
:10E6E000002CF2D12DB15DB18DB10F4B984728466A
:10E6F00070BD0E4B186831460A4B98470546F2E745
:10E700000B4B18683146074B98470546ECE73146F6
:10E710000848044B98470546E7E700BF99E44000E6
:10E72000D00E0020BDE04000A9E54000C80E00204A
:10E73000CC0E0020940F0020264B1B68002B2FD1FD
:10E7400010B50022244B1A60244B1B681B6B1A68FF
:10E75000B2F1A53F28D0214B186819683431204BFD
:10E760009847204B1B68B3FA83F3DBB2C3F11F0356
:10E770001D489A00D418A10001444C6864684C609C
:10E780001A4491000831084484421AD003EB8303F1
:10E790009A00154B13445B68DA68104B1A6010BD81
:10E7A00001220D4B1A6070475A68B2F1A53FD2D1D1
:10E7B0009A68B2F1A53FCED1DB68B3F1A53FCAD1CB
:10E7C000CFE7606803EB83029100074A0A44506078
:10E7D000DCE700BF3C0F0020AC0F0020C40E00207F
:10E7E00039F64000440F0020D00E002010B50C4632
:10E7F000044B19681831044B984701212046034BFC
:10E80000984710BDC40E0020D1D64000E9E2400078
:10E8100038B50D461446064B19681831054B984714
:10E820000CB14FF0FF3521462846034B984738BDC1
:10E83000C40E0020B9D64000E9E2400038B5C368F4
:10E84000DC6804F118052846144B9847144B1B68E4
:10E85000E3B9251D2846114B9847E36A01229A40E7
:10E860001049086802430A6003EB83039A002946B3
:10E870000D4810440D4B9847E26A0D4B1B68DB6A4C
:10E880009A4208D901200B4B186038BD29460A4826
:10E89000064B9847F0E7002038BD00BF05D7400081
:10E8A0003C0F0020440F0020D00E0020B9D64000BD
:10E8B000C40E0020AC0F00207C0F0020034B1B680F
:10E8C0000360034B1B684360704700BF780F002054
:10E8D000A80F0020F8B504460D46124B9847124B7E
:10E8E00019686268881A2B68B3F1FF3F16D0276851
:10E8F0000E4E3668B74201D0914211D2984206D3EB
:10E9000000232B6001240A4B98472046F8BD1B1AB0
:10E910002B602046074B98470024F4E70024F2E7D9
:10E920000124F0E7E5D74000A80F0020780F002071
:10E9300005D84000BDE840000122014B1A60704735
:10E94000AC0F0020054B1B6823B1054B1B681BB99E
:10E95000022070470120704700207047900F002070
:10E960003C0F0020002854D038B50446C26A2A491A
:10E970000968C96A8A4242D28169002905DB2649B1
:10E980000968C96AC1F105018161606902EB82020F
:10E990009100224A0A44904207D000223AB91E4A06
:10E9A0001268D26AE262012038BD0122F6E7251D15
:10E9B00028461B4B984768B9E36A03EB83018A003A
:10E9C00016498A5832B901229A4016490B6823EA3F
:10E9D00002030B60104B1B68DB6AE362012404FA3C
:10E9E00003F21049086802430A6003EB83039A00AC
:10E9F00029460A4810440C4B9847204638BDC26C43
:10EA0000054B1B68DB6A9A4201D2012038BD002009
:10EA100038BD0020704700BFC40E0020D00E00207B
:10EA200005D74000440F0020B9D64000002834D05C
:10EA300038B50446026D013A0265C06AE16C88424D
:10EA40002DD00AB1002038BD251D2846154B98470A
:10EA500068B9E36A03EB83018A0013498A5832B923
:10EA600001229A4011490B6823EA02030B60E36C10
:10EA7000E362C3F10502A261012404FA03F20B4927
:10EA8000086802430A6003EB83039A00294606489C
:10EA90001044074B9847204638BD0020704700209F
:10EAA00038BD00BF05D74000D00E0020440F002025
:10EAB000B9D64000002843D038B50446C26C8A421B
:10EAC00000D20A46E16A8A4202D0206D012800D0B5
:10EAD00038BDE262A069002802DBC2F10502A26132
:10EAE000636901EB81018800164A0244934225D0F4
:10EAF0000022002AECD0251D2846134B984768B900
:10EB0000E36A03EB83018A000E498A5832B9012275
:10EB10009A400E490B6823EA02030B60E36A012264
:10EB20009A400A49086802430A6003EB83039A008B
:10EB3000294604481044064B9847C9E70122D8E704
:10EB4000704700BFD00E002005D74000440F0020C2
:10EB5000B9D64000054B1B6823B1044B1A68136DEE
:10EB600001331365014B1868704700BFC40E0020C5
:10EB700038B505460C461A4B98471A4B1B685B6D17
:10EB80002BB9184B1B68012283F85820ACB9164BDF
:10EB90009847134B9847134B1B685C6D24B1CDB954
:10EBA000104B1B68621E5A650E4B1B68002283F8CF
:10EBB00058200D4B9847204638BD114620460B4B38
:10EBC00098474FF080520A4B1A60BFF34F8FBFF344
:10EBD0006F8FDCE7034B1B6800225A65E4E700BF38
:10EBE000E5D74000C40E002005D84000E9E240000F
:10EBF00004ED00E0F8B507460D4614461E46214BCD
:10EC00009847214B1B6893F85830DBB2022B0AD08F
:10EC10001D4B1A68506D20EA070050651B680122E1
:10EC200083F85820CEB9194B9847164B98471CB11A
:10EC3000154B1B685B6D2360134B1B6893F85830B2
:10EC4000DBB2022B16D000240F4B1B68002283F886
:10EC500058200E4B98472046F8BD114630460C4BC5
:10EC600098474FF080520B4B1A60BFF34F8FBFF3A2
:10EC70006F8FD8E7044B1A68536D23EA0505556575
:10EC80000124E1E7E5D74000C40E002005D840008C
:10EC9000E9E2400004ED00E0F8B504460F461546F1
:10ECA0001E46214B98470EB1636D336094F858307F
:10ECB000DBB2022284F858206A1E032A1AD8DFE841
:10ECC00002F0020C1114626D174367650125012BD8
:10ECD00014D0164B98472846F8BD626D0132626524
:10ECE0000125F4E767650125F1E7022B04D067658C
:10ECF0000125ECE70125EAE70025E8E7261D304677
:10ED00000B4B9847E36A01229A400A49086802437C
:10ED10000A6003EB83039A00314607481044074B0F
:10ED20009847074B1B68D4E7E5D7400005D840005B
:10ED300005D74000440F0020D00E0020B9D6400077
:10ED4000C40E0020F8B5EFF311854FF0500484F3A2
:10ED50001188BFF36F8FBFF34F8F0BB1446D1C60F1
:10ED600090F85830DBB2022480F85840013A032A68
:10ED70001AD8DFE802F0020C1114426D114341650C
:10ED80000126012B14D085F311883046F8BD426D61
:10ED9000013242650126F4E741650126F1E7022BC5
:10EDA00004D041650126ECE70126EAE70026E8E702
:10EDB0000446164B1B68F3B9071D3846144B984799
:10EDC000E36A01229A401349086802430A6003EB90
:10EDD00083039A00394610481044104B9847E26A62
:10EDE0000F4B1B68DB6A9A42CDD9069B4BB10123BE
:10EDF000069A1360C7E700F118010A48074B9847C5
:10EE0000EDE70122084B1A60BDE700BF3C0F002070
:10EE100005D74000440F0020D00E0020B9D6400096
:10EE2000C40E00207C0F0020AC0F0020F8B5EFF3DB
:10EE300011854FF0500383F31188BFF36F8FBFF339
:10EE40004F8F90F85830DBB2022280F85820426D84
:10EE500001324265012B02D085F31188F8BD0E46C0
:10EE60000446154B1B68E3B9071D3846134B9847FA
:10EE7000E36A01229A401249086802430A6003EBE0
:10EE800083039A0039460F4810440F4B9847E26AB3
:10EE90000E4B1B68DB6A9A42DED946B10123336010
:10EEA000DAE700F118010A48074B9847EFE701221B
:10EEB000084B1A60D0E700BF3C0F002005D7400088
:10EEC000440F0020D00E0020B9D64000C40E002010
:10EED0007C0F0020AC0F0020064B1A681368B3FAB1
:10EEE00083F35B09036013B9D36818687047002087
:10EEF000704700BFB00F002008B54160006191422B
:10EF00000CD8D21A83699A4201D3012008BD011D91
:10EF1000094B1868094B9847002008BD9A4201D256
:10EF2000994206D2011D064B1868044B98470020F1
:10EF300008BD012008BD00BFB40F0020D1D640009D
:10EF4000B00F002070B5104B9847104B1B6813B1E1
:10EF50000F4B984770BD0F4D28460F4EB0470F4CD2
:10EF60002046B0470E4B1D600E4B1C6000220C214A
:10EF70000A200D4B9847054B18600028E8D00B4934
:10EF80000B4B9847E4E700BFE5D74000E40F0020B3
:10EF900005D84000B80F00209DD64000CC0F0020BF
:10EFA000B00F0020B40F002099DB40002841410041
:10EFB00031E040002DE9F041079C7CB198461546B0
:10EFC0000E460746064B98472760A661E561C4F8E0
:10EFD0002080069B6362201D024B9847BDE8F081AC
:10EFE00045EF4000B3D6400010B582B0094B9847BA
:10EFF000094B1B685BB1094B01930323009300236A
:10F00000462207490748084CA04702B010BD00201F
:10F01000FBE700BF45EF4000E40F0020E80F0020B1
:10F020003041410021F34000ADE340002DE9F041C3
:10F0300082B005460E46174698462C20084B984746
:10F04000044640B10190089B009343463A4631463E
:10F050002846044DA847204602B0BDE8F08100BF15
:10F0600039D94000B5EF400030B585B0134C256864
:10F070000DB31C46019102920390052913DC104B3D
:10F080009847022807D000231A4601A90B480068B8
:10F090000C4CA0470DE00023089A01A9074800681E
:10F0A000084CA04705E00023224601A92846064C4B
:10F0B000A04705B030BD0020FBE700BFE40F0020F3
:10F0C00045E94000D5DB40002DDD400070B582B041
:10F0D000154B1B681A6802B3DB681E68DC68251DC7
:10F0E0002846124B9847636A20469847E369012BEC
:10F0F000EED1A36933449E4207D26360246129465E
:10F10000094B18680A4B9847E2E7002100910B462B
:10F1100032462046074CA047DAE7074A1068024902
:10F120000860136002B070BDB00F002005D740002A
:10F13000D1D6400069F04000B40F002038B5054634
:10F14000084B98470446084B1B68984205D3002398
:10F150002B60054B1C60204638BD044B98470123AB
:10F160002B60F6E7A9E44000E00F0020CDF040005E
:10F1700070B582B005460E460F4B1B68DB68DC6835
:10F18000201D0E4B9847E369012B04D0636A20468B
:10F19000984702B070BDA1692B46324629442046EB
:10F1A000074EB0470028F1D0002100910B462A46B7
:10F1B0002046044DA847E9E7B00F002005D74000DE
:10F1C000F9EE400069F0400070B582B006460C468A
:10F1D000174B984701A8174B9847019B23BB05463F
:10F1E0000CB9B04219D22CB1134B1B681C68B4FA8D
:10F1F00084F464092246711B104B1868104B984721
:10F20000104B984738B94FF080520F4B1A60BFF33C
:10F210004F8FBFF36F8F02B070BD0A4B98472946DE
:10F2200030460A4B9847F6E7064B9847F3E700BF8E
:10F2300099E440003DF14000B40F0020E40F0020AD
:10F2400059E04000A9E5400004ED00E071F1400004
:10F2500030B587B0002203A92A4B18682A4B98477B
:10F2600000284CD0039B002BF4DB059C636913B191
:10F27000201D264B984702A8254B9847039B092B36
:10F28000E8D801A252F823F0B1F24000B1F24000F8
:10F29000B1F2400055F24000E5F24000F7F24000C4
:10F2A000B1F24000B1F2400055F24000E5F24000FA
:10F2B0000499A5690B46024629442046154DA847E6
:10F2C0000028C7D0636A20469847E369012BC1D163
:10F2D000A269002100910B460498024420460E4C7E
:10F2E000A047B7E70499A1610346024601442046BE
:10F2F000084CA047AEE72046084B9847AAE707B05E
:10F3000030BD00BFE40F0020A5DD400005D7400060
:10F310003DF14000F9EE400069F040005DD9400049
:10F3200000B583B001A8044B98470199034B984757
:10F33000034B9847F6E700BFD9EE4000C9F1400003
:10F3400051F24000064BDB6BC3F30023054A1370F8
:10F35000054BDB6BC3F34033044A1370704700BFA7
:10F3600000100E40EC0F0020000E0E40ED0F0020AC
:10F3700008B5054BDB6B13F4004F02D1034B9847E4
:10F3800008BD034B984708BD000E0E40814C40005D
:10F39000A54C400030B583B004460D4600230193D0
:10F3A0002E4B984213D02E4B9C421AD02D4B9C4290
:10F3B00021D02D4B9C4228D02C4B9C422FD02C4B43
:10F3C0009C4236D02B4B9C423DD003B030BD01A9AE
:10F3D0002046294B98470028F9D19DF804302B701E
:10F3E000E1E701A92046244B98470028F9D19DF870
:10F3F00004302B70DAE701A920461F4B98470028FC
:10F40000F9D19DF804302B70D3E701A920461A4B9F
:10F4100098470028F9D19DF804302B70CCE701A95A
:10F420002046154B98470028F9D19DF804302B70E1
:10F43000C5E701A92046104B98470028F9D19DF84F
:10F4400004302B70BEE701A920460B4B98470028DB
:10F45000F9D19DF804302B70B7E700BF00C200401F
:10F4600000020240004202400082014000C201400E
:10F4700000820040000204405DD3400038B50446DD
:10F480000D46274B984213D0264B984218D0264B56
:10F4900098421DD0254B984222D0254B984227D028
:10F4A000244B98422CD0244B984231D0002038BDB8
:10F4B00029462046214B98470028F9D1012038BD24
:10F4C000294620461D4B98470028F9D1012038BD18
:10F4D00029462046194B98470028F9D1012038BD0C
:10F4E00029462046154B98470028F9D1012038BD00
:10F4F00029462046114B98470028F9D1012038BDF4
:10F50000294620460D4B98470028F9D1012038BDE7
:10F5100029462046094B98470028F9D1012038BDDB
:10F5200000C200400002024000420240008201404E
:10F5300000C20140008200400002044035D3400078
:10F5400000B583B002A9002341F8043D084B1868B8
:10F55000084B9847019B3BB14FF08052064B1A6015
:10F56000BFF34F8FBFF36F8F03B05DF804FB00BF95
:10F57000F00F00202DEE400004ED00E070B58AB0E1
:10F580001D4B0FCB0AAC04E90F001C4D1C4B1D603A
:10F590001C4A1D4B1A601D4A1D4B1A60069B0093A6
:10F5A000079B0193089B0293099B039300240494F7
:10F5B000184E3046184B984701213046174B984754
:10F5C000174A69462846174B98472846164B9847CE
:10F5D0002846164B9847164E336821469868154DB5
:10F5E000A847336821465868A84733682146986879
:10F5F000A8470AB070BD00BF3841410000820140F9
:10F60000F81F00207DF44000F41F002095F3400017
:10F61000F01F0020008001401DCF400085D0400039
:10F620000000DC05C1D340000DD3400019D34000D9
:10F63000F80200209510410008B50A46014602482C
:10F64000024B9847FEE700BFF0414100150741001B
:10F65000704770472DE9F04383B04A4B98474A4AB8
:10F66000936843F0254343F480139360474B9847D6
:10F67000474B9847474B9847474B9847474B9847C6
:10F68000474B98470446474B9847F022014620468F
:10F69000454B9847454B98474548464B03602223C6
:10F6A000037123234371444D2946444CA0474448E9
:10F6B000444B03602B2303712A2343712946A0473F
:10F6C000414B9847414B98474148424B98474248E5
:10F6D000424CA04742494348A04743494348A047BA
:10F6E000434A44494448A04700230193042200921E
:10F6F0004FF4807241494248424CA047012802D051
:10F700004148364B98473D48404B9847404B18601E
:10F71000404B9847404B9847404B9847404B984741
:10F72000404A00210F20404EB047404C03220B219D
:10F7300020463F4DA847DFF808914A46002128207F
:10F74000B0473C4F03220C213846A8472820DFF859
:10F75000F480C04701463846374FB8474A46002133
:10F760000D20B04703220B212046A8470D20C0479B
:10F7700001462046B847314B9847002003B0BDE80A
:10F78000F08300BF6945400010140E409DCD40003D
:10F7900045714000816540007DF54000516D40009D
:10F7A000096F4000116F4000C96D4000E56D4000D9
:10F7B0006020002000000240A0860100156A400081
:10F7C0004C20002000C0014039AC4000496440009A
:10F7D00041F540005D4540004841410015074100AA
:10F7E0006041410074414100F83A410080414100CC
:10F7F00094414100A0414100AC414100C44141005D
:10F800001D6F4000ADE34000CC414100C1E6400027
:10F81000F00F0020118E400041A3400031964000BF
:10F820006186400071F340009DAF4000000E0E4025
:10F830000DB0400000100E401BCD400021E4400000
:10F8400045F340003FCD400030B583B000248DF833
:10F8500004408DF805408DF806400F4B98470F4B3C
:10F86000984720460E4B98470E4D01A928460E4B4F
:10F87000984772B60D480E4CA0472846A0470D4B3E
:10F8800098470D4B98470D4B98470D4A136823F046
:10F890000103136003B030BD1171400099E44000D2
:10F8A000C94B40004C200020515A400060200020ED
:10F8B000AD6A40006D4B400085AC4000656E400075
:10F8C00010E000E0004870476020002000487047CA
:10F8D0004C20002008B5014B984708BD196F400027
:10F8E00008B5014B984708BD1B6F400001207047C9
:10F8F00008B50248024B984708BD00BF60200020B1
:10F900004D6B400008B50248024B984708BD00BF48
:10F910004C2000204D6B4000014B1878704700BF11
:10F92000ED0F0020014B1878704700BFEC0F00204E
:10F93000064A936823F07F4323F4706343F0254322
:10F9400043F4E0639360024B1360FEE700140E4043
:10F95000080000A570B58AB0044600F06FF8324B7D
:10F9600093F900506B1C064609D02146204600F052
:10F970008DFE20B90021204600F07EFE10B13046F9
:10F980000AB070BD294B08902046019300F006FB99
:10F99000CDE90401CDE902012046CDB9244B4FF059
:10F9A00060420021CDE9062300F03EFE002833D05E
:10F9B00002230093684600F085F9A8B1089BC3B9FB
:10F9C000DDE9060100F03EFB064630460AB070BD98
:10F9D000184B00220021CDE9062300F025FE68B176
:10F9E00002239D420093E5D100F066FE22230360CE
:10F9F000E4E700F061FE089B0360E1E70123022DCC
:10FA000000930BD100F058FE212303600A4800F058
:10FA10005BF9CDE90601D1E701230093684600F0C8
:10FA200051F90028F2D1EDE7F4020020084241002C
:10FA3000FFFFEFC70000F0FF1C4141002DE9F84F28
:10FA400030F000432DD00028014604464ADBB0F1D7
:10FA5000FF4F3BDAB0F5000F3CDB00268D4AC4F3C4
:10FA600016052A4402F40002E41582F07E507F3C21
:10FA700034444FF07E51284304EBD25400F036FB5F
:10FA800005F10F03C3F316030F2B064631DC0021EB
:10FA900000F0CAFD002800F094804CB90020BDE8B9
:10FAA000F88F00214FF04C4000F0DEFCBDE8F88FED
:10FAB000204600F0D1FB7849054600F021FC77494B
:10FAC0000446284600F01CFC0146204600F010FBCE
:10FAD000BDE8F88F4FF0984100F012FC6FF0180667
:10FAE0000446BBE700F002FB002100F0BDFCBDE8CE
:10FAF000F88F4FF0804100F0FBFA0146304600F0ED
:10FB0000B3FC8046204600F0A7FB414681464046B4
:10FB100000F0F6FB0146834600F0F2FB6049DFF897
:10FB2000A0A1074600F0ECFB5E4900F0E1FA39467F
:10FB300000F0E6FB5C4900F0DBFA394600F0E0FB40
:10FB40005A4900F0D5FA594600F0DAFB5849834685
:10FB5000384600F0D5FB574900F0CAFA394600F0A4
:10FB6000CFFB554900F0C4FA394600F0C9FB014605
:10FB7000584600F0BDFAC5F55713AA4403F52273A1
:10FB800043EA0A03002B074665DD4FF07C513046FF
:10FB900000F0B6FB314600F0B3FB0546002C32D135
:10FBA0002946384600F0A4FA414600F0A9FB014678
:10FBB000284600F09BFA0146304600F097FABDE86F
:10FBC000F88F3E49304600F09BFB01464FF07C50D9
:10FBD00000F08CFA31460546304600F091FB0146B4
:10FBE000284600F08DFB0546002C2ED0204600F064
:10FBF00033FB2949074600F083FB28490446384671
:10FC000000F07EFB14E02449484600F079FB2946C9
:10FC10000446384600F06CFA414600F071FB1F497B
:10FC20000746484600F06CFB0146384600F060FA93
:10FC30000146284600F05AFA314600F057FA0146CC
:10FC4000204600F053FABDE8F88F0146304600F038
:10FC50004DFABDE8F88F7CB10F49484600F050FBE3
:10FC600039460446304600F041FA414600F048FB70
:10FC70000A4905464846C3E70146304600F036FAD1
:10FC8000414600F03DFB0146304600F02FFABDE84A
:10FC9000F88F00BF20FB4A008071313FD1F7173742
:10FCA0009788173E25333A3E2549923EABAA2A3F14
:10FCB0004FD01C3E298E633ECDCCCC3EABAAAA3E93
:10FCC000305CCFFF0020704700200149704700BF23
:10FCD0000000F87F81F0004102E000BF83F00043A4
:10FCE00030B54FEA41044FEA430594EA050F08BFD7
:10FCF00090EA020F1FBF54EA000C55EA020C7FEA9B
:10FD0000645C7FEA655C00F0E2804FEA5454D4EB17
:10FD10005555B8BF6D420CDD2C4480EA020281EAE1
:10FD2000030382EA000083EA010180EA020281EA19
:10FD30000303362D88BF30BD11F0004F4FEA01316B
:10FD40004FF4801C4CEA113102D0404261EB41017A
:10FD500013F0004F4FEA03334CEA133302D0524200
:10FD600063EB430394EA050F00F0A780A4F10104BC
:10FD7000D5F1200E0DDB02FA0EFC22FA05F28018F6
:10FD800041F1000103FA0EF2801843FA05F35941DC
:10FD90000EE0A5F120050EF1200E012A03FA0EFC5B
:10FDA00028BF4CF0020C43FA05F3C01851EBE37185
:10FDB00001F0004507D54FF0000EDCF1000C7EEBA2
:10FDC00000006EEB0101B1F5801F1BD3B1F5001FE0
:10FDD0000CD349085FEA30004FEA3C0C04F10104FF
:10FDE0004FEA445212F5800F80F09A80BCF1004F28
:10FDF00008BF5FEA500C50F1000041EB045141EAAA
:10FE0000050130BD5FEA4C0C404141EB010111F4AA
:10FE1000801FA4F10104E9D191F0000F04BF014655
:10FE20000020B1FA81F308BF2033A3F10B03B3F133
:10FE300020020CDA0C3208DD02F1140CC2F10C02C3
:10FE400001FA0CF021FA02F10CE002F11402D8BF21
:10FE5000C2F1200C01FA02F120FA0CFCDCBF41EAED
:10FE60000C019040E41AA2BF01EB0451294330BDBC
:10FE70006FEA04041F3C1CDA0C340EDC04F1140499
:10FE8000C4F1200220FA04F001FA02F340EA030070
:10FE900021FA04F345EA030130BDC4F10C04C4F1B6
:10FEA000200220FA02F001FA04F340EA0300294696
:10FEB00030BD21FA04F0294630BD94F0000F83F4E0
:10FEC000801306BF81F480110134013D4EE77FEAC3
:10FED000645C18BF7FEA655C29D094EA050F08BF0F
:10FEE00090EA020F05D054EA000C04BF19461046F0
:10FEF00030BD91EA030F1EBF0021002030BD5FEA34
:10FF0000545C05D14000494128BF41F0004130BD5B
:10FF100014F580043CBF01F5801130BD01F00045AF
:10FF200045F0FE4141F470014FF0000030BD7FEA22
:10FF3000645C1ABF194610467FEA655C1CBF0B461D
:10FF4000024650EA013406BF52EA033591EA030F34
:10FF500041F4002130BD00BF90F0000F04BF00212C
:10FF6000704730B54FF4806404F132044FF000055F
:10FF70004FF0000150E700BF90F0000F04BF0021D8
:10FF8000704730B54FF4806404F1320410F000453E
:10FF900048BF40424FF000013EE700BF42004FEA39
:10FFA000E2014FEA31014FEA02701FBF12F07F43B6
:10FFB00093F07F4F81F06051704792F0000F14BFB3
:10FFC00093F07F4F704730B54FF4607401F00045F7
:10FFD00021F0004120E700BF50EA010208BF70474E
:10FFE00030B54FF000050AE050EA010208BF704743
:10FFF00030B511F0004502D5404261EB41014FF4AC
:020000040041B9
:10000000806404F132045FEA915C3FF4DCAE4FF0AF
:1000100003025FEADC0C18BF03325FEADC0C18BF96
:10002000033202EBDC02C2F1200300FA03FC20FAE7
:1000300002F001FA03FE40EA0E0021FA02F1144434
:10004000C1E600BF4FEA4102B2F1E04324BFB3F57D
:10005000001CDCF1FE5C0DD901F0004C4FEAC0023F
:100060004CEA5070B2F1004F40EB830008BF20F023
:100070000100704711F0804F21D113F13872BCBFDD
:1000800001F00040704741F480114FEA5252C2F132
:100090001802C2F1200C10FA0CF320FA02F018BF7B
:1000A00040F001004FEAC1234FEAD32303FA0CFCCE
:1000B00040EA0C0023FA02F34FEA4303CCE77FEA5D
:1000C000625307D150EA01331EBF4FF0FE4040F4A7
:1000D0004000704701F0004040F0FE4040F4000056
:1000E000704700BF80F0004002E000BF81F0004197
:1000F00042001FBF5FEA410392EA030F7FEA226CCE
:100100007FEA236C6AD04FEA1262D2EB1363C1BF5D
:10011000D218414048404140B8BF5B42192B88BFCC
:10012000704710F0004F40F4000020F07F4018BFEF
:10013000404211F0004F41F4000121F07F4118BF0F
:10014000494292EA030F3FD0A2F1010241FA03FCB7
:1001500010EB0C00C3F1200301FA03F100F000439F
:1001600002D5494260EB4000B0F5000F13D3B0F167
:10017000807F06D340084FEA310102F10102FE2AD6
:1001800051D2B1F1004F40EBC25008BF20F0010046
:1001900040EA03007047490040EB000010F4000FF4
:1001A000A2F10102EDD1B0FA80FCACF1080CB2EB87
:1001B0000C0200FA0CF0AABF00EBC25052421843E6
:1001C000BCBFD0401843704792F0000F81F400018B
:1001D00006BF80F400000132013BB5E74FEA41035E
:1001E0007FEA226C18BF7FEA236C21D092EA030FCA
:1001F00004D092F0000F08BF0846704790EA010F44
:100200001CBF0020704712F07F4F04D1400028BF70
:1002100040F00040704712F100723CBF00F5000052
:10022000704700F0004343F0FE4040F40000704788
:100230007FEA226216BF08467FEA23630146420234
:1002400006BF5FEA412390EA010F40F48000704747
:100250004FF0000304E000BF10F0004348BF4042ED
:100260005FEA000C08BF704743F0964301464FF029
:1002700000001CE050EA010208BF70474FF0000385
:100280000AE000BF50EA010208BF704711F00043C6
:1002900002D5404261EB41015FEA010C02BF844696
:1002A0000146002043F0B64308BFA3F18053A3F5F5
:1002B0000003BCFA8CF2083AA3EBC25310DB01FA3C
:1002C00002FC634400FA02FCC2F12002BCF1004FC0
:1002D00020FA02F243EB020008BF20F00100704751
:1002E00002F1200201FA02FCC2F1200250EA4C00A5
:1002F00021FA02F243EB020008BF20EADC707047EB
:100300004FF0FF0C1CEAD0521EBF1CEAD15392EAF8
:100310000C0F93EA0C0F6FD01A4480EA010C4002D4
:1003200018BF5FEA41211ED04FF0006343EA50102E
:1003300043EA5111A0FB01310CF00040B1F5000F70
:100340003EBF490041EAD3715B0040EA010062F11F
:100350007F02FD2A1DD8B3F1004F40EBC25008BF09
:1003600020F00100704790F0000F0CF0004C08BF27
:1003700049024CEA502040EA51207F3AC2BFD2F1F4
:10038000FF0340EAC250704740F400004FF0000302
:10039000013A5DDC12F1190FDCBF00F0004070473C
:1003A000C2F10002410021FA02F1C2F1200200FA7A
:1003B00002FC5FEA310040F1000053EA4C0308BF41
:1003C00020EADC70704792F0000F00F0004C02BF92
:1003D000400010F4000F013AF9D040EA0C0093F00D
:1003E000000F01F0004C02BF490011F4000F013B67
:1003F000F9D041EA0C018FE70CEAD15392EA0C0FD5
:1004000018BF93EA0C0F0AD030F0004C18BF31F03F
:10041000004CD8D180EA010000F00040704790F015
:10042000000F17BF90F0004F084691F0000F91F0B9
:10043000004F14D092EA0C0F01D142020FD193EA7F
:100440000C0F03D14B0218BF084608D180EA010007
:1004500000F0004040F0FE4040F40000704740F0E3
:10046000FE4040F4400070474FF0FF0C1CEAD052B1
:100470001EBF1CEAD15392EA0C0F93EA0C0F69D00D
:10048000A2EB030280EA010C49024FEA402037D078
:100490004FF0805343EA111143EA10130CF000406F
:1004A0008B4238BF5B0042F17D024FF4000C8B425F
:1004B00024BF5B1A40EA0C00B3EB510F24BFA3EB3F
:1004C000510340EA5C00B3EB910F24BFA3EB91030F
:1004D00040EA9C00B3EBD10F24BFA3EBD10340EA69
:1004E000DC001B0118BF5FEA1C1CE0D1FD2A3FF6AF
:1004F00050AF8B4240EBC25008BF20F00100704764
:100500000CF0004C4CEA50207F32C2BFD2F1FF0306
:1005100040EAC250704740F400004FF00003013A37
:1005200037E792F0000F00F0004C02BF400010F4DB
:10053000000F013AF9D040EA0C0093F0000F01F0EF
:10054000004C02BF490011F4000F013BF9D041EA11
:100550000C0195E70CEAD15392EA0C0F08D1420244
:100560007FF47DAF93EA0C0F7FF470AF084676E717
:1005700093EA0C0F04D14B023FF44CAF08466EE7F0
:1005800030F0004C18BF31F0004CCAD130F00042BE
:100590007FF45CAF31F000437FF43CAF5FE700BF16
:1005A0004FF0FF3C06E000BF4FF0010C02E000BF3F
:1005B0004FF0010C4DF804CD4FEA40024FEA4103E1
:1005C0007FEA226C18BF7FEA236C11D001B052EA97
:1005D000530C18BF90EA010F58BFB2EB030088BF5D
:1005E000C81738BF6FEAE17018BF40F001007047CC
:1005F0007FEA226C02D15FEA402C05D17FEA236CAE
:10060000E4D15FEA412CE1D05DF8040B704700BFF4
:10061000844608466146FFE70FB5FFF7C9FF00288B
:1006200048BF10F1000F0FBD4DF808EDFFF7F4FFC4
:100630000CBF012000205DF808FB00BF4DF808ED5D
:10064000FFF7EAFF34BF012000205DF808FB00BF80
:100650004DF808EDFFF7E0FF94BF012000205DF8A2
:1006600008FB00BF4DF808EDFFF7D2FF94BF012053
:1006700000205DF808FB00BF4DF808EDFFF7C8FF4C
:1006800034BF012000205DF808FB00BF4FEA4002A4
:100690004FEA41037FEA226C02D15FEA402C08D185
:1006A0007FEA236C02D15FEA412C02D14FF00000B7
:1006B00070474FF001007047014B1868704700BF4A
:1006C000F802002070B50F4E0F4D761BB61018BF04
:1006D000002405D0013455F8043B9847A642F9D1CF
:1006E0000A4E0B4D761B03F047FEB61018BF0024D0
:1006F00006D0013455F8043B9847A642F9D170BDA5
:1007000070BD00BF84434100844341008C434100DD
:10071000844341000FB400B5074983B004AB0868B7
:1007200053F8042B8168019300F038FE03B05DF8A4
:1007300004EB04B0704700BFF8020020024B0146F2
:10074000186800F00BB800BFF8020020024B014609
:10075000186801F03FBF00BFF80200202DE9F04FFC
:1007600001F10B06162E83B0054640F29E8036F04E
:10077000070600F1BD80B14200F2BA8000F06CFCC7
:10078000B6F5FC7FC0F09382730A00F0B880042BAA
:1007900000F27981B30903F1390003F1380EC30087
:1007A000BF4F3B44A3F108015C68A14206D10CE0B5
:1007B000002A80F2AA80E468A14206D0636823F090
:1007C00003039A1B0F2AF3DD70463C69DFF8E4E26D
:1007D000744500F0AB81636823F003039A1B0F2A72
:1007E00000F39081002AC7F814E0C7F810E080F207
:1007F0009D80B3F5007F80F06181DB0803F1010C7F
:1008000099107A6857F83C80C4F8088001238B401F
:1008100007EBCC0113430839E1607B6047F83C40AB
:10082000C8F80C408210012494409C4200F28B8056
:100830001C4206D120F0030064001C4200F10400B9
:10084000FAD007EBC009CC468046DCF80C309C455A
:1008500007D16DE1002A80F27B81DB689C4500F0C6
:100860006781596821F003018A1B0F2AF2DDD3F852
:100870000CC0D3F8088000939C19284646F0010666
:1008800042F001055E60C8F80CC0CCF808807C61BD
:100890003C61C4F80CE0C4F808E065605A5000F010
:1008A000E1FB009B03F108041EE0102920D800F0B2
:1008B000D3FB102618230220794F3B44A3F10802F2
:1008C0005C68944200F03D816368E168A66823F0AB
:1008D0000303234428465A68F16042F001028E6007
:1008E0005A6000F0BFFB0834204603B0BDE8F08F2B
:1008F00000240C2320462B6003B0BDE8F08F40207D
:100900004FF400734FF03F0E4AE72344E1685A6802
:10091000A66842F00102F16028468E605A6000F03D
:10092000A1FB0834204603B0BDE8F08F23442846DD
:100930005A6842F001025A6000F094FB08342046E5
:1009400003B0BDE8F08FBC68636823F00308B045CE
:1009500004D3A8EB06030F2B00F38580DFF8589132
:10096000504BD9F800201B680132334404EB080ACD
:1009700000F0558103F580530F3323F47F6B2BF088
:100980000F0B5946284600F073FB411C024600F04D
:10099000FC80824500F2F780434B19685944196086
:1009A00000F04D81D9F8000001301BBFA2EB0A0A0C
:1009B0005144C9F80020196012F0070100F01581B8
:1009C000C1F10800C1F580510244083102EB0B0966
:1009D000C9F30B09A1EB0909494628460193009286
:1009E00000F046FB431C9DE80C0000F04381801A98
:1009F000484440F001001968BA604944BC42506064
:100A0000196017D0B8F10F0F40F2FB806068A8F1B1
:100A10000C0222F0070204EB020E00F001004FF07E
:100A2000050C10430F2A6060CEF804C0CEF808C051
:100A300000F217811D4BBC681A68914288BF19608B
:100A40001B4B1A689142626888BF196022F003024A
:100A50009642A2EB060301D80F2B04DC284600F0D7
:100A600001FB002440E7A21943F0010346F0010610
:100A700066602846BA60536000F0F4FA08342046F5
:100A800003B0BDE8F08F142B71D9542B00F2A38072
:100A9000330B03F16F0003F16E0EC30080E600BF5D
:100AA0002807002024100020F40F00201C10002034
:100AB0002010002030070020300B00205A0A042AA2
:100AC0005BD9142A00F2AE8002F15C01C9005B32EE
:100AD00007EB010C7958ACF1080C8C4500F08880CC
:100AE0004A6822F00302934273D289688C45F7D199
:100AF000DCF80C207B68E260C4F808C09460CCF895
:100B00000C408FE6A11946F0010C42F00106C4F832
:100B100004C0284679613961C1F80CE0C1F808E0E9
:100B20004E60E25000F09EFA0834DDE67B6879E61C
:100B300008F1010818F0030F0CF1080C7FF485AEE2
:100B40002DE0DC68A34208BF02303FF43EAEBBE6B6
:100B500019441C464A68DB6854F8086F42F00102E9
:100B60004A602846F3609E6000F07CFABCE603F120
:100B70005C0003F15B0EC30012E69A0902F1390131
:100B8000C9003832A4E7BC4254D0BC68626822F085
:100B900003025DE759F80839994540F0868010F066
:100BA000030F00F1FF30F5D17B6823EA04037B607B
:100BB00064009C423FF6C7AE002C3FF4C4AE1C421A
:100BC00040467FF43EAE64001C4200F10400FAD0BF
:100BD00037E68C468CE7B3F5AA7F15D8F30B03F103
:100BE000780003F1770EC300DAE54FF48051EDE6AB
:100BF0007B689210012101FA02F213437B60624686
:100C000079E70123536029E740F25452934222D8F6
:100C1000B30C03F17D0003F17C0EC300C0E503F1CA
:100C2000100BAEE6542A29D81A0B02F16F01C90045
:100C30006E324DE7204B196859441960B2E6CAF389
:100C40000B0000287FF4AEAE08EB0B03BA6843F04C
:100C500001035360EEE67F204FF47E734FF07E0E6B
:100C60009EE504F108012846009301F0B3FC009BC7
:100C70001968DFE601204FF00009BCE6B2F5AA7F53
:100C800005D8DA0B02F17801C900773220E740F28B
:100C900054518A4205D89A0C02F17D01C9007C3278
:100CA00016E74FF47E717E2212E77B6880E7F0083A
:100CB00006F1080300E600BFF40F0020000000006A
:100CC00001F0FF01102A2BDB10F0070F08D010F8FD
:100CD000013B013A8B422DD010F0070F42B3F6D101
:100CE000F0B441EA012141EA014122F007047FF01A
:100CF00000070023F0E80256083C85EA010586EA71
:100D0000010685FA47F5A3FA87F586FA47F6A5FAAC
:100D100087F68EB9EED1F0BC01F0FF0102F00702B8
:100D200032B110F8013B013A83EA010313B1F8D163
:100D30000020704701387047002D06BF3546033844
:100D4000073815F0010F07D1013015F4807F02BF7D
:100D5000013015F4C03F0130F0BC0138704700BFCE
:100D6000032A70B422D940EA01039B0711D003780B
:100D70000C78A3421DD10A44013105E010F8013F6F
:100D800011F8014BA34214D19142F7D1002070BC5D
:100D900070470D680668AE420C46034601F1040137
:100DA00000F1040008D1043A032AF2D8002ADED167
:100DB000ECE7181B70BC704721461846D7E700BF08
:100DC000844641EA000313F003036DD1403A41D356
:100DD00051F8043B40F8043B51F8043B40F8043B15
:100DE00051F8043B40F8043B51F8043B40F8043B05
:100DF00051F8043B40F8043B51F8043B40F8043BF5
:100E000051F8043B40F8043B51F8043B40F8043BE4
:100E100051F8043B40F8043B51F8043B40F8043BD4
:100E200051F8043B40F8043B51F8043B40F8043BC4
:100E300051F8043B40F8043B51F8043B40F8043BB4
:100E400051F8043B40F8043B51F8043B40F8043BA4
:100E5000403ABDD2303211D351F8043B40F8043B44
:100E600051F8043B40F8043B51F8043B40F8043B84
:100E700051F8043B40F8043B103AEDD20C3205D354
:100E800051F8043B40F8043B043AF9D2043208D04C
:100E9000D2071CBF11F8013B00F8013B01D30B88BE
:100EA00003806046704700BF082A13D38B078DD09C
:100EB00010F003038AD0C3F10403D21ADB071CBF6E
:100EC00011F8013B00F8013B80D331F8023B20F8D8
:100ED000023B7BE7043AD9D3013A11F8013B00F811
:100EE000013BF9D20B7803704B7843708B78837099
:100EF000604670478842F0B50DD98B1898420AD2E7
:100F00008418002A51D0224613F8014D02F8014DF1
:100F10009942F9D1F0BD0F2A48D941EA00039B0755
:100F200046D100F1100401F11003154653F8106C7E
:100F300044F8106C53F80C6C44F80C6C53F8086CC3
:100F400044F8086C103D53F8046C44F8046C0F2D01
:100F500003F1100304F11004E8D8A2F1100323F008
:100F60000F0302F00F0E1033BEF1030F19440344B8
:100F700021D91E1F0D467446043C55F8047B46F8E3
:100F8000047F032CF8D8AEF1040424F003040434E5
:100F90002144234402F0030262B1013B0A4411F8E8
:100FA000014B03F8014F8A42F9D1F0BD0346F3E744
:100FB0000346F2E7F0BD7246EEE700BF70B4860765
:100FC00046D0541E002A41D0CAB2034602E014F1B2
:100FD000FF343BD303F8012B9D07F8D1032C2ED906
:100FE000CDB245EA05250F2C45EA054519D903F18F
:100FF00010022646103E0F2E42F8105C42F80C5CA0
:1010000042F8085C42F8045C02F11002F2D8A4F144
:10101000100222F00F0204F00F041032032C1344CC
:101020000DD91E462246043A032A46F8045BFAD834
:10103000221F22F003020432134404F003042CB1F3
:10104000C9B21C4403F8011B9C42FBD170BC704721
:1010500014460346C2E700BF014801F055BD00BF7A
:1010600084200020014801F051BD00BF84200020F1
:1010700038B5074C0023054608462360FCF7E6FA1E
:10108000431C00D038BD2368002BFBD02B6038BD3B
:101090009820002000290CBF022200224FF4806318
:1010A00000F000B82DE9F043614C256883B0044698
:1010B0000F4690461E4615B1AB6B002B64D0B8F1BD
:1010C000020F06D0B8F1010F00F29F80002EC0F28F
:1010D0009C80636ED80734D52146284601F0FCF881
:1010E000216B41B104F14003994202D0284601F03E
:1010F00071FA00232363B4F90C300022A26162600C
:101100001A063AD423F44A6323F00303B8F1020F1A
:10111000A3811DD001AB6A462146284601F0F8FCA8
:10112000A3891843A081002E32D1009E3046FFF7DC
:1011300005FB074600286BD0A38943F08003A381F9
:1011400028E0A3899905C7D4A06D01F0DDFCC3E7B1
:101150000025616E002604F1430243F002030120E2
:10116000A660CE07A38122602261606101D4980548
:101170003ED5284603B0BDE8F0832169284601F03A
:1011800029FAB4F90C30BDE7284601F0FDF896E7DE
:10119000002FCBD0AB6B002B33D0009BB4F90C20CD
:1011A00027609E421CBF42F40062A281B8F1010F89
:1011B00004BF42F00102A28192B212F0080327613B
:1011C00066610ED0D1071AD5656E7642002315F000
:1011D0000105A661A36009D00025284603B0BDE83B
:1011E000F083A360656E15F00105F5D19305C0D4B9
:1011F000A06D01F08BFC284603B0BDE8F083A6602B
:10120000F0E7284601F0C0F8C7E74FF0FF35B0E738
:10121000DDF80090B14504D04846FFF78FFA074645
:1012200020B9B4F90C304FF0FF3592E74E4683E712
:10123000F802002000000000000000000000000094
:1012400090F800F06DE9024520F007016FF0000C06
:1012500010F0070491F820F040F049804FF00004AE
:101260006FF00700D1E9002391F840F000F1080089
:1012700082FA4CF2A4FA8CF283FA4CF3A2FA8CF3C1
:101280004BBBD1E9022382FA4CF200F10800A4FA28
:101290008CF283FA4CF3A2FA8CF3E3B9D1E904237C
:1012A00082FA4CF200F10800A4FA8CF283FA4CF3B3
:1012B000A2FA8CF37BB9D1E9062301F1200182FA6D
:1012C0004CF200F10800A4FA8CF283FA4CF3A2FA73
:1012D0008CF3002BC6D0002A04BF04301A4612BA81
:1012E000B2FA82F2FDE8024500EBD2007047D1E984
:1012F000002304F00305C4F100004FEAC50514F013
:10130000040F91F840F00CFA05F562EA05021CBFE3
:1013100063EA050362464FF00004A9E72DE9F84FA0
:101320004B6E9C0493462FD59368126853B30E46B8
:10133000074602F1080919E920045FEA9A0817D064
:10134000043D002401E0A04510D0324655F8041FAA
:10135000384601F0BBF8431C04F10104F3D100232B
:10136000CBF80830CBF80430BDE8F88FDBF8083054
:101370002AF0030AA3EB0A03CBF8083009F10809A5
:10138000002BD8D10020EAE701F00AFA0023CBF8BD
:101390000830CBF80430BDE8F88F00BF2DE9F04FDE
:1013A000ADB01D468B4690460793069018B1836BEF
:1013B000002B00F0F380DBF86430BBF90C00DF0792
:1013C00081B202D48E0540F1FC808C040AD4DBF893
:1013D000643040F4005123F40053ABF80C10CBF808
:1013E000643089B2080740F1B380DBF81030002B7D
:1013F00000F0AE8001F01A030A2B00F0B580002344
:101400000DF170090B93119310930393CDF83C9059
:10141000CA46CDF810B098F800304446FBB1252BF1
:1014200002D11CE0252B03D014F8013F002BF9D189
:10143000A4EB08059DB1109B119ACAF800800133F6
:101440002A44072BCAF80450119210937ADD002A1F
:1014500040F0B084039B10922B44CA460393237838
:10146000002B00F0E08300204FF000038DF83730B0
:1014700004F1010862780546064603464FF0FF3442
:1014800008F10108A2F12001582900F2DE82DFE80C
:1014900011F02102DC02DC022902DC02DC02DC02A7
:1014A000DC02DC02DC0289029502DC02A200BD0241
:1014B000DC029F01A401A401A401A401A401A401D0
:1014C000A401A401A401DC02DC02DC02DC02DC02D7
:1014D000DC02DC02DC02DC02DC02B201DC02DC0247
:1014E000DC02DC02DC02DC02DC02DC02DC02DC020C
:1014F0009701DC02DC02DC02DC02DC029B01DC0284
:10150000DC025302DC02DC02DC02DC02DC02DC0274
:10151000DC02DC02DC02DC025A021B02DC02DC021E
:10152000DC026E021B02DC02DC027302DC02F5014B
:1015300082010902D702DC029A02DC02A700DC0267
:10154000DC022E020AF1080A039B2B44039386E770
:101550005946069800F0ACFD18BBBBF80C1001F022
:101560001A030A2B7FF44BAFBBF90E30002BFFF6AA
:1015700046AFDBF86430DB0705D48F0503D4DBF816
:10158000580001F0C3FA2B4642465946069800F02F
:101590004DFD039003982DB0BDE8F08F00F0F4FEF0
:1015A00009E7DBF86430D90704D4BBF80C309A059E
:1015B00040F1AA844FF0FF33039303982DB0BDE8A8
:1015C000F08FDBF8580001F09FFABBF90C0081B2F4
:1015D000FBE67642079243F0040398F800204FE7B9
:1015E00008969E0600F150840799DD060A4600F130
:1015F000EF83580640F1EC830E8804310027012266
:1016000007914FF000018DF837100025611C00F0A4
:10161000168123F08001029156EA070140F01481FF
:10162000002C40F05C83002A40F0B78313F00103E4
:10163000059300F057840DF1B00B30230BF8413DBA
:10164000059BA342B8BF234601930DB1013301931B
:10165000029B13F00203099302D0019B0233019312
:10166000029B13F084030A9340F01782089B019AAF
:101670009D1A002D40F31182102D40F39084109B91
:10168000119AC44ED6461027A2461946069C07E07A
:1016900001F1020C0EF1080E0146103D102D11DD76
:1016A000481C1032072811928EE8C0001090EFDD20
:1016B000002A40F0E481103D102D11464FF0010C3E
:1016C000CE46EDDC54466146F2462A440729119283
:1016D000CAF80060CAF80450109100F3EC829DF83B
:1016E00037500AF1080A481C002D40F0DE81099BA2
:1016F000002B00F0F88102320EA902230728119274
:1017000010908AE80A0040F3EA81002A40F08C83B6
:101710000A9B802B4FF001001146CA4640F0E7813A
:10172000089B019D5E1B002E40F3E181102E9A4D17
:1017300040F35084D4461027A246069C07E001F1EE
:10174000020E0CF1080C0146103E102E11DD481C53
:101750001032072811928CE8A0001090EFDD002ACB
:1017600040F09D82103E102E4FF0010E1146CC46E7
:10177000EDDC5446E2463244BEF1070F11928AE88E
:101780006000CDF840E000F369830AF1080A0EF129
:1017900001007146ABE1089613F0200240F08C8303
:1017A00013F0100140F01A8313F0400200F016838A
:1017B00007980A460146043106880791002720E76A
:1017C000089643F01003E7E7089643F0100308E794
:1017D00043F0800398F8002052E6A2F13001002681
:1017E00018F8012B06EB860601EB4606A2F1300144
:1017F0000929F5D946E60896002840F0088443F008
:1018000010039E0600F14C83DD0600F1F3825806BA
:1018100040F1F082079DB5F900602A46F7170432BF
:10182000304639460792002871F10002C0F25D830C
:10183000611C9DF837504FF001027FF4EAAE56EA82
:10184000070100F04D820293012A00F08C82022AE7
:1018500040F05C820B98CB46330906F00F0143EA57
:1018600007733A091E461746435C0BF8013D56EADA
:101870000703F1D1A9EB0B030593E1E6002840F043
:10188000C083990600F16783DA0600F1F1805B06F8
:1018900040F1EE80079A136804320792BDF80C20DD
:1018A0001A80B8E507983D4A08960B920668782298
:1018B000302104308DF8392043F0020307900027CF
:1018C0008DF8381002229CE60896002899D08DF8F1
:1018D000375096E798F80020002D7FF4D1AD012015
:1018E0002025CDE543F0010398F80020C8E50896CF
:1018F000002840F0938329490B919F0600F1E8826C
:101900000798DE06014600F170825D0640F16D82A7
:101910000431068807910027D80740F1228256EA51
:10192000070100F01E8230218DF8392043F00203B8
:101930008DF83810022264E60896002840F06B8388
:1019400017490B91D9E7079908960A688DF848203E
:101950004FF000000A468DF8370004320120019054
:10196000079205900DF1480B0293002470E643F0B6
:10197000400398F8002083E598F800206C2A03BF04
:1019800098F8012043F0200308F1010843F0100308
:1019900076E500BF444241005442410028424100E4
:1019A0001442410007990E680A46002E02F1040213
:1019B000FFF60FAE079298F8002061E598F8002036
:1019C00001202B255CE507990896D1F800B04FF06F
:1019D00000028DF837200E1DBBF1000F00F0E582EC
:1019E000671C00F0C4822246002158460193FFF78D
:1019F00067F9019B002800F0E582A0EB0B0205923D
:101A0000079602939DF83750002419E698F80020B5
:101A10002A2A08F1010700F0E982A2F13001092920
:101A2000B8464FF000043FF62DAD18F8012B04EB3B
:101A3000840401EB4404A2F130010929F5D921E520
:101A400043F0200398F800201AE50896002840F09B
:101A5000DB82002A00F0E78001218DF848204FF05A
:101A6000000201918DF8372005910DF1480B7BE7BD
:101A7000079A136804320792039A1A60CBE40FAAFC
:101A800004992046FFF74AFC002840F0398110995C
:101A9000119A01F1010CCE46FFE51099119A481CEC
:101AA0009DF83750002D3FF422AE01320DF137057D
:101AB0000121072811921090CAF80050CAF80410AA
:101AC00040F30881002A40F0BC81099B002B3FF4C1
:101AD0001FAE0EAB022208461C931D92CA46014659
:101AE0000AF1080A01300A9B802B3FF419AE059BCE
:101AF000E41A002C2EDD102CB34D1EDDD646102628
:101B0000069FDDF810A006E0881C0EF1080E1946AD
:101B1000103C102C10DD4B1C1032072B11928EE85C
:101B200060001093F0DD002A65D1103C102C4FF0BE
:101B300001001146CE46EEDCF246224407281192FF
:101B4000CAF80050CAF80440109000F385800AF1EA
:101B5000080A01300599CAF800B00A440728119212
:101B6000CAF80410109040F38280002A40F01881D7
:101B7000029B1092580735D5089B01995C1A002CDE
:101B800040F3E780CA46102C40F3188210998F4E1C
:101B9000069FDDF810B0102506E0881C0AF1080A3F
:101BA0001946103C102C11DD4B1C1032072B1192E2
:101BB000CAF80060CAF804501093EEDD42BB103C36
:101BC000102C4FF001001146CA46EDDC22440728D4
:101BD0001192CAF80060CAF80440109051DD002A42
:101BE00040F09B81039B089A01998A42ACBF9B18E5
:101BF0005B1803934EE00FAA51463846FFF78EFB61
:101C0000002840F03F811099119A481CCE467FE78A
:101C10000FAA59463846FFF781FB60B91099119A0F
:101C2000481CCA46BDE7119BDDF810B0002B40F000
:101C3000D48100231093DBF8643013F0010FBBF85C
:101C40000C3002D19A0540F1DE805B063FF5B2AC64
:101C500003982DB0BDE8F08F002A40F00681059A68
:101C60001D9201231192CDF870B01093CA460AF16B
:101C7000080A029B590704D5089B01995C1A002C9D
:101C800081DC039B089901988142ACBF5B181B184B
:101C9000039372BB00231093CA46FFF7BCBB0FAA85
:101CA00004992046FFF73AFB50BB1099119A01F1B5
:101CB000010ECC4648E5002A40F040819DF83710DF
:101CC000002900F01B8101220DF1370110461D9201
:101CD0001C91CA4601460AF1080A013007E5029B39
:101CE000012A00F09880022A0DD1029300260027D5
:101CF000B0E50FAA04990698FFF710FB0028C9D099
:101D0000DDF810B097E7029300260027494600E06F
:101D10005946F20842EA4772F80806F007030746F8
:101D20001646303356EA070201F8013C01F1FF3B49
:101D3000EED1029AD6077FF59DAD302B3FF49AADD8
:101D4000023930230BF8013CA9EB010305938B46C4
:101D500076E4039B089A8A42ACBF9B185B180393F6
:101D600098E702224DE4002F08BF0A2E52D3CB463B
:101D7000304639460A22002301F010FB30320BF8BE
:101D8000012D3046394600230A2201F007FB0646A2
:101D90000F4656EA0703EBD16CE50594CB464FE4BA
:101DA0000FAA04990698FFF7B9FA0028A8D1119A4A
:101DB000CA465EE70FAA04990698FFF7AFFA002813
:101DC0009ED1CA46FFF7C0BB544241004442410085
:101DD0000431166807910122002712E40798014692
:101DE00004310668079100270BE40E68043107915F
:101DF000002791E507990E680A46F7170432079203
:101E0000304639460FE5DBF8580000F07FFEBBF89E
:101E10000C301AE7029B02930DF1B00B3036012310
:101E20000BF8416D05930BE40FAA04990698FFF790
:101E300075FA00287FF464AF1099119A481CCA46BD
:101E400051E60FAA04990698FFF768FA00287FF474
:101E500057AF1099119A481CCA4648E4002A40F02E
:101E6000918001201146CA4641E60FAA04990698BE
:101E7000FFF754FA00287FF443AF1098119A01300D
:101E8000CA4667E6D346D6E6079E073626F007021F
:101E900002F10801D2E9006707910122FFF7B1BB07
:101EA000079E073626F00706D6E9000106F108026C
:101EB000079206460F46B6E4079E073626F007024D
:101EC00002F10801D2E9006707910022FFF799BBF0
:101ED000079E073626F0070101F108000790D1E9B7
:101EE000006719E5CB46FFF7ABBB2D25764267EBC4
:101EF00047078DF837500122FFF788BB099BB3B91C
:101F000011460120CA46F2E5DBF8580000F0FEFD5C
:101F10004FF0FF330393FFF750BB0FAA04990698C5
:101F2000FFF7FCF900287FF4EBAE119AA9E60EAB9F
:101F300002221C931D920120CA46D0E50FAA0499E3
:101F40000698FFF7EBF900287FF4DAAE1099119AA2
:101F5000481CCA46A4E5079A03991368CD1708469A
:101F6000043229460792C3E90001FFF754BA5846E4
:101F700007960293FFF764F9002405909DF8375007
:101F8000FFF75EBB0FAA04990698FFF7C7F9002870
:101F90007FF4B6AE1099119A481CCA46A7E510996D
:101FA000119A204E0131FFF790BB062C28BF062462
:101FB000059407960194DFF870B0D5E41098194E97
:101FC000013003E605949DF83750079602930446C6
:101FD000FFF736BB8646FFF7CEBB06980FAA5946D9
:101FE000FFF79CF900283FF424AE24E6079998F8FF
:101FF00001200C68043144EAE474B8460791FFF705
:102000003FBA8DF837503CE48DF8375021E58DF814
:102010003750FFF7F4BB8DF8375091E48DF8375007
:1020200069E400BF444241003C4241002DE9F041D7
:102030000C46ADF58D6D8989666EE589199621F09E
:1020400002010646E069ADF80C1017464FF48061B6
:10205000626AADF80E5098461AAD0023079016A894
:1020600009920693009504950291059100F048FDB0
:1020700043463A4669463046FFF790F9051E07DBAE
:102080003046694600F028F9002818BF4FF0FF35A8
:10209000BDF80C305B0603D5A38943F04003A38150
:1020A000169800F02FFD28460DF58D6DBDE8F081E6
:1020B00038B5304B1B6805460C4613B19A6B002AA5
:1020C00038D0B4F90C2093B218070CD52069A8B108
:1020D00013F001021ED0636900225B42A361A2607B
:1020E000F0B1002038BDD9063CD5580726D4206968
:1020F00042F00803A3819BB20028E9D103F42072C7
:10210000B2F5007FE4D02846214600F02FFDA389D8
:102110002069DDE7990758BF6269A2600028E0D115
:10212000B4F90C301A06DDD543F04003A3814FF01B
:10213000FF3038BD184600F027F9C2E7216B51B1D6
:1021400004F14003994204D0284600F043FAB4F960
:102150000C200023236300232069636022F0240203
:102160002060C5E742F0400209232B604FF0FF30AA
:10217000A28138BDF8020020024B13B1024800F0E2
:1021800005B8704700000000F92341000023014614
:102190001A46184600F0DABFB1F90C309AB22DE9B0
:1021A000F0410D46110780463AD46A6843F4006353
:1021B000002AAB816FDDAC6A002C49D000229BB2B3
:1021C000D8F80060C8F8002013F4805267D02A6D58
:1021D0005F0705D569682B6B521A0BB1EB6BD21AEE
:1021E0000023E9694046A047441C3CD0B5F90C30B7
:1021F0002A692A6023F400630022AB81DB046A6051
:1022000047D4296BC8F8006011B305F14003994227
:1022100002D0404600F0DEF900202863BDE8F081DE
:102220002E69AEB12C682E6091070CBF6B6900233C
:10223000A41BAB600AE0234632466F6AE969404658
:10224000B8470028A4EB0004064404DD002CF2DCAF
:102250000020BDE8F081AB8943F04003AB814FF033
:10226000FF30BDE8F081D8F800401D2CF3D8194BA1
:10227000E340DB4313F00103EDD1B5F90C206B60B3
:1022800022F400632969AB81DA042960B9D5002CF6
:10229000B7D12865B5E7EA6B002A8CDCD8E70123C3
:1022A000E9694046A047431C024602D0AB89AC6AAC
:1022B0008EE7D8F80030002BF8D01D2B01D0162B5C
:1022C00002D1C8F80060C3E7AB8943F04003AB819B
:1022D000BDE8F0810100402038B50D46044608B144
:1022E000836BBBB1B5F90C0088B16B6EDB0701D411
:1022F000810517D520462946FFF74EFF6B6EDA079A
:10230000044602D4AB899B0507D5204638BD044658
:10231000204638BD00F038F8E4E7A86D00F0F6FB81
:10232000204638BDA86D00F0EFFBE3E7014900F05F
:10233000AFBB00BF3532410010B500230446818198
:10234000C2810360436083604366036143618361CC
:10235000194608225C30FEF731FE07480749084A53
:10236000084B2062E4616162A262E36204F15800FA
:10237000BDE8104000F0C4BB792F41009D2F410003
:10238000D92F4100F92F410010B50446124800F042
:10239000BBFBA26BD2B904F53B731048C4F8E8321A
:1023A0000321C4F8E022E063C4F8E4126068042169
:1023B000FFF7C2FF01220921A068FFF7BDFF02223B
:1023C0001221E068FFF7B8FF0123A3630248BDE8CC
:1023D000104000F09BBB00BF802000202D23410057
:1023E000014800F091BB00BF94200020014800F09C
:1023F0008DBB00BF9420002038B50A4C0A4D641BE9
:10240000A4100AD004F18043013B05EB8305013C95
:1024100055F804399847002CF9D1BDE8384001F04F
:10242000B5BF00BF9C434100984341002DE9F047F0
:1024300082B080468946144600F054FB012836D00D
:102440004A4604F15C0301A9404600F031FE421CFB
:10245000064625D0A8B39DF804E000250DF1040A36
:1024600009E023685A1C226083F800E00135B54278
:1024700027D215F80AE0A368013B002BA360F0DA2D
:10248000A769BB4271462246404602DBBEF10A0FF5
:10249000E7D100F0B5FD431CE8D102B0BDE8F087FC
:1024A000A38943F04003A38102B0BDE8F08709F19E
:1024B000FF33FE2BC4D85FFA89FE06468DF804E090
:1024C000CBE7484602B0BDE8F08700BF30B5536E99
:1024D00013F0010FB2F90C30144683B005469AB2DE
:1024E00001D190051CD5900406D4626E43F40053CC
:1024F00042F40052A381626628462246FFF796FF07
:10250000636EDA07054602D4A3899B0502D52846E7
:1025100003B030BDA06D00F0F9FA284603B030BD1D
:10252000A06D019100F0F0FAB4F90C3001999AB263
:10253000D9E700BFF8B5244F0C460646FEF78CFDE0
:10254000BB685D68C4F57E610F3125F00305294441
:1025500021F47F6121F00F01A1F58054B4F5805F73
:1025600007DB00213046FEF783FDBB682B44984211
:1025700004D03046FEF776FD0020F8BD61423046BB
:10258000FEF776FD01300DD0104BBA6819682D1B8F
:1025900045F001053046091B55601960FEF762FDE4
:1025A0000120F8BD00213046FEF762FDBA68831AAB
:1025B0000F2BDEDD064C0549246843F00103001BA8
:1025C00053600860D5E700BF28070020F40F002003
:1025D000300B0020002944D02DE9F0410D46804603
:1025E000FEF73AFD55F8047C694927F00103A5F18F
:1025F0000804E2188E685068B24220F003005ED0F2
:10260000FE0750600BD455F8087CE41B01F1080E5E
:10261000A56875453B446DD0E768EF60BD6015184F
:102620006D68ED073ED543F001026260E350B3F5FB
:10263000007F17D2DB08581C9A104D6851F8307093
:10264000A7600123934001EBC0022B43083AE260EC
:102650004B6041F83040FC604046BDE8F041FEF779
:1026600001BD70475A0A042A52D89A0902F1390763
:10267000FF0002F13805C819CA59083890424FD0F6
:10268000516821F003018B4232D292689042F7D117
:10269000C368A060E3609C60C4604046BDE8F04150
:1026A000FEF7E0BC95683B4FBD42034440D0D06884
:1026B000E86043F0010285606260E350B7E7FF071E
:1026C000034407D455F8082CA41A1344A068E26800
:1026D000C2609060304A126843F00100934260602B
:1026E0008C60B9D32D4B40461968FFF723FFB3E741
:1026F0001046CDE711184968C90744D49168D268DB
:10270000CA60034443F0010091606060E350A3E7B6
:10271000142A16D802F15C07FF0002F15B05AAE754
:10272000AA1001234D6893402B434B600346B0E74A
:1027300043F001024C610C61E560A5606260E3500A
:102740008AE7542A06D81A0B02F16F07FF0002F13C
:102750006E0590E7B2F5AA7F06D8DA0B02F178078A
:10276000FF0002F1770586E740F25450824206D816
:102770009A0C02F17D07FF0002F17C057BE74FF424
:102780007E777E2577E743F001016160136063E7A0
:102790002807002030070020340B002024100020E0
:1027A0009368002B73D02DE9F04F8B8983B00C46D2
:1027B00019070090164626D5226922B313F00200AD
:1027C00035682CD04FF00009B04FC846B246B84526
:1027D00043464A4628BF3B460098B8F1000F50D008
:1027E000E169666AB047002858DDDAF808301B1A3C
:1027F0008144A8EB0008CAF80830002BE7D100207C
:1028000003B0BDE8F08F21460098FFF751FC002887
:1028100040F03381A389356813F00200D2D113F060
:10282000010945D14F46019637B39A05D4F808807F
:1028300040F183804745C346C0F0AB8013F4906FEE
:1028400040F0AC802068BA465A464946FEF752FB33
:10285000A2682368A2EB08025B44A2602360019A8D
:102860009368A3EB0A03D144A7EB0A079360002BFC
:10287000C5D0A389002FD8D1D5F800906F6808354E
:10288000D2E7D5F80090D5F8048008359FE70020FE
:10289000704721460098FFF71FFD70B3B4F90C3064
:1028A00043F040034FF0FF30A38103B0BDE8F08F49
:1028B000814633464E46A8469A464D464EB380B3AF
:1028C000206823696269B145CB4628BFB346984268
:1028D0005F4604D9A36813449B4500F3A680934543
:1028E0004BDB1346676AE16900982A46B847071E22
:1028F000D4DDB9EB0709CCD00120DAF80830DB1BB6
:102900003D44F61BCAF80830002B3FF478AF002E88
:10291000D5D108F1080313E9600098460833002E6A
:10292000F9D032460A212846FEF7CAF9002800F0FD
:10293000A1800130A0EB0509C2E720682369984215
:1029400002D863699F425DD2B84528BFB846424667
:102950004946FEF7CFFAA3682268A3EB0803424476
:10296000A36022600BB1C24679E721460098FFF7C9
:10297000B3FC002892D1C24671E75A462946FEF7B9
:10298000B9FAA2682368A2EB0B025B44A260236041
:10299000AFE72068B846BA46BB4655E7626920688B
:1029A000216902EB4208A0EB010A08EBD8780AF192
:1029B00001004FEA680838444045424684BF8046DB
:1029C00042465B0544D511460098FDF7C7FE834695
:1029D000002855D052462169FEF7F2F9A38923F465
:1029E000906343F08003A3810BEB0A00A8EB0A037A
:1029F000C4F810B0C4F814802060A360B846BA468A
:102A0000BB4621E76FF00041B94228BF39464A462C
:102A100091FBF3F10098666A03FB01F3E169B047AB
:102A2000B0F1000A3FF71BAF38E71A462946019379
:102A3000FEF760FA2268019B00981A442260214642
:102A4000FFF74AFC019B00287FF428AF1F4650E7A0
:102A5000009800F0EBF883460028C5D1009D21695D
:102A60002846FFF7B7FDB4F90C300C2223F08003A1
:102A70002A6015E706F1010922E74FF0FF30BFE6B3
:102A8000009A0C231360B4F90C3009E700FCFF7FB7
:102A90002DE9F84310F538771FD0884606464FF0E9
:102AA00000097D68BC68013D11D4A389012B05F1A3
:102AB000FF3508D9B4F90E3001332146304602D033
:102AC000C04749EA00096B1C04F16804EDD13F6876
:102AD000002FE6D14846BDE8F883B9464846BDE830
:102AE000F88300BF044B054A1B685B6B002B08BFD3
:102AF000134693F828017047F80200203C0B002091
:102B0000704700BF704700BF704700BF704700BFED
:102B100070B50C46B1F90E10002990B015461E464E
:102B200014DB01AA00F0E8FB00280FDB029A02F494
:102B30007042A2F50052B2FA82F252094FF4806359
:102B40004FF4006032602B6010B070BDA28900238A
:102B500012F08000336004D0402218462A6010B082
:102B600070BD4FF480632B6010B070BD8A899207EE
:102B70000B4606D501F1430201211A601A61596121
:102B80007047F0B583B001AB6A460C460646FFF7C6
:102B9000BFFF009905463046FDF7E0FDB4F90C3063
:102BA000D8B1019A154F0099F76343F08003A381D0
:102BB0002060206161611AB92B43A38103B0F0BD8D
:102BC0003046B4F90E1000F0ABFBA0B1A38923F09E
:102BD000030343F001031BB2EEE79A05EED423F0A2
:102BE000030304F1430243F002030121A3812260A5
:102BF00022616161E2E7B4F90C30DDE72D23410089
:102C000082B049B15AB16BB113780B601278101CC5
:102C100018BF012002B0704701A9002AF3D1104665
:102C200002B070476FF00100F4E700BF002900F028
:102C300095802DE9F04F0D46164683B0804606F18B
:102C40000B07FEF709FA55F804EC162F2EF00304D3
:102C5000A5F108093CD810221746BE423DD894423F
:102C600043DAC44B996809EB0400884200F0B48051
:102C7000436823F0010101444968C9074CD51EF09F
:102C8000010F00F09B8031464046FDF767FD064688
:102C900000283AD055F8043C23F001034B44A0F13E
:102CA00008029A4200F02181221F242A00F20781A3
:102CB000132A00F2DB8003462A4611681960516826
:102CC000596092689A6029464046FFF783FC1CE0F1
:102CD00027F00707002F3A46BFDA00260C233046BC
:102CE000C8F8003003B0BDE8F08F2E46E31B0F2B71
:102CF0001ED8D9F8043003F0010323434C44C9F82B
:102D00000430636843F0010363604046FEF7AAF9AC
:102D1000304603B0BDE8F08F23F00303E118914281
:102D20001FDBC36882682E46D3600C469A60DDE7DD
:102D3000D9F8042009EB070102F001024C4443F0EA
:102D400001031743C9F804704B60636843F0010343
:102D5000083163604046FFF73DFCD6E71146FDF7BA
:102D6000FDBC1EF0010F8ED155F8081CA9EB010A1D
:102D7000DAF8041021F003010B442344934225DBCD
:102D8000C26881685646CA609160DAF80C1056F83D
:102D9000080F221F242AC160886000F29480132A41
:102DA0006FD92968CAF808106968CAF80C101B2A7C
:102DB00000F2A28008350AF1100263E055F8083CE1
:102DC000A9EB030ADAF8041021F003016318934217
:102DD000FFF659AF5646D8E7416821F0030BA344EC
:102DE00007F11000834556DA1EF0010F7FF44BAF58
:102DF00055F8081CA9EB010ADAF8041021F00301C8
:102E00008B445845E2DC5646DAF80C1056F8080FA9
:102E1000221F242AC160886000F28F80132A40F2AA
:102E20008A802968CAF808106968CAF80C101B2A39
:102E300000F28A8008350AF1100229681160696879
:102E40005160A96891600AEB0701ABEB070242F001
:102E5000010299604A60DAF8043003F001031F436D
:102E60004046CAF80470FEF7FDF851E72B6803608E
:102E70006B6843601B2A2DD800F1080305F1080296
:102E80001BE732462968116069685160A968916042
:102E90001C46D1462AE709EB0701ABEB070B4BF0C9
:102EA000010299604A6055F8043C03F001031F4396
:102EB000404645F8047CFEF7D5F82E4628E729461B
:102EC000FEF718F8FFE6294630461C46D146FEF7C5
:102ED00011F80BE7AB688360EB68C360242A17D056
:102EE00000F1100305F11002E7E650F8043C23F06E
:102EF00003031C442E46F9E6A968CAF81010E968D5
:102F0000CAF81410242A0CD010350AF11802B9E7B7
:102F10002B6903616B69436105F1180200F1180325
:102F2000CBE62A69CAF818206A69CAF81C20183545
:102F30000AF12002A6E732467FE729463046019390
:102F4000FDF7D8FF019B7EE7A968CAF81010E96871
:102F5000CAF81410242A03D010350AF118026CE7BD
:102F60002A69CAF818206A69CAF81C2018350AF1BB
:102F7000200262E72807002010B50C46B1F90E10B8
:102F800000F0F6F9002803DB236D0344236510BD30
:102F9000A38923F48053A38110BD00BF2DE9F04124
:102FA0001646B1F90C201F46D3050C46054607D539
:102FB00000220223B1F90E1000F0C4F9B4F90C207C
:102FC000B4F90E1022F48052A2813B4632462846C4
:102FD000BDE8F04100F0A4B810B50C46B1F90E10F0
:102FE00000F0B0F9A389421C0EBF23F4805343F4D0
:102FF00080532065A38110BDB1F90E1000F008B90F
:10300000F8B50D461446064610B1836B002B4BD025
:10301000B4F90C20A369A36091B2080739D52369DC
:10302000002B36D0EDB289042F4615D52268616990
:10303000D31A8B421CDA0133A168501C0139A160FC
:103040002060157062699A421AD0A389DB0701D506
:103050000A2D15D03846F8BD616E42F4005221F4B5
:103060000051A281226861666169D31A8B42E2DB5A
:1030700021463046FFF730F940B922680123DBE7EB
:1030800021463046FFF728F90028E3D04FF0FF37FC
:10309000E0E721463046FFF70BF80028F6D1B4F9F7
:1030A0000C20236991B2BDE7FFF76EF9B0E700BFCE
:1030B000F0B5064685B01F4689B1104C104D246806
:1030C000646B002C08BF2C46D4F8E040A047431C9A
:1030D00003D100228A233A60336005B0F0BD0C466C
:1030E0000649074A0968496B002908BF114622466C
:1030F000D1F8E04001A9A047E9E700BFF8020020AD
:103100003C0B002021B1FF2A04D80A70012070472F
:10311000084670478A2303604FF0FF30704700BFB6
:1031200070B50D46084C114606461A46284600233F
:103130002360F9F7A5FE431C00D070BD2368002B67
:10314000FBD0336070BD00BF982000202DE9F8430C
:103150002C4D0646286898460F469146FFF7D4FC4A
:10316000294B1C68D4F84831002B3ED05A681F2ADE
:103170001CDC02F1010E76B103EB82010124C1F8DF
:103180008890D3F8880194402043022EC3F8880128
:10319000C1F8088123D00232C3F804E0286843F85C
:1031A0002270FFF7B3FC0020BDE8F883174B0BB388
:1031B0004FF4C870FDF7C2FA0346D8B1D4F84821DD
:1031C0000260002141600A46C4F848014FF0010E38
:1031D000C0F88811C0F88C11002EDCD0CCE7D3F8F1
:1031E0008C110C43C3F88C41D5E704F5A673C4F8E1
:1031F0004831BBE72868FFF789FC4FF0FF30BDE896
:10320000F88300BF380B0020104241003D07410009
:1032100038B5074C0023054608462360FAF732FA12
:10322000431C00D038BD2368002BFBD02B6038BD79
:103230009820002070B559B105460C4610B1836B3B
:10324000002B3CD0636ED80705D5B4F90C302BB9F0
:103250000026304670BDA38999053CD521462846F5
:10326000FEF79AFFE36A064633B1E16928469847BC
:103270000028B8BF4FF0FF36A3891A0622D4216B6D
:1032800041B104F14003994202D02846FFF7A2F968
:1032900000232363616C21B12846FFF79BF90023CB
:1032A0006364FFF79DF8636E0022DB07A2810ED5F1
:1032B000A06DFFF727FCFFF799F8304670BDFFF7C8
:1032C00063F8BFE721692846FFF784F9D7E7A06DC7
:1032D000FFF71CFCECE7A06DFFF716FCB4F90C300F
:1032E000002BBBD1666E16F00106B1D1A06DFFF7C1
:1032F0000DFC304670BD00BF38B50B46074C054687
:103300001146184600232360FAF7BFF9431C00D08A
:1033100038BD2368002BFBD02B6038BD98200020DF
:1033200038B5074C0023054608462360FAF7B2F982
:10333000431C00D038BD2368002BFBD02B6038BD68
:103340009820002070B50D46084C114606461A46D6
:10335000284600232360FAF79FF9431C00D070BD74
:103360002368002BFBD0336070BD00BF9820002085
:1033700070B50D46084C114606461A4628460023ED
:103380002360F9F763FD431C00D070BD2368002B58
:10339000FBD0336070BD00BF9820002053B94AB9FC
:1033A000002908BF00281CBF4FF0FF314FF0FF304D
:1033B00000F07AB9ADF1080C6DE904CE00F006F822
:1033C000DDF804E0DDE9022304B070472DE9F047A1
:1033D0008C460D460446089E002B51D18A42174662
:1033E0006DD9B2FA82FEBEF1000F0BD0CEF1200CE7
:1033F00001FA0EF520FA0CFC02FA0EF74CEA050C65
:1034000000FA0EF44FEA174A250CBCFBFAF81FFA33
:1034100087F90AFB18CC45EA0C4508FB09F3AB42D7
:103420000AD9ED1908F1FF3280F02381AB4240F256
:103430002081A8F102083D44ED1AA4B2B5FBFAF0D0
:103440000AFB105544EA054400FB09F9A14509D9D6
:10345000E41900F1FF3380F00A81A14540F20781B1
:1034600002383C44A4EB090440EA08400021002E45
:1034700061D024FA0EF4002334607360BDE8F08755
:103480008B4207D9002E54D0002186E8210008463F
:10349000BDE8F087B3FA83F1002940F08E80AB429B
:1034A00002D3824200F2FA80841A65EB0305012000
:1034B000AC46002E3FD086E81010BDE8F08712B968
:1034C0000127B7FBF2F7B7FA87FEBEF1000F34D140
:1034D000EB1B3A0C1FFA87FC0121B3FBF2F8250C19
:1034E00002FB183345EA03450CFB08F3AB4207D94E
:1034F000ED1908F1FF3002D2AB4200F2D1808046D4
:10350000ED1AA3B2B5FBF2F002FB105543EA0544F5
:103510000CFB00FCA44507D9E41900F1FF3302D2EB
:10352000A44500F2B8801846A4EB0C0440EA084019
:103530009DE731463046BDE8F087CEF1200405FA1C
:103540000EF307FA0EF720FA04F83A0C25FA04F401
:1035500048EA0308B4FBF2F14FEA184502FB1144B4
:103560001FFA87FC45EA044501FB0CF3AB4200FA65
:103570000EF409D9ED1901F1FF3080F08A80AB42D9
:1035800040F2878002393D44EB1A1FFA88F5B3FBFD
:10359000F2F002FB103345EA034500FB0CF3AB42AB
:1035A00007D9ED1900F1FF386FD2AB426DD902385F
:1035B0003D44EB1A40EA01418FE7C1F1200722FAAE
:1035C00007F88B4005FA01F448EA030320FA07FEE6
:1035D0004FEA134CFD404EEA040EB5FBFCF94FEAEE
:1035E0001E440CFB19551FFA83F844EA054509FBF4
:1035F00008F4AC4202FA01F200FA01FA08D9ED1817
:1036000009F1FF3043D2AC4241D9A9F102091D446E
:103610002D1B1FFA8EFEB5FBFCF00CFB10554EEA7D
:10362000054400FB08F8A04507D9E41800F1FF3570
:1036300029D2A04527D902381C4440EA0940A4EB0E
:103640000804A0FB02894C45C6464D4615D312D04E
:1036500056B1BAEB0E0364EB050404FA07F7CB404E
:103660001F43CC40376074600021BDE8F0871846E6
:10367000F8E69046E0E6C245EAD2B8EB020E69EB06
:1036800003050138E4E72846D7E7404691E781463D
:10369000BEE7014678E702383C4445E7084608E7BC
:1036A000A8F102083D442BE7704700BF010000006D
:1036B00002000000040000000800000010000000EC
:1036C000200000004000000080000000000080009A
:1036D00000000001000000020000000400000008DB
:1036E00000000010000000000000000000000000CA
:1036F00000000000000000000000000000000000CA
:10370000000000000000000000000000012801107F
:103710000203800253290351FF01026902026B1068
:10372000058000404011088102560009000F000882
:103730008202560009000F0002350002250103F045
:10374000AA1104C00040000AC2010A010A010A00CD
:10375000900203FF5A8102650B0EF9585F666D7483
:103760007B828990979EA5AC03F0AA1202D3200316
:10377000BF37BE02360003F0AA1104C500014000A5
:10378000012801100253290351FF01026902026B53
:103790001005800140401103F0AA1104C000400050
:1037A0000AC2010A010A010A0090022D70110000EC
:1037B000891080078003C0078003C003C002000394
:1037C000580020C637000D000F0011000818001027
:1037D000F0030C2000060B0B3308810256000B008F
:1037E000110008820256000B00110002350002256C
:1037F0000103F0AA1002D10203F0AA110AC2010AC1
:10380000010A010A00900203FF5A8102650B0EF9BA
:10381000585F666D747B828990979EA5AC03F0AA71
:103820001202D32003BF37BE02038102360003F029
:10383000AA1104C500014000012801100203800202
:1038400053290351FF01026900026B1005800040FB
:103850004011088104AC0010001000088204AC0084
:103860001000100002350002250103F0AA1002D159
:103870000203F0AA110AC2010A010A010A00908299
:1038800003F0AA1202D32003BF07BE03FF5A81022E
:10389000650B0EF9585F666D747B828990979EA5C3
:1038A000AC0236000000000001010203800253292F
:1038B0000351FF01026900026B10058000404011B6
:1038C00008810256000A00100008820256000A0011
:1038D000100002350002250103F0AA110AC2010AF4
:1038E000010A010A00900203F0AA1202D32003BFCA
:1038F00007BE03FF5A8102650B0EF9585F666D74AF
:103900007B828990979EA5AC03F0AA1105C4AA55A5
:10391000018004C5001FFF0001280110020381027D
:1039200053290351FF01026900026B102D70110031
:103930000089108009F004F804F804F804F8020083
:10394000041B002091BF0011000F0019000918008E
:1039500010F0030C2000060B0B330580013E3E11D6
:10396000088101E10006001000088201E100060064
:10397000100002250103F0AA1002D10203F0AA11DF
:103980000AC2010A010A010A00900203F0AA120207
:10399000D32003BF07BE03FF5A8102650B0EF958FF
:1039A0005F666D747B828990979EA5AC00000000D5
:1039B000012801100203810253290351FF0102690A
:1039C00000026B102D7011000089108009F004F8BE
:1039D00004F804F804F80200041B002091BF001151
:1039E000000F00190009180010F0030C2000060B4E
:1039F0000B330580013E3E11088101E100100010EB
:103A000000088201E1001000100002250103F0AA65
:103A10001002D10203F0AA110AC2010A010A010A26
:103A200000900203F0AA1202D32003BF07BE03FFD7
:103A30005A8102650B0EF9585F666D747B8289901E
:103A4000979EA5AC00000000565852303000000090
:103A5000302E322E313400005553415254000000B4
:103A60004661696C656420746F206372656174657A
:103A7000207573617274207461736B0D0A0000000D
:103A800048494420436F6D6D616E6473000000000F
:103A90004661696C656420746F206372656174654A
:103AA0002048494420636F6D6D616E642070726FB1
:103AB000636573736F72207461736B0D0A0000008D
:103AC000484944205265706F727400004661696C09
:103AD000656420746F206372656174652048494491
:103AE00020706572696F646963207265706F7274AB
:103AF000207461736B0D0A00302E322E31340000B9
:103B000056585244454C45544500000000FFFFFF05
:103B1000FFFFFF0009279550D2040000021E010498
:103B2000A5000078E7000000000000000000000091
:103B30000000010101010101010101010101010177
:103B40000101CAB40080F080187040209200FFFF8D
:103B50000000001EA5510080A00020A0402002040B
:103B6000FFFF0000001E0000000000000000000039
:103B70000000000000000000000000100000000035
:103B800000000000000000000000017570127900C4
:103B900000030014689F0080FF137F003F801F0018
:103BA000FF091F000F80010000000000000000005E
:103BB0000000000000000000000000000000000005
:103BC00000000000000000000000000000000000F5
:103BD00000000000000000000000000000000000E5
:103BE00000000000000000000000000000000000D5
:103BF00000000000000000000000000000000000C5
:103C000000000000000000000000B19000FFFFFF76
:103C1000FFFFFF0009273412D2040000FF20010437
:103C2000A5000078007875AA553BB22910505400C1
:103C30000000010101010101010101010101010176
:103C40000101000000100000000000000000000062
:103C50000000000000000010000000000000000054
:103C60000000000000000000001000000000000044
:103C70000000000000000000000000FC0042657928
:103C80006F6E640A202020202020015B70207907BD
:103C90000022091441B70E88DF137F003F801F0008
:103CA000EF0917000E8001007E00073A02928100A2
:103CB00008000000000000000000000000000000FC
:103CC00000000000000000000000000000000000F4
:103CD00000000000000000000000000000000000E4
:103CE00000000000000000000000000000000000D4
:103CF00000000000000000000000000000000000C4
:103D000000000000000000000000CA9000FFFFFF5C
:103D1000FFFFFF0009273412D2040000FF20010436
:103D2000A5000078007875AA553BB22910505400C0
:103D30000000010101010101010101010101010175
:103D40000101000000100000000000000000000061
:103D50000000000000000010000000000000000053
:103D60000000000000000000001000000000000043
:103D70000000000000000000000000FC0042657927
:103D80006F6E640A202020202020015B70207907BC
:103D90000022091439540F88DF137F003F801F0071
:103DA000EF0917000E8001007E00073A02928100A1
:103DB00008000000000000000000000000000000FB
:103DC00000000000000000000000000000000000F3
:103DD00000000000000000000000000000000000E3
:103DE00000000000000000000000000000000000D3
:103DF00000000000000000000000000000000000C3
:103E000000000000000000000000349000FFFFFFF1
:103E1000FFFFFF0009273412D2040000FF20010435
:103E2000A5000078007875AA553BB22910505400BF
:103E30000000010101010101010101010101010174
:103E40000101000000100000000000000000000060
:103E50000000000000000010000000000000000052
:103E60000000000000000000001000000000000042
:103E70000000000000000000000000FC0042657926
:103E80006F6E640A202020202020015B70207907BB
:103E9000002209141EF50A88FF0EFF003F801F0054
:103EA0007F071B000E8001007E00073A029281000E
:103EB00008000000000000000000000000000000FA
:103EC00000000000000000000000000000000000F2
:103ED00000000000000000000000000000000000E2
:103EE00000000000000000000000000000000000D2
:103EF00000000000000000000000000000000000C2
:103F000000000000000000000000869000FFFFFF9E
:103F1000FFFFFF0009273412D2040000FF20010434
:103F2000A5000078007875AA553BB22910505400BE
:103F30000000010101010101010101010101010173
:103F4000010100000010000000000000000000005F
:103F50000000000000000010000000000000000051
:103F60000000000000000000001000000000000041
:103F70000000000000000000000000FC0042657925
:103F80006F6E640A202020202020015B70207907BA
:103F90000022092839540F88DF137F003F801F005B
:103FA000EF0917000E8001001EF50A08FF0EFF0042
:103FB0003F801F007F071B000E8001007E00073A34
:103FC00002928100080000000000000000000000D4
:103FD00000000000000000000000000000000000E1
:103FE00000000000000000000000000000000000D1
:103FF00000000000000000000000000000000000C1
:1040000000000000000000000000E1907669646597
:104010006F5F70726F6300004661696C6564207445
:104020006F2063726561746520766964656F2070C6
:10403000726F636573736F72207461736B0D0A0026
:1040400070726F785F74696D656F75745F74696D98
:1040500065720000FF00FF00493243004661696C51
:10406000656420746F206372656174652049324312
:10407000207461736B0D0A0054494D45445F5354DD
:10408000415254004661696C656420746F2063720C
:10409000656174652074696D656420737461727400
:1040A0007570207461736B0D0A0000004144430079
:1040B0004661696C656420746F2063726561746524
:1040C00020414443207461736B0D0A004C45440049
:1040D0004661696C656420746F2063726561746504
:1040E000204C4544207461736B0D0A0046414E001C
:1040F0004661696C656420746F20637265617465E4
:104100002046616E207461736B0D0A0031323334C6
:10411000202020202020202020202020000000001F
:1041200049444C4500000000546D725100000000ED
:10413000546D72205376630000C20100C00000007D
:1041400000080000000000002D2D20426967736305
:104150007265656E204265796F6E64202D2D0A00B0
:10416000444953504C4159424F4152442056302EFD
:10417000342E32002D2D202573202D2D0A00000015
:104180002D2D2056657273696F6E202573202D2D9D
:104190000A00000031353A34393A33350000000066
:1041A0005365702031352032303233002D2D2043BD
:1041B0006F6D70696C65643A202573202573202D1E
:1041C0002D0A00005553424C6F6164004661696CD2
:1041D000656420746F206372656174652055534275
:1041E000204C6F61646572207461736B0D0A00006E
:1041F000737461636B206F766572666C6F772025D0
:10420000782025730D0A00006C6F676600000000BF
:1042100000030020303132333435363738394142EB
:1042200043444546000000003031323334353637E0
:10423000383961626364656600000000286E756C41
:104240006C29000020202020202020202020202059
:10425000202020203030303030303030303030309E
:104260003030303043000000504F534958000000B8
:104270002E000000002020202020202020202828A0
:104280002828282020202020202020202020202016
:104290002020202020881010101010101010101056
:1042A0001010101010040404040404040404041086
:1042B0001010101010104141414141410101010114
:1042C00001010101010101010101010101010101DE
:1042D00010101010101042424242424202020202EA
:1042E00002020202020202020202020202020202AE
:1042F000101010102000000000000000000000005E
:1043000000000000000000000000000000000000AD
:10431000000000000000000000000000000000009D
:10432000000000000000000000000000000000008D
:10433000000000000000000000000000000000007D
:10434000000000000000000000000000000000006D
:10435000000000000000000000000000000000005D
:10436000000000000000000000000000000000004D
:104370000000000000000000F8B500BFF8BC08BC59
:104380009E4670477921410029444000F8B500BF9E
:10439000F8BC08BC9E4670470544400030F0FF7FE3
:1043A0000100000030B482B0049C5BB31D4603687A
:1043B00043F480330360C9B241F0B4414160836883
:1043C0000193019B13F0010FF9D1002306E099003E
:1043D00001F58001096845F823100133A342F6D3A3
:1043E000D2B242F0B442426083680193019B13F061
:1043F000010FF9D0036823F480330360002002B07A
:1044000030BC70470220FAE70160704782B041601B
:1044100083680193019B13F0010FF9D0019800F01C
:104420000E0002B070470000714440007544400027
:10443000774440007B4440007F444000B944400042
:1044400009454000814440008544400091444000BB
:104450000180FFFFFFFF00000110FFFF0210FFFFC0
:104460000310FFFF0410FFFF0120FFFF0220FFFFEA
:1044700005000000010000000C3F41000A0101009E
:10448000807C797673706D6A6764615F5C5957549C
:10449000524F4D4B48464442403E3B3A3836343208
:1044A000302F2D2B2A282725242221201E1D1C1BBE
:1044B0001A181716151413121111100F0E0D0D0CDA
:1044C0000B0B0A090908080707060605050404047A
:1044D00003030303020202020101010101010000C2
:1044E00000000000000000010102020202020303BA
:1044F000030303030304040404040505050505067A
:1045000006060707070808080909090A0A0B0B0C21
:104510000C0D0D0E0F0F1011111213141515161787
:1045200018191B1C1D1E202122242527292A2C2E68
:1045300030323437393C3E4144474A4D5054575B42
:104540005F63676C70757A804747000054020020F3
:10455000C401002000000000CC01002068020020FF
:1045600009028500030100C032080B0002010100AE
:104570000209040000000101000209240100011EDB
:104580000001010C240201010200020300000009E5
:1045900024030201010001000904010000010200DE
:1045A00002090401010101020002072401020101C4
:1045B000000B2402010202100180BB0009058405E2
:1045C00000010100000725010000000009040200AD
:1045D0000103000000092111010001222600070546
:1045E00081034000040000001201000200000040AE
:1045F000BD3501010001010203010000940000200B
:10460000A80000207402002099A44000B9A4400032
:1046100011A54000BBA440000000000006FFFF09F8
:1046200001A10109020903150026FF007508954044
:10463000810209060907150026FF0075089540B19B
:1046400002C00000000300000000000000000000A5
:10465000000000000000000000000000000000005A
:1046600000000000000000000403090442696773B1
:10467000637265656E0000004265796F6E640001CB
:1046800000127A00AAAAAAAA0100000000030020D2
:104690000000000000000000EC050020540600208F
:1046A000BC06002000000000000000000000000028
:1046B00000000000000000000000000000000000FA
:1046C00000000000000000000000000000000000EA
:1046D00000000000000000000000000000000000DA
:1046E00000000000000000000000000000000000CA
:1046F00000000000000000000000000000000000BA
:1047000000000000000000000000000000000000A9
:104710000000000000000000000000000000000099
:104720000000000000000000000000000000000089
:104730000000000000000000000000000100000078
:10474000000000000E33CDAB34126DE6ECDE050048
:104750000B0000000000000000000000000000004E
:104760000000000000000000000000000000000049
:104770000000000000000000000000000000000039
:104780000000000000000000000000000000000029
:104790000000000000000000000000000000000019
:104AC00000000000280700202807002030070020F1
:104AD000300700203807002038070020400700205A
:104AE000400700204807002048070020500700200A
:104AF00050070020580700205807002060070020BA
:104B00006007002068070020680700207007002069
:104B10007007002078070020780700208007002019
:104B200080070020880700208807002090070020C9
:104B3000900700209807002098070020A007002079
:104B4000A0070020A8070020A8070020B007002029
:104B5000B0070020B8070020B8070020C0070020D9
:104B6000C0070020C8070020C8070020D007002089
:104B7000D0070020D8070020D8070020E007002039
:104B8000E0070020E8070020E8070020F0070020E9
:104B9000F0070020F8070020F80700200008002098
:104BA0000008002008080020080800201008002045
:104BB00010080020180800201808002020080020F5
:104BC00020080020280800202808002030080020A5
:104BD0003008002038080020380800204008002055
:104BE0004008002048080020480800205008002005
:104BF00050080020580800205808002060080020B5
:104C00006008002068080020680800207008002064
:104C10007008002078080020780800208008002014
:104C200080080020880800208808002090080020C4
:104C3000900800209808002098080020A008002074
:104C4000A0080020A8080020A8080020B008002024
:104C5000B0080020B8080020B8080020C0080020D4
:104C6000C0080020C8080020C8080020D008002084
:104C7000D0080020D8080020D8080020E008002034
:104C8000E0080020E8080020E8080020F0080020E4
:104C9000F0080020F8080020F80800200009002093
:104CA0000009002008090020080900201009002040
:104CB00010090020180900201809002020090020F0
:104CC00020090020280900202809002030090020A0
:104CD0003009002038090020380900204009002050
:104CE0004009002048090020480900205009002000
:104CF00050090020580900205809002060090020B0
:104D0000600900206809002068090020700900205F
:104D1000700900207809002078090020800900200F
:104D200080090020880900208809002090090020BF
:104D3000900900209809002098090020A00900206F
:104D4000A0090020A8090020A8090020B00900201F
:104D5000B0090020B8090020B8090020C0090020CF
:104D6000C0090020C8090020C8090020D00900207F
:104D7000D0090020D8090020D8090020E00900202F
:104D8000E0090020E8090020E8090020F0090020DF
:104D9000F0090020F8090020F8090020000A00208E
:104DA000000A0020080A0020080A0020100A00203B
:104DB000100A0020180A0020180A0020200A0020EB
:104DC000200A0020280A0020280A0020300A00209B
:104DD000300A0020380A0020380A0020400A00204B
:104DE000400A0020480A0020480A0020500A0020FB
:104DF000500A0020580A0020580A0020600A0020AB
:104E0000600A0020680A0020680A0020700A00205A
:104E1000700A0020780A0020780A0020800A00200A
:104E2000800A0020880A0020880A0020900A0020BA
:104E3000900A0020980A0020980A0020A00A00206A
:104E4000A00A0020A80A0020A80A0020B00A00201A
:104E5000B00A0020B80A0020B80A0020C00A0020CA
:104E6000C00A0020C80A0020C80A0020D00A00207A
:104E7000D00A0020D80A0020D80A0020E00A00202A
:104E8000E00A0020E80A0020E80A0020F00A0020DA
:104E9000F00A0020F80A0020F80A0020000B002089
:104EA000000B0020080B0020080B0020100B002036
:104EB000100B0020180B0020180B0020200B0020E6
:104EC000200B0020FFFFFFFF0000020074200020E5
:104ED000430000000000000000000000000000008F
:104EE00000000000000000000000000000000000C2
:104EF000430000000000000000000000000000006F
:104F000000000000000000000000000000000000A1
:104F1000430000000000000000000000000000004E
:104F20000000000000000000000000000000000081
:104F3000430000000000000000000000000000002E
:104F40000000000000000000000000000000000061
:104F5000430000000000000000000000000000000E
:104F60000000000000000000000000000000000041
:104F700043000000000000000000000000000000EE
:104F80000000000000000000000000000000000021
:104F900043000000000000000000000000000000CE
:104FA0000000000000000000000000000000000001
:104FB00005314100012C4100000000007442410015
:104FC000704241001C4141001C4141001C41410014
:104FD0001C4141001C4141001C4141001C41410059
:104FE0001C4141001C414100FFFFFFFFFFFFFFFF8D
:104FF000FFFFFFFFFFFF000001004153434949004D
:1050000000000000000000000000000000000000A0
:105010000000000000000000000041534349490027
:105020000000000000000000000000000000000080
:10503000000000000000000000000000CAA5784544
:00000001FF
